:020000040800F2
:1000000000200010AD490308ED01020889620008D4
:10001000E9010208E5010208E10102080000000010
:10002000000000000000000000000000DD010208E8
:10003000D901020800000000D5010208B97B0008C0
:10004000154A0308154A0308154A0308154A030808
:10005000154A0308154A0308510E01087D0F0108CF
:10006000410F0108050F0108C90E0108D930000829
:10007000C9300008B9300008A930000899300008DC
:100080008530000871300008154A0308154A030836
:10009000090C0208154A0308154A03088D0E0108C9
:1000A0000173000851730008F172000861730008C1
:1000B0004173000831730008154A0308154A030804
:1000C000154A0308154A0308154A0308154A030888
:1000D000154A030879FC0008C17C0008457C00082B
:1000E000150E0108154A0308C5010208154A030840
:1000F00011730008154A030821730008154A030804
:10010000000000000000000000000000154A030885
:10011000154A0308154A0308A13002088530020871
:100120005D300008493000083530000821300008F3
:100130000D300008154A0308000000000000000010
:10014000154A0308154A0308154A03080000000071
:10015000000000000000000000000000000000009F
:100160000000000000000000154A0308154A0308BB
:10017000154A030800000000000000000000000015
:0801800000000000154A03080D
:10018800002870B51EDB0928044620DD012303EB97
:1001980083035B00B0FBF3F2092AF8D87BB10E4E5B
:1001A800B4FBF3F00928CCBF57223022A6FB03E5A5
:1001B800024403FB1044EB0801F8012BF0D10023A3
:1001C8000B7070BD2D230B7040420131DBE73030DE
:1001D80001F8010BF3E700BFCDCCCCCC884230B49A
:1001E8004FF001042ED301FB04F4B0FBF4F58D426B
:1001F800F9D284B1AAB901E0B0FBF4F5092DCCBF5E
:10020800572230222A4404FB150003F8012BB4FBC3
:10021800F1F4002CF0D100221A7030BC7047B0FB0A
:10022800F4F5092DCCBF372230222A4404FB1500EF
:1002380003F8012BB4FBF1F4002CF0D100221A7062
:1002480030BC70470546002AEBD1D7E72DE9F047C7
:1002580014461D46064600234FF47A722046294666
:1002680034F0CCF9DFF840814B4A4C4F88FB003121
:100278000144C31782FB002EC3EB611188FB0128E0
:1002880087FB00278644464AC3EBEE2EC1EB011CD0
:1002980082FB0E29A0EB8C0C0744424A86F806C064
:1002A800C3EB27474FEAEE7C08EB010ACCEBA90C1D
:1002B80082FB07824FEAE1780CEB4C0CC8EB6A181A
:1002C800AEEBCC0EC8EB0818DFF8E0C086F804E007
:1002D800A1EB880171718CFB0010F917C1EBE212D8
:1002E80040F2B55101FB1272C3EBE050B2F5896FD1
:1002F8004FEA80073CDA40F2DA239A4242DCB2F550
:10030800B77FB4BF4FF0000C4FF0010C4FEA4C0917
:10031800DFF89C8009EB0C0308EBC3031FFA8CFE83
:10032800D88A09EB0C0108EBC10116310B2301E057
:1003380031F8020D824218DA013BF9D1CC4401238D
:1003480038F83C00B37007F2B2770132121ABE4493
:10035800F270A6F800E0204629464FF47A7200238E
:1003680034F04CF93281BDE8F0870133DBB2E9E7BC
:100378004FF0030EF44640F29650DFF834804FF009
:100388000609CEE74FF0020EDFF82480F44640F26B
:1003980029404FF00409C4E7C5B3A29107452EC20E
:1003A800ABAAAA2A73B06D1689888888792D03119B
:1003B800A85F030803685A1C02601970704700BFE1
:1003C8002DE9F047089C2578002B804689460CBF0C
:1003D8004FF0200A4FF0300A661C35B3002A29DD99
:1003E800334601E0024698B113F8011B501E00295C
:1003F800F8D1971E60B13D46013D51464046C84779
:100408006B1C002BF8DC257827EAE770013055B122
:10041800041B29464046C847301916F8015B002DD1
:10042800F7D1BDE8F087BDE8F087002A04DC28464C
:10043800BDE8F0870020EBE7571EDCE783684268D9
:10044800D0ED037A00EB83010133934281ED040A76
:10045800836004BF0023836000EB830393ED047A79
:10046800036870EE277A9A42C0ED037A77EEC77A6E
:10047800C0ED037A0CDA013307EE103AF8EEC76ADA
:10048800B7EE007A87EEA60A036030EE070A7047D7
:1004980007EE102AB8EEC77A87EE870A704700BFC2
:1004A80090ED057A90ED004AD0ED066AD0ED014A4C
:1004B800D0ED047A90ED035AD0ED025AA4EE007AFA
:1004C800B0EE406AB0EE470AB0EE667AA6EE247A3D
:1004D80067EEC07AA0EE457AE6EE257A80ED057AD9
:1004E800C0ED067A704700BFD0ED057A90ED013A6D
:1004F800D0ED003AD0ED064A90ED024A90ED077A29
:1005080090ED035A90ED086AD0ED045AC0ED067AD2
:10051800F0EE406A27EE830AC0ED056AA3EEA60A4C
:1005280080ED087AA4EE240AA5EE470AA5EEC60ACD
:1005380080ED070A704700BFD0ED007A90ED017A90
:1005480030EE670AE7EE007AB0EE670AC0ED007A8F
:10055800704700BF704700BF0A44914214D030B4BE
:100568000139551E41F2210211F8014F082380EA92
:10057800042004044CBF82EA40004000013B80B2E2
:10058800F7D18D42F0D130BC70474378007840EA0B
:10059800032010FB01F04FF4807190FBF1F000F3A1
:1005A8000F0000B270472DE9F74F6A4CDFF8A8E159
:1005B80023880091DEF80010B4F90480C3EB2112FF
:1005C8005B00C3EBE103B4F9021052435943131320
:1005D80008FB03F84FEAA83808EBE12101EB810298
:1005E800B1F5FA3802F180024FEAE1794FEA2223A5
:1005F80049F1FF39B4F908200193A8FB08AB08FBBF
:1006080009F30BEB430BA161D31702FB09F108FBBC
:100618000311A2FB08230B441F03160347EA1257D2
:10062800B4F90A2002FB0BF1D3170AFB03130546A2
:10063800A2FB0A011944020A42EA016292194FEA2E
:100648002123E6887B41003243F50043A2FB0601E3
:1006580006FB03114A10CB1752EA03016FD0B4F915
:100668001060B4F90E00F71706FB0BF10AFB07112F
:10067800A6FB0AAB8B4400FB09F6C11708FB016116
:10068800A0FB08898944DEF804104FEA4846C1F502
:10069800801E4FEA494747EAD8371AEB060AB4F9E9
:1006A8000C8076464BEB070BF71700264FEACE7007
:1006B800F90716EB0A064FEAC80741EA5E0147EB5D
:1006C8000B0740F6354E861B61EB0707A6FB0E01AC
:1006D8000EFB071133F092FFB4F916204E13470BA7
:1006E80047EAC14702FB06FED31707FB03EEA2FB4E
:1006F80007237344564307FB0366A2FB07233344CF
:10070800560E46EAC3163218B4F914604FEA636706
:1007180047EB01037143F71700FB0717A6FB00011E
:100728003944C60C46EA413692194FEAE147B4F912
:1007380012607B41100A40EA0360320112180DB1C1
:10074800120A2A60009B13B11A46019B136003B07A
:10075800BDE8F08F5C3D0020481E002070477047C0
:1007680010B5064C237A0BB9002010BD07F0DCF851
:10077800E368C01AD0F5FA50F6D410BD481E002020
:100788004FF40063838270474FF40063838270479D
:10079800012380F84530704707B5F7216A462FF0E6
:1007A8003BFD9DF801309DF800100C4A1B0143EAFF
:1007B80001339DF8021043EA111353609DF8043089
:1007C8009DF803101B0143EA01339DF8051043EA25
:1007D8001113136003B05DF804FB00BF481E00202E
:1007E80038B504460D46FFF7BBFF246808B107F08B
:1007F800E7F8054B00221A7249215B7A2A462046FF
:1008080010F056FC012038BD481E002070B4046862
:10081800037B2268022101FA03F31A4213D04269CA
:100828000A495C2000FB02124FF6FE765068528996
:10083800C5680068296831402960C168D24392B20E
:100848000A40C260636070BC704700BF4452002019
:1008580030B40A4B1D7875B1094B002003EBC50570
:100868001A6899885062D4682143D160083323F804
:10087800040CAB42F4D130BC704700BF24550020B3
:100888002855002010B40268047B11680223A34095
:10089800194209D00649406800240C7001684FF6D7
:1008A800FE742140016053605DF8044B704700BF3F
:1008B800C7480020014B18680FF084BAEC1E0020CE
:1008C8003122F42110F006BDF0B5836983B00546E6
:1008D80013B11A689B8813856869264F8389C324D6
:1008E8004FF47A734FF0060E6E464FF6FF710137DC
:1008F80003E0013B9BB28B421DD002899207F8D5D9
:1009080004734FF47A7302E0A3B28B4213D00289C6
:10091800D20703F1FF34F7D5027BD2B20EB13270A1
:100928000136BEF1000F08D00EF1FF3EFF24002F64
:10093800E3D03C78DBE710F09FFBAB6913B11A6892
:100948009B8893619DF805009DF801609DF8021051
:100958009DF803409DF804209DF8063041EA0621E1
:1009680043EA002342EA0422012029876A87AB87E9
:1009780003B0F0BD086003082DE9F04F89B090F886
:1009880055300390002B40F07985039BBF4CC04D38
:10099800DFF804931033184680226B21029310F07D
:1009A80099FCBC48DFF8F4E24FF0640A4FF0100CF1
:1009B8004FF47A76D9F80430C3F30803002B40F0DB
:1009C8005B84EFF31183002B40F056842168826822
:1009D80000BF23689942F9D12F6806FB07F39B1AD9
:1009E800B3FBF7F306FB013101270191D9F8043075
:1009F800C3F30803002B40F00584EFF31183002BA9
:100A080040F000842368816800BF22689342F9D1CE
:100A1800D5F800B006FB0BF2521AB2FBFBF206FB4C
:100A28000323019A9B1AB3F57A7FDFD3BAF1010A3F
:100A3800C0D1072268210298DFF85C92954E10F029
:100A480049FCDFF858C24FF0640A4FF010084FF421
:100A58007A77D9F80430C3F30803002B40F0F08309
:100A6800EFF31183002B40F0EB832168B26800BFDD
:100A780023689942F9D1286807FB00F39B1AB3FB56
:100A8800F0F307FB013101200191D9F80430C3F3D9
:100A98000803002B40F09983EFF31183002B40F0FB
:100AA80094832368B16800BF22689342F9D1D5F8CE
:100AB80000B007FB0BF2521AB2FBFBF207FB032351
:100AC800019A9B1AB3F57A7FDFD3BAF1010AC0D134
:100AD80052466B210298DFF8C09110F0FBFB6D487D
:100AE800DFF8B8E14FF0640A4FF0100C4FF47A7653
:100AF800D9F80430C3F30803002B40F06984EFF3FE
:100B08001183002B40F064842168826800BF236849
:100B18009942F9D12F6806FB07F39B1AB3FBF7F349
:100B280006FB013101270191D9F80430C3F308030A
:100B3800002B40F02D83EFF31183002B40F0288326
:100B48002368816800BF22689342F9D1D5F800B0C4
:100B580006FB0BF2521AB2FBFBF206FB0323019AC7
:100B68009B1AB3F57A7FDFD3BAF1010AC0D101220B
:100B78006B210298DFF8209110F0ACFB4548DFF8B4
:100B88001CE14FF00F0A4FF0100C4FF47A76D9F8A9
:100B98000430C3F30803002B40F0FD83EFF3118307
:100BA800002B40F0F8832168826800BF23689942CF
:100BB800F9D12F6806FB07F39B1AB3FBF7F306FB83
:100BC800013101270191D9F80430C3F30803002B40
:100BD80040F0C182EFF31183002B40F0BC82236800
:100BE800816800BF22689342F9D1D5F800B006FBAE
:100BF8000BF2521AB2FBFBF206FB0323019A9B1A73
:100C0800B3F57A7FDFD3BAF1010AC0D1039B02980A
:100C180093F84F30DFF88090042B34BF18221A2243
:100C28001B2110F057FB1B48DFF870E04FF00F0A4C
:100C38004FF0100C4FF47A76D9F80430C3F3080358
:100C4800002B40F0FE83EFF31183002B40F0F98373
:100C58002168826800BF23689942F9D12F6806FB92
:100C680007F39B1AB3FBF7F306FB01310127019148
:100C7800D9F80430C3F30803002B40F04F82EFF398
:100C88001183002B40F04A820AE000BFC47600209E
:100C9800C876002010E000E000ED00E0C0760020FB
:100CA8002368816800BF22689342F9D1D5F800B063
:100CB80006FB0BF2521AB2FBFBF206FB0323019A66
:100CC8009B1AB3F57A7FD3D3BAF1010AB4D11822AB
:100CD8001C210298DFF8E89210F0FCFAB648DFF819
:100CE800DCE24FF00F0A4FF0100C4FF47A76D9F887
:100CF8000430C3F30803002B40F08783EFF311831C
:100D0800002B40F082832168826800BF23689942E3
:100D1800F9D12F6806FB07F39B1AB3FBF7F306FB21
:100D2800013101270191D9F80430C3F30803002BDE
:100D380040F0D781EFF31183002B40F0D281236874
:100D4800816800BF22689342F9D1D5F800B006FB4C
:100D58000BF2521AB2FBFBF206FB0323019A9B1A11
:100D6800B3F57A7FDFD3BAF1010AC0D1039B0298A9
:100D780093F84E20DFF848921A2110F0ABFA8E480B
:100D8800DFF838E24FF00F0A4FF0100C4FF47A7684
:100D9800D9F80430C3F30803002B40F0A682EFF320
:100DA8001183002B40F0A1822168826800BF23686C
:100DB8009942F9D12F6806FB07F39B1AB3FBF7F3A7
:100DC80006FB013101270191D9F80430C3F3080368
:100DD800002B40F06981EFF31183002B40F0648110
:100DE8002368816800BF22689342F9D1D5F800B022
:100DF80006FB0BF2521AB2FBFBF206FB0323019A25
:100E08009B1AB3F57A7FDFD3BAF1010AC0D1039BED
:100E1800029893F85020DFF8A891192110F05AFA97
:100E28006548DFF898E14FF0640A4FF0100C4FF472
:100E38007A76D9F80430C3F30803002B40F03982DE
:100E4800EFF31183002B40F034822168826800BFE1
:100E580023689942F9D12F6806FB07F39B1AB3FB65
:100E6800F7F306FB013101270191D9F80430C3F3E8
:100E78000803002B40F0FB80EFF31183002B40F0B8
:100E8800F6802368816800BF22689342F9D1D5F8BB
:100E980000B006FB0BF2521AB2FBFBF206FB03236F
:100EA800019A9B1AB3F57A7FDFD3BAF1010AC0D150
:100EB800102237210298DFF8089110F00BFA3E480B
:100EC800DFF8F8E04FF00F0A4FF0100C4FF47A7685
:100ED800D9F80430C3F30803002B40F04082EFF345
:100EE8001183002B40F03B822168826800BF236891
:100EF8009942F9D12F6806FB07F39B1AB3FBF7F366
:100F080006FB013101270191D9F80430C3F3080326
:100F1800002B40F08F80EFF31183002B40F08A8084
:100F28002368816800BF22689342F9D1D5F800B0E0
:100F380006FB0BF2521AB2FBFBF206FB0323019AE3
:100F48009B1AB3F57A7FDFD3BAF1010AC0D13821F1
:100F58000298DFF86C80194F012210F0BBF916498E
:100F68004FF00F094FF0100E4FF47A70D8F8043094
:100F7800C3F30803002B40F0D481EFF31183002B57
:100F880040F0CF8122688E6800BF23689A42F9D169
:100F9800D5F800C000FB0CF39B1BB3FBFCF300FB74
:100FA800023301930126D8F80430C3F308032BBB9E
:100FB800EFF3118313BB05E010E000E0C0760020DA
:100FC80000ED00E02368D1F808A000BF2268934232
:100FD800F8D1D5F800B000FB0BFCACEB0A0CBCFB5D
:100FE800FBFC00FB03C3019A9B1AB3F57A7FDAD3A3
:100FF800B9F10109BAD109B0BDE8F08FEFF3118A50
:101008008EF312888A680B68DB0344BF3E608A68E7
:101018002368D7F800C05FFA8AFA8AF31188D5F8EE
:1010280000A09C4400FB0AF39B1AB3FBFAF300FBF5
:101038000C33D8E7EFF311888CF3128881680368C2
:10104800DB0344BFCEF8007081682368DEF8002017
:101058005FFA88F888F31188D5F800801A4406FBEF
:1010680008F35B1AB3FBF8F306FB023367E7EFF309
:1010780011888CF3128881680368DB0344BFCEF8BB
:10108800007081682368DEF800205FFA88F888F32A
:101098001188D5F800801A4406FB08F35B1AB3FBE5
:1010A800F8F306FB0233FBE6EFF311888CF31288A2
:1010B80081680368DB0344BFCEF800708168236849
:1010C800DEF800205FFA88F888F31188D5F80080E8
:1010D8001A4406FB08F35B1AB3FBF8F306FB02336A
:1010E8008DE6EFF311888CF3128881680368DB03BF
:1010F80044BFCEF8007081682368DEF800205FFAEC
:1011080088F888F31188D5F800801A4406FB08F39C
:101118005B1AB3FBF8F306FB02331FE6EFF3118803
:101128008CF3128881680368DB0344BFCEF8007033
:1011380081682368DEF800205FFA88F888F3118850
:10114800D5F800801A4406FB08F35B1AB3FBF8F3E2
:1011580006FB0233B3E5EFF311888CF3128881683C
:101168000368DB0344BFCEF8007081682368DEF8AB
:1011780000205FFA88F888F31188D5F800801A44AF
:1011880006FB08F35B1AB3FBF8F306FB023335E5FD
:10119800EFF311888CF3128881680368DB0344BF7E
:1011A800CEF8007081682368DEF800205FFA88F8BE
:1011B80088F31188D5F800801A4406FB08F35B1AF7
:1011C800B3FBF8F306FB0233C9E4EFF3118E88F39F
:1011D8001288B1683368DB0344BFCCF80000B168FB
:1011E8002368DCF800205FFA8EFE8EF31188D5F8AC
:1011F80000E01A4407FB0EF35B1AB3FBFEF307FB90
:1012080002335DE4EFF311888CF312888168036878
:10121800DB0344BFCEF8007081682368DEF8002045
:101228005FFA88F888F31188D5F800801A4406FB1D
:1012380008F35B1AB3FBF8F306FB0233FFF7F1BBC5
:10124800EFF3118288F31288B0683368D90303D5A5
:101258000123CCF80030B0682368DCF80010D2B263
:1012680082F311882A68194407FB02F31B1AB3FB9F
:10127800F2F307FB013106E4EFF311828CF31288D5
:1012880087680368D90303D50123CEF8003087683F
:101298002368DEF80010D2B282F311882A68194454
:1012A80006FB02F3DB1BB3FBF2F306FB0131FFF78E
:1012B8009BBBEFF311828CF3128887680368D9030C
:1012C80003D50123CEF8003087682368DEF80010C4
:1012D800D2B282F311882A68194406FB02F3DB1B99
:1012E800B3FBF2F306FB0131BDE5EFF311828CF39A
:1012F800128887680368D90303D50123CEF8003024
:1013080087682368DEF80010D2B282F311882A6851
:10131800194406FB02F3DB1BB3FBF2F306FB0131B6
:1013280050E5EFF311868EF31288D1F808C00B68E8
:10133800DA0303D501233B60D1F808C023683A6873
:10134800F6B286F311882E681A4400FB06F3A3EB65
:101358000C03B3FBF6F300FB0233019322E6EFF331
:1013680011828CF3128887680368D90303D5012397
:10137800CEF8003087682368DEF80010D2B282F316
:1013880011882A68194406FB02F3DB1BB3FBF2F34E
:1013980006FB0131B6E5EFF311828CF312888768FA
:1013A8000368D90303D50123CEF800308768236882
:1013B800DEF80010D2B282F311882A68194406FBBD
:1013C80002F3DB1BB3FBF2F306FB0131FFF7F9BBBA
:1013D800EFF311828CF3128887680368D90303D569
:1013E8000123CEF8003087682368DEF80010D2B2F7
:1013F80082F311882A68194406FB02F3DB1BB3FB4E
:10140800F2F306FB0131FFF78DBBEFF311828CF38A
:10141800128887680368D90303D50123CEF8003002
:1014280087682368DEF80010D2B282F311882A6830
:10143800194406FB02F3DB1BB3FBF2F306FB013195
:101448006FE4EFF311828CF3128887680368D9037D
:1014580003D50123CEF8003087682368DEF8001032
:10146800D2B282F311882A68194406FB02F3DB1B07
:10147800B3FBF2F306FB0131FFF7F8BB1C09013C93
:10148800052C03F00F0300F293805C4A32F8140035
:1014980040FA03F2D50740F18B80012505FA03F3E2
:1014A800013B184033F0FAF8554B564F1E5D064481
:1014B80017EBC6047CD057F83600B4F804E0038A6A
:1014C8001EEA03037FF461AA00F13842920A4E49EA
:1014D800E3718B5C03F01F025B092021022B05FAE4
:1014E80002F2A17100F08580032B7DD0012B64D01E
:1014F80006A90025CDF818E0079528F043FBA38836
:101508000398424AC260B3FA83F2C2F11F02511C27
:101518003ED0D1B201F0FC0303F1804303F58033E0
:1015280001F00301D3F808E04FEA81084FF00F0CEF
:1015380057F83610364F0CFA08F62EEA060600F170
:101548000C0E47F822E09E60D3F808E0314E324F87
:10155800C1F3872101FA08F141EA0E014FF00108B1
:10156800996008FA02FEB118C7F800E0082306A837
:10157800069291F868708DF81D308DF81E808DF8F0
:101588001C502EF0BBFE254AD35DF02B1ADCA38835
:10159800B3FA83F3C3F11F03581C3FF4F6A90122E1
:1015A80002FA03F31E490A6813430B60FFF7EDB90B
:1015B800039A164BD3600123F4E71A494B691A437F
:1015C8004A6195E7F319F02193F878308DF81430D3
:1015D80005A803238DF816508DF81780D1558DF87E
:1015E800153028F099FAD2E70E49CB691A43CA6137
:1015F8007EE70C498B691A438A6179E728880308D2
:1016080034880308FC7E00203C88030899070008FA
:1016180034220020A85F030814040140742200202B
:1016280000040140001002402DE9F04F4269B24C1D
:101638001388DFF8D082B14E23F040031B041B0C43
:10164800138013889BB223F0380343F030031380D0
:1016580013889BB283B043F040031380019006F0D7
:1016680063F9DFF8A4E2A649844610274FF47A7597
:101678000120DEF80430C3F30803002B40F01D817D
:10168800EFF31183002B40F018812368D1F80890FC
:1016980000BF22689342F8D1D8F800A005FB0AF2EF
:1016A800A2EB0902B2FBFAF205FB03239C45E0D04A
:1016B800019D2846FFF760F9AB6913B11A689B884A
:1016C8001385019B586940F2E93302E0002B00F0D2
:1016D80038810289013B12F0020F9BB2F6D06A23CF
:1016E800037340F2E93302E0002B00F02A810289FB
:1016F800013B12F0010F9BB2F6D0037B019B5869A6
:1017080040F2E93302E0002B00F01E810289013B20
:1017180012F0020F9BB2F6D01023037340F2E933A4
:1017280002E0002B00F010810289013B12F0010F4A
:101738009BB2F6D0037B019B9B6913B11A689B8807
:101748009361DFF8C4916E486C4F4FF0640A4FF014
:10175800100E4FF47A75D9F80430C3F30803002B40
:1017680040F0D480EFF31183002B40F0CF80216844
:10177800826800BF23689942F9D1D8F8006005FB58
:1017880006F39B1AB3FBF6F305FB01310126009122
:10179800D9F80430C3F30803002B56D1EFF31183B3
:1017A800002B52D12368816800BF22689342F9D187
:1017B800D8F800B005FB0BF2521AB2FBFBF205FB9E
:1017C8000323009A9B1AB3F57A7FE1D3BAF1010A91
:1017D800C1D1019B4A4D5A69484F138823F04003F1
:1017E8001B041B0C1380138823F038031B041B0CE9
:1017F800138013889BB243F04003138006F094F8DB
:10180800DFF804C181464FF0100E4FF47A760120BC
:10181800DCF80430C3F30803002B31D1EFF3118354
:1018280073BB2368A96800BF22689342F9D1D8F82E
:1018380000A006FB0AF2521AB2FBFAF206FB0323D7
:101848009945E5D003B0BDE8F08FEFF3118C8EF326
:10185800128881680368DA0344BF3E6081682368A0
:101868003A685FFA8CFC8CF31188D8F800C01A44E7
:1018780005FB0CF35B1AB3FBFCF305FB0233A0E793
:10188800EFF311818EF31288D5F808A02B68DB03DB
:1018980044BF3860D5F808A023683A68C9B281F314
:1018A8001188D8F800101A4406FB01F3A3EB0A03C9
:1018B800B3FBF1F306FB0233C2E7EFF3118987F3B9
:1018C8001288D1F808A00B68DB0344BF3060D1F858
:1018D80008A0236832685FFA89F989F31188D8F873
:1018E80000901A4405FB09F3A3EB0A03B3FBF9F3D1
:1018F80005FB0233DAE600BFC4760020C07600207C
:1019080010E000E0C876002000ED00E0EFF311825F
:101918008EF3128886680368D90302D501233B60D9
:10192800866823683968D2B282F31188D8F8002013
:10193800194405FB02F39B1BB3FBF2F305FB0131D2
:1019480024E70FF099FBD9E60FF096FBF3E600BF0A
:1019580010B490E80600047B40690223A3404B6062
:1019680013685DF8044B4FF6FE710B4013600EF0E0
:10197800BDB9F8B5174D2B78A52B28D16B78BE2BA0
:1019880025D1022229464FF6FF70FEF7E5FD124FDA
:10199800AC1C22884AB1A618BE4218D2052A16D90C
:1019A8002146FEF7D9FD3446F3E721460222FEF729
:1019B800D3FD0222A118FEF7CFFD0634074B641BA6
:1019C8001C8041F60F53C31A58425841F8BD0020F5
:1019D800F8BD00BF00F0030800000408162D002021
:1019E8002DE9F04FDFF848914C4F8BB00326A7EB59
:1019F80009071822002104A834F063FA484BCDF8EF
:101A0800109005971A69120604D5464A5A6002F1E1
:101A180088325A6001228DF824203422DA60424B41
:101A2800424C1B88ADF800300222694604A80FF02A
:101A3800EDFD022269464FF6FF70FEF78DFDDFF8D7
:101A4800F4A080464FF0000B544536D30AAC00256D
:101A580024F8245D0222214604A80FF0D7FD0222B3
:101A680021464046FEF778FD40BAC043ADF808006D
:101A7800022202A904A80FF0C9FD079860B106ABBD
:101A8800C0F104022946184434F01BFA069904A848
:101A98000FF062FD079508909DF82430089A23B14D
:101AA8001F490B6943F080030B61013E2DD0002ACA
:101AB8009FD1FFF75EFF50B32CE065888DF80DB01D
:101AC800C5F30B05AB1DADF808302388C3F30B0233
:101AD800ADF80A201B0B062202A904A88DF80C30C9
:101AE8000FF094FD062202A94046FEF735FD616815
:101AF80080462A4604A80FF089FD616840462A46B8
:101B0800FEF72AFD143480469EE7002AD1D005202E
:101B180004F01EFC0BB0BDE8F08F00BF0000040805
:101B280000200240230167452760030898C1030885
:101B380000F003080CC603080378202B024600F1C6
:101B48000100F9D0092BF7D02D2B2CD02B2B03BF5C
:101B58005378B7EE000A0246B7EE000AA3F1300147
:101B6800C8B209289FED467A10D8F2EE046A07EE4B
:101B7800901AF8EEE77A12F8013FE7EE267AA3F119
:101B88003001C8B20928B0EE677AF0D92E2B4CD0B4
:101B980003F0DF03452B0BD0F7EE007A67EE276AD8
:101BA80020EE260A70475378BFEE000A0246D5E7B2
:101BB80010B451782D2959D02B290ABF9178501C7F
:101BC800901C0024A1F13003092B53D8002303EB08
:101BD800830301EB430310F8011FA1F13002092A26
:101BE800A3F13003F3D9B3F59A7F28BF4FF49A7362
:101BF800072B42D9DFED236A1A46F7EE007A083A36
:101C0800072A67EEA67AFAD803F007032BB1F2EE9B
:101C1800046A013B67EEA67AFBD124B3C7EE276AB4
:101C28005DF8044B20EE260A70475378A3F1300183
:101C3800C8B2092802F10102AAD8F2EE046AF0EE4D
:101C4800665A07EE901AF8EEE77A12F8013F87EE27
:101C5800A66AA3F13001C8B2092866EEA56A37EE74
:101C6800067AEED994E767EE276AD9E7901C91784F
:101C78000124A7E7F7EE007ACFE7F7EE007AC5E789
:101C88000000000020BCBE4CB5EEC00ADFED317A82
:101C9800F1EE10FACCBF30EE270A30EE670ADFED1E
:101CA8002E7A20EE270A30B5FDEEC07A87B017EEFF
:101CB800904A054684EAE470002303A9A0EBE47087
:101CC80001930093029328F0C1FE002CACBF20239F
:101CD8002D2303A88DF8003031F0C6FF012803A991
:101CE80024D002282DD0032805BF30236846684633
:101CF8008DF8013034F0EDF8684631F0B5FF03385F
:101D0800C4B222466946284634F01AF900232B55F6
:101D1800284631F0A9FF2E22431C2A540DEB04015A
:101D2800E81834F0F3F8284607B030BD3023684689
:101D38008DF801308DF802308DF8033034F0C9F891
:101D4800DAE7302368468DF801308DF8023034F038
:101D5800C0F8D1E76F12033A00007A442DE9F04148
:101D6800064615460846B6FBF2F43CB905FB146472
:101D7800124B1B5D00F8013BBDE8F081B4FBF2F7A4
:101D880067B90E4B05FB174705FB1464DA5D00F8CD
:101D9800012B1B5D00F8013BBDE8F081B7FBF2F8B1
:101DA800B8F1000F02D04046FFF7D8FF05FB1878BE
:101DB800024B13F8082000F8012BE3E7C88A030850
:101DC800104B2DE93048D3E9004554EA05020BD100
:101DD8000346012200201871587198719A70DA70C0
:101DE80018801881BDE83088074B1A6814EB020B7D
:101DF80045F1000C5A466346FEF728FA0120BDE873
:101E0800308800BFA01E0020C4760020F0B40288ED
:101E18008578154FC37804794179A2F2B27202F03D
:101E2800030606EB4606013D05EB8605013B37F840
:101E380015608579008940F2B557920807FB023290
:101E4800931903EB430304EBC303C3EB031301EB45
:101E58008303C3EB031305EB830300214FF47A726A
:101E6800C2FB0301F0BC7047A85F0308FAB170B465
:101E78008E18044603E0101A14D1B14214D014F895
:101E8800012BA2F14103192B11F8013BA3F14105E4
:101E980098BF2032192D03F12000ECD9D01A01D1B6
:101EA800002BEAD170BC7047002070BC7047104608
:101EB800704700BF4FF0FF32FFF7D8BFA0F16103B2
:101EC800192B98BF20387047A0F14103192B98BFF0
:101ED80020307047202805D0093804288CBF0020FE
:101EE8000120704701207047613819288CBF0020F5
:101EF80001207047413819288CBF00200120704705
:101F0800303809288CBF002001207047A0F1300329
:101F1800092B07D920F02000413819288CBF002050
:101F2800012070470120704730B402681146531CE5
:101F3800036011F8024B0160D31C51780360937859
:101F4800151D05601B0443EA0123D078234343EAA7
:101F5800006030BC704700BF0368591C1A46016016
:101F680012F8021B0260587841EA0020704700BF4F
:101F780003685A1C02601878704700BF38B50446D9
:101F88000068154632F00CFE22682A44226038BDEB
:101F9800036810B40A0A5C1C04601A7003685A1CAF
:101FA800026019705DF8044B704700BF03685A1C43
:101FB800026010B4197003680A0A5C1C04601A7085
:101FC80003680A0C5C1C04601A700368090E5A1C2A
:101FD800026019705DF8044B704700BF03685A1C13
:101FE800026019700368090A5A1C02601970704768
:101FF8002DE9F047002488B080460F461E46A146CA
:1020080005AD531C0393117839B3252933D1931C9B
:10201800CDF810900393507830284ED04FF0000A36
:10202800A0F13003DBB2092B42D96C2819D06428FF
:1020380000F0938024D825281CD063D9582876D05E
:1020480063281BD131784046B847039A531C039341
:102058001178043601340029D7D1204608B0BDE8EC
:10206800F087039B5A1C03921B78642B7CD02AD8D8
:10207800252B54D1252140460134B847039AC0E79F
:10208800732833D044D975284FD106F1040E30682F
:102098002B4600220A217646FEF7A0F8049A0095FE
:1020A800534639464046FEF78BF9039A0444A8E79D
:1020B80004AA03A92EF05AFFB7E7D31C039390781C
:1020C8004FF0010AACE7732B10D05BD9752B3AD0CF
:1020D800782B96D1A3F15802B2FA82F230685209ED
:1020E8002B4610210436FEF779F8D7E73368049AAF
:1020F8000093394600234046FEF762F9043604444B
:10210800039A7EE70028B9D1204608B0BDE8F087D9
:102118006E28B3D1039A336804361C6071E72AD954
:10212800582BD7D0632B8DD06BE77828A6D1A0F198
:102138005802B2FA82F2306852092B461021FEF793
:102148004DF80436AAE706F1040E30682B46002243
:102158000A217646FEF742F8A0E7331D3068294683
:102168001E46FEF70DF899E7331D306829461E46CE
:10217800FEF706F892E7002B7FF443AF204608B03D
:10218800BDE8F0876E2BC6D03BE700BF0EB400B5A4
:1021980084B005AB019053F8042B0649039301A8BA
:1021A800FFF726FF019B00221A7004B05DF804EBCC
:1021B80003B07047BD0300082DE9F04707468CB00F
:1021C8001E469246002A6AD1154614460A8840F2ED
:1021D800B1739A423AD98B78581E0B2836D891F8A1
:1021E80003E00EF1FF301E2830D891F804C0BCF18E
:1021F800170F2BD891F80590B9F13B0F26D888799D
:102208003B2823D8B1F80880B8F57A7F1ED24FF062
:102218000108002E34D109890491002CB4BF2D2166
:102228002B21002CB8BF6442039005910795CDF887
:102238000890CDF804C0CDF800E0384606942F4940
:10224800FFF7A4FF40460CB0BDE8F087002301214A
:1022580018468E46ADF824308DF828308DF8293090
:102268008DF82A30ADF82C3099469C461A46984687
:102278008DF826108DF827100B4609A9002ECAD014
:102288000390CDF80890CDF804C0CDF800E03846AA
:102298001B49FFF77BFF40460CB0BDE8F087194C9F
:1022A80084FB0234A318D417C4EB6314C4EB0415DD
:1022B800A2EB85052DB2002D0846B8BF6D42FFF789
:1022C800A5FD4FF47A7200238046894632F096F9CC
:1022D8003C230AFB030A4FF47A720023404649461E
:1022E80032F08CF94FF47A7192B20023C1FB0A23C1
:1022F80009A8FDF7ABFF24B209A967E7108B03080B
:10230800F08A0308898888880FB430B583B006AB93
:102318000B490C4853F8042B096800680193FFF730
:1023280067FE094C0546206803685B6998470028E2
:10233800F9D0284603B0BDE8304004B0704700BF6C
:10234800E82A0020EC2A0020EC1E0020DFED2B7A82
:10235800B4EEE70AF1EE10FA4ADDDFED296A9FEDE7
:10236800297A01E0B0EE670AB4EEC70AF1EE10FA76
:1023780070EE667AF6DC9FED247AF4EEC77AF1EE19
:1023880010FA38D5DFED1E6A9FED207A01E0F0EEF5
:10239800407AF4EEC77AF1EE10FA37EEA60AF6D4D0
:1023A800DFED1B7AB4EEE70AF1EE10FA14DDDFED8B
:1023B800137A37EEC00A60EE006A9FED166A9FED49
:1023C800167ADFED167AA6EE867A20EE266AE6EE13
:1023D800877AA6EE270A7047DFED117AB4EEE70A8E
:1023E800F1EE10FA44BFDFED087A37EEC00AE2E7F3
:1023F800F0EE407ABFE7B0EE670AD1E7DB0F49405D
:10240800DB0FC940E4CB1641DB0F49C0E4CB16C152
:10241800DB0FC93F92E741B99730083C15A82ABE9F
:10242800DB0FC9BF09B909E0194690FBF1F301FBBD
:1024380013030846002BF7D1084670470146FBE70F
:1024480007EE901AF8EE677A9FED837A27EE800AF6
:1024580020EE070AFDEEC07A17EE903A2033402BA3
:1024680000F28C80DFED7D7AB4EEE70AF1EE10FA27
:1024780040F3E880B0EE407A9FED796ADFED796A43
:1024880001E0B0EE677AB4EEE67AF1EE10FA77EE94
:10249800467AF6DC9FED747AF4EEC77AF1EE10FA1C
:1024A80040F1CD809FED6E6ADFED706A01E0F0EEDD
:1024B800477AF4EEE67AF1EE10FA37EE867AF6D439
:1024C800DFED6B7AB4EEE77AF1EE10FA51DCDFED6E
:1024D800697AB4EEE77AF1EE10FA44BFDFED627A7A
:1024E80037EEC77A27EE076ADFED635ADFED637AC6
:1024F800DFED636A9FED635AE6EE257A67EE065ACA
:10250800E6EE276AF7EE007AA5EEA67AF0EE675AAD
:10251800E7EE055AE7EE457A87EEA55ADFED547ADD
:1025280030EE277AFDEEC76A16EE903A2033402B3C
:1025380029D99FED557AF6EE006AB7EE006AF7EEF4
:10254800004AC4EEA57A0023836143610362C36134
:1025580080ED045A67EEA66A27EE866A27EE877A28
:10256800C0ED006AC0ED026A80ED016A80ED037A71
:102578007047DFED3A7A37EEC77AB3E7B7EE005A1D
:10258800F0EE455ACAE7B4EEE70AF1EE10FA5FDD5D
:102598009FED336ADFED336A01E0B0EE677AB4EE9F
:1025A800E67AF1EE10FA77EE467AF6DC9FED2E7AAF
:1025B800F4EEC77AF1EE10FA47D59FED296ADFED00
:1025C8002B6A01E0F0EE477AF4EEE67AF1EE10FAC3
:1025D80037EE867AF6D4DFED267AB4EEE77AF1EEB6
:1025E80010FA27DCDFED237AB4EEE77AF1EE10FA81
:1025F80044BFDFED1D7A37EEC77A27EE076ADFEDB5
:102608001E4ADFED1E6ADFED1E7AE6EE246A67EEEB
:10261800064AE6EE267AB7EE006AA4EEA77AF6EE48
:10262800006A36EE476AF8EE007A27EE277A66EEF9
:10263800266A84E7DFED097A37EEC77ADDE7B0EE80
:10264800677A3DE7F0EE407A24E7B0EE677AC2E7B2
:10265800F0EE477AAAE700BF27D4D236DB0F49400D
:10266800DB0FC940E4CB1641DB0F49C0E4CB16C1F0
:10267800DB0FC93FDB0FC9BF92E741B99730083C70
:1026880015A82ABEF304353F0000008070B4066820
:102698008E4217D90139751E002311F8014F0822FF
:1026A800634013F0800F4FEA430318BF83F0D5034C
:1026B800013ADBB2F5D18D42EFD1721C0260337062
:1026C80070BC70470023F8E710B44C09012250F899
:1026D800243001F01F0102FA01F10B4340F82430C5
:1026E8005DF8044B704700BF4B0901F01F0150F81B
:1026F8002320012303FA01F1114214BF18460020D8
:10270800704708B50EF02EFD0A2005F059F9012092
:1027180008BDF8B50F4D46686A721446027A0F462E
:1027280042F0800225213046FFF7EBFF3A4626218A
:102738003046FFF7E6FF04F00F0242F0800227213F
:102748003046FFF7DEFF05F0EFF8E8600120287259
:10275800F8BD00BF481E002070B50478032C0E4653
:10276800154603D0BDE870400EF0B4BD4468027A47
:1027780025212046FFF7C5FF324626212046FFF7D0
:10278800C0FF2A4663212046FFF7BBFF812227218D
:102798002046FFF7B6FF012070BD2DE9F04104780F
:1027A800032C884617461E4621D14468027A252103
:1027B80042F080022046FFF7A4FF42462621204629
:1027C800FFF79FFF06F00F0242F080022721204604
:1027D800FFF797FF042005F04DF972B649213346FB
:1027E8003A4620460EF064FC62B6BDE8F081BDE8CA
:1027F800F0410EF0FBBC37B500F10C040546002291
:102808000A212046FFF7A8FF0F220A212046FFF7DA
:10281800A3FF01AA032310212046FFF7BEFF9DF85E
:10282800043080336B839DF805308033AB839DF88B
:1028380006308033EB8300220A212046FFF78CFF05
:102848000DF10302012302212046FFF7A6FF012311
:102858000DF1030209212046FFF79FFF11220A21EB
:102868002046FFF779FF012003B030BD2DE9FF476F
:10287800037B0546884600F10C061BB1022B06D9DE
:10288800032B3DD00024204604B0BDE8F087012387
:102898000DF1070202213046FFF77FFF0028F1D033
:1028A8009DF80730D907EDD5072302AA0321304642
:1028B800FFF773FF0446002CE4D09DF80E70112238
:1028C8000A213046FFF748FF3B07DBD4B5F91A1059
:1028D80002A8FDF75AFE4042A8F80000B5F91C10FE
:1028E8000DF10A00FDF751FE4042A8F80200B5F9C3
:1028F8001E1003A8FDF749FE4042A8F80400C2E7ED
:10290800224F4FF0010A0024B9463B7C012B1BD013
:102918000FD3022BCFD1FDF723FF81460028B1D179
:1029280002A905F11000FDF75BFF87F81090044637
:10293800C1E73B7A23B9012202213046FFF7E9FEBD
:10294800012389F810309DE7FDF70AFF002899D187
:1029580002A905F11000FDF743FF9DF80830044671
:1029680008B1DA0707D4002389F81030BAF1000F4C
:1029780088D09A46C9E73B7A23B907220321304613
:10298800FFF7C7FE022389F810307BE7481E0020B6
:10299800028822F040021204120C0280028822F0FF
:1029A80038031B041B0C59B141F48071002991FABA
:1029B800A1F2B2FA82F108BF4FF0FF310139C90024
:1029C8000B439BB2038003889BB243F04003038010
:1029D800704700BF08B540F2E93300E09BB10289B7
:1029E800013B12F0020F9BB2F8D0017340F2E933B9
:1029F80000E043B10289013B12F0010F9BB2F8D00D
:102A0800007BC0B208BD0EF037FBC0B208BD00BFE6
:102A1800F8B584894FF6FF764FF47A742BB311B367
:102A28000F78013101E0B44217D00589013CAD07A8
:102A3800A4B2F8D507734FF47A7402E0BCB2B4427A
:102A48000BD00589ED0704F1FF37F7D5057BEDB20B
:102A58000AB115700132013BE0E70EF00DFB0030C2
:102A680018BF0120F8BDFF27DFE70120F8BD00BF30
:102A7800F0B55B4B5B4A97B01968914200AF00F024
:102A8800A3805949594A00234FF47000C1F88800BF
:102A98003B607B60136843F48033136003E03B685A
:102AA800B3F5A04F09D0136803F400337B603B688B
:102AB80001333B607B68002BF1D04C4B1B6813F44F
:102AC800003318BF01237B607B68012B52D0464C32
:102AD800464B474AE260474A596A11605A6A42F0CF
:102AE80080725A625A6942F4FC025A610025032234
:102AF80007F10801012341F6FF764FF09040FD6091
:102B0800BE603A73BB7327F03DF84FF6FF7307F1C9
:102B180008013948BB6027F035F807F10801374844
:102B2800374E27F02FF807F10801364827F02AF822
:102B380007F10801344827F025F807F10801334860
:102B480027F020F807F1080027F076F8BB6830492D
:102B5800304AA1FB031330499B0CF0204FF0070EBD
:102B68005C370B60566084F823009560C2F800E07B
:102B7800BD46F0BD294A1D4B122111605A685A60A2
:102B88005A685A605A6842F480625A605A6822F455
:102B98007C125A605A6842F4E8125A601A6842F085
:102BA80080721A601A689201FCD559680F4A21F0A0
:102BB80003015960596841F002015960536803F0F4
:102BC8000C03082BFAD182E700221A6062B6144B74
:102BD8001B6883F30888134B1B689847FEE700BF00
:102BE800FC9F0020EFBEADDE00ED00E000100240CB
:102BF8000005FA0590550020000400480008004828
:102C08003F190100000C004800100048001400485B
:102C180083DE1B4310E000E0C8760020002002405D
:102C280000D8FF1F04D8FF1F064A002351688142BD
:102C380002F11C0204D001330C2BF7D1002070479D
:102C4800D8B270474C00002070B50F4C0F4DC0EB48
:102C5800C00004EB8004686926693043686182B06B
:102C68009209667BA1600025012101A863618DF8A6
:102C780004608DF805208DF806508DF8071026F0B1
:102C88004BFF02B070BD00BF4C0000200010024096
:102C9800074BC0EBC00030B403EB8000054C05695E
:102CA80063692B4363610176427630BC704700BF8D
:102CB8004C000020001002402DE9F04F554C54F80C
:102CC800204083B0002C60D0A56D1F469046524B23
:102CD8006A682265A160236004F15E014FF4807385
:102CE80004F5AF726161A261E36023610646287E44
:102CF80029F0B4FEE86858B1FFF796FF721CD2B20B
:102D08000C21FFF7C5FF236DEA6862632433E3648F
:102D1800A86890B1FFF788FF721C8146D2B20B21D8
:102D2800FFF7B6FF2346EA7E3C494846FFF78CFF8B
:102D3800236DAA68A2632833A36494F85D000DF09C
:102D4800D9FB814694F85C000DF0D4FB3A07824623
:102D580095F819B01DD5B9F1000F1AD017F0110F59
:102D68004FF00B0306F1010614BF4E213E2189F8EE
:102D7800063089F807605A4648460DF07FFCFB0785
:102D880043D5636B6BB3A36B5BB3204603B0BDE85D
:102D9800F08F17F0010F0CBF2E274E2718F0020FE7
:102DA8000DD0B9F1000F0AD00B22731C89F8062048
:102DB80089F8073048465A4639460DF05FFC18F046
:102DC800010FDED0BAF1000FDBD001360C238AF8F0
:102DD80007605A4639468AF8063050460DF04EFCD0
:102DE800CFE72B7FAA7E8DF804209B0900210122C2
:102DF80001A88DF805308DF806108DF8072026F00B
:102E08008BFE204603B0BDE8F08F48460DF0C4FFA6
:102E1800B7E700BFF42A00202C60030859190008FE
:102E280000B97047F0B595B005462AF09BF86C4E8E
:102E3800C368026832600446002B00F0C38028464D
:102E48000DF058FB674B586118B129220023827195
:102E5800C371227A644D2E210DF010FC306804F005
:102E6800F3FB29F0FBFD3068604A038823F0010377
:102E78001B041B0C038014A91E232B8001270F237E
:102E88000025138021F84C7D2D230293ADF80C50BA
:102E9800ADF80650ADF80E502AF012F8E379ADF807
:102EA800145060229907ADF816500695ADF81C50DD
:102EB800ADF81E50ADF82050ADF82250049200F144
:102EC800838013F0010F0CBF002202224FF480739D
:102ED800ADF81470ADF81C20ADF82030002304AA1A
:102EE80061793068069304F005F861793068404FDD
:102EF80029F0C6FF33685A6C42F400425A641A88B3
:102F080092B242F080021A80E2796079196A9207D7
:102F18004CBF04220122824021EA02011962196A87
:102F28000A431A621A8892B242F001021A80207C7F
:102F380000222921FFF7ACFE2E49207C00236022C5
:102F4800FFF782FEE068386026F052FD38680368B3
:102F58004FF6FE721340036026F04AFD09A826F0DA
:102F680019FD33686279244938680A913433134467
:102F7800099380221023002509A940F22A3E0E92C7
:102F88000B934FF400724FF400530D951095139561
:102F980011950F921293ADF830E026F009FD627991
:102FA80033680C2A98BF1549D86898BF31F8125071
:102FB8003A6813490543DD601368012043F00203B2
:102FC8001360087015B0F0BD13F0010F0CBF2A464E
:102FD80008220423ADF81E20ADF816307EE700BFA6
:102FE80090820020481E00208682002084820020D3
:102FF8008C8200208D08000820490020C87F030823
:10300800888200200348D0F83C3113B100F59A704B
:10301800184770474C0000200348D0F8203113B1FE
:1030280000F58C70184770474C0000200348D0F812
:1030380004310BB1FC301847704700BF4C0000202A
:103048000348D0F8E8300BB1E0301847704700BFAC
:103058004C0000200348D0F8CC300BB1C4301847DE
:10306800704700BF4C0000200348D0F8B0300BB1C7
:10307800A8301847704700BF4C0000200348D0F81C
:1030880094300BB18C301847704700BF4C000020BB
:103098000248836F0BB17030184770474C0000200E
:1030A8000248C36D0BB15430184770474C000020DC
:1030B8000248036C0BB13830184770474C000020A9
:1030C8000248436A0BB11C30184770474C00002077
:1030D8000248836803B11847704700BF4C000020BE
:1030E800F8B505015A4C5B4B625961199A4204EBD9
:1030F800050704BF01230B730646387A29F0AEFC96
:103108003B7A03F01F015B090122022B02FA01F24C
:1031180078D0032B71D0012B67D063190136187949
:103128000DF0E8F9F6B2074610B11223C6718371A3
:10313800631958790DF0DEF910B11323C671837144
:10314800631998790DF0D6F910B11423C6718371FB
:1031580066190E21F27938460DF090FA70790DF063
:10316800C9F9F2790E210DF089FAB0790DF0C2F99A
:10317800F2790E210DF082FA6359374A934251D001
:10318800344A934259D0354A934240D02C44227B4A
:10319800002A2FD1012002249A8822F48052120496
:1031A800120C9A80998889B241F4805199801A88C2
:1031B80002F4415242F44572024322431A809A882B
:1031C80022F470621204120C42F4E0629A809A8B24
:1031D80022F400621204120C07219A8319821A88B9
:1031E80092B242F040021A80F8BD1D4B996A0A4318
:1031F8009A6292E700200446CEE7194B19690A4300
:103208001A618AE7164BD9680A43DA6085E702F53E
:10321800EA32116941F400411161116921F4004158
:103228001161B3E702F56042D16841F48051D16081
:10323800D16821F48051D160A8E702F5EC32116918
:1032480041F480411161116921F4804111619DE7C8
:10325800283D00200038004000300140003C00407C
:1032680000100240F0B53A4C059D00EB800004EBDD
:1032780080046468002C69D0364E49004FF4204021
:10328800CFB23060A169090453D46068DFF8D0E098
:1032980047F4903100EA0E0001434FF4204061608A
:1032A800306003E0411E002847D00846A16989071D
:1032B800F8D54FF42040A262306003E0421E002897
:1032C8003BD01046A2695106F8D5234A6168DFF859
:1032D80090E0306042EA0342174301EA0E021743C6
:1032E8006760BBB1013BDBB201332B444FF4204193
:1032F800A269316052074FF4204005D4421EE0B164
:103308001046A2695207F9D5626A306005F8012BA8
:103318009D42EDD14FF42040306002E0431E60B181
:103328001846A3699B06F9D520233060E361012084
:10333800F0BD411E08B10846A4E7084A13880133C6
:103348009BB24FF0FF3113803160F0BD2046F0BDD5
:10335800647600207C22002000240002142D002026
:10336800009800FCF0B5037C012B85B0044663D0BF
:10337800022B67D1836913B11A689B88138560692A
:1033880040F2E93301E0002B6CD00289013B12F0D6
:10339800020F9BB2F7D0C323037340F2E93301E075
:1033A800002B5FD00289013B12F0010F9BB2F7D0CE
:1033B800037B60694FF0060E838902AE4FF47A737F
:1033C8004FF6FF71FF2703E0013B9BB28B423CD0D5
:1033D80002899507F8D507734FF47A7302E0ABB208
:1033E8008B4232D00289D20703F1FF35F7D5027B31
:1033F800D2B20EB132700136BEF1010EE8D1A36926
:1034080013B11A689B8893619DF80C009DF80860B9
:103418009DF809109DF80A509DF80B209DF80D3075
:1034280041EA062143EA002342EA052201202187D6
:103438006287A38705B0F0BD90F91400431C01D042
:10344800022805DD002005B0F0BD0DF015FED6E719
:1034580002AB617D009343220623FFF703FF002898
:10346800D2D1EFE70DF008FEA3E700BFF0B5037A6D
:10347800012B85B0044663D0022B67D1036913B1D1
:103488001A689B881385E06840F2E93301E0002B55
:103498006CD00289013B12F0020F9BB2F7D0BB231C
:1034A800037340F2E93301E0002B5FD00289013B4E
:1034B80012F0010F9BB2F7D0037BE0684FF0060EC5
:1034C800838902AE4FF47A734FF6FF71FF2703E04A
:1034D800013B9BB28B423CD002899507F8D5077314
:1034E8004FF47A7302E0ABB28B4232D00289D20732
:1034F80003F1FF35F7D5027BD2B20EB13270013637
:10350800BEF1010EE8D1236913B11A689B88936153
:103518009DF80C009DF808609DF809109DF80A5068
:103528009DF80B209DF80D3041EA062143EA00235F
:1035380042EA05220120E1822283638305B0F0BDBF
:1035480090F90C00431C01D0022805DD002005B0CD
:10355800F0BD0DF091FDD6E702AB617B00933B22F5
:103568000623FFF77FFE0028D2D1EFE70DF084FD98
:10357800A3E700BF1749184B184A194810B4D1F8E7
:10358800884044F47004C1F888401C6844F0010481
:103598001C605C6822405A601A6822F0847222F427
:1035A80080321A601A6822F480221A605A6822F45B
:1035B800FE025A60DA6A22F00F02DA621A6B0024FD
:1035C80010404FF0006218639C608A605DF8044BFD
:1035D800704700BF00ED00E0001002400CC07FF80B
:1035E800CCFC00FF2DE9F04F80462DED028BB0F9A1
:1035F80008000881C5B28FB028460C4692462CF0C8
:1036080085F840B101231A46184662810FB0BDEC17
:10361800028BBDE8F08FA5F10A03ED2B00F2F080D4
:10362800DFE813F0B701EE00EE00EE00EE00EE006A
:10363800EE00EE00EE00EE00EE00EE00EE00EE0012
:10364800EE00EE00EE00EE00EE00EE00EE00EE0002
:10365800EE00EE00FB01EE00EE00EE00EF04EE00DF
:10366800EE00EE00FE04EE000B05EE006A05EE002B
:103678007904EE008504EE008D04EE00B304EE003C
:10368800EE00EE00C804CE04EE00D504EE00EE0015
:10369800E804EE009706EE00EE00EE007507EE0077
:1036A800EE00EE00EE002507EE00C901EE00F5057C
:1036B8001A06EE00EE00EE00EE00EE00EE00EE0060
:1036C8003D06EE006906EE001902EE006802EE0003
:1036D800BB02EE00EE00EE00EE00CE02B305EE05F2
:1036E8004407EA01EE00EE00B203C803EE00FA0355
:1036F8003104EE00EE00EE00EE001907EE00EE00D9
:10370800BF06EE00EE00EE000A07F4020A031D03EE
:10371800EE00EE00EE005E03EE006C037A03EE00AE
:10372800EE00EE00EE00EE00EE00EE00EE00EE0021
:10373800EE00EE00EE00EE00EE00EE00CE02EE002F
:10374800EE00EE00EE00EE00EE00EE00EE00EE0001
:10375800EE00EE00EE00EE00EE00EE00EE00EE00F1
:10376800EE00EE00EE00EE00EE00EE00EE00EE00E1
:10377800EE00EE00EE00EE00EE00EE00EE00EE00D1
:10378800EE00EE00EE009A03EE00EE00EE00EE0012
:10379800EE00EE00EE00EE00EE00EE00EE00EE00B1
:1037A800EE00EE00EE00EE00EE00EE00EE00EE00A1
:1037B800EE00EE00EE00EE00EE00EE00EE00EE0091
:1037C800EE00EE00EE00EE00EE00EE00EE00EE0081
:1037D800EE00EE00EE00EE00EE00EE00EE00EE0071
:1037E800EE00EE00EE00EE00EE00EE00EE00EE0061
:1037F800A8034E04EE00EE00EE00EE00EE00830596
:10380800742D58D0772D10D1D8F80030D8F804206E
:103818009A421EBF5A1CC8F800201978A74A08BF48
:10382800002120462EF0C8FAECE6F52D54D0D8F841
:103838000410D8F80060A5F1210381468A1B362BB5
:1038480000F26C87DFE813F00E076A076A076A0759
:103858006A076A076A076A0734076A076A076A070E
:103868006A076A076A076A076A076A076A076A07C8
:103878006A076A076A076A07FA066A076A076A0729
:103888006A076A076A076A076A076A076A076A07A8
:103898006A076A076A076A076A076A076A076A0798
:1038A8006A076A076A076A076A076A07C3066A0730
:1038B800A0066A079B06D8F80030D8F804209A4278
:1038C8001EBF5A1CC8F8002019787D4A08BF00217D
:1038D80020462EF071FA95E6D8F80030D8F8042082
:1038E8009A4242F00180774BFF221A724FF000088B
:1038F800754D1EF035FA41462022744885F800803F
:1039080032F0DFFA8DF814809DF81430072B02F29C
:103918001E816F4F6D4E42469DF8143003EB4303F2
:1039280007EBC3035B7CE3B19DF8143003EB43035F
:1039380007EBC30320215B699BB19DF8143003EBAF
:10394800430307EBC303586946F822000DF068F8F3
:103958002B7856F823000DF025FA2A780132D2B2D6
:103968002A709DF814300133DBB28DF814309DF8BD
:103978001430072BD0D92368591C21601A70BAF16A
:10398800000F3FF43FAE534BCAF8003001231A46EC
:103998003AE6514D284630F067F900287FF732AEF5
:1039A8002B460544226813F8011B501C9D422060D9
:1039B8001170F7D126E6494E3378002B3FF422AE3A
:1039C800474F0025B846236817F81520591C216071
:1039D8001A7098F8011001EB810101EB810101F2E5
:1039E800EE2189B22046FEF7F9FA337801359D4277
:1039F80008F10208E7DB05E6384E3378002B3FF480
:103A080001AE384F002537F8021F2046FEF7E6FAC8
:103A1800337801359D42F6DBF4E5334D05F1500668
:103A280028782EF01DFA2368027A591C21601A7032
:103A380023686A78591C21601A702368AA78591C6F
:103A480021601A702368EA780435591CAE42216057
:103A58001A70E5D1D6E5254E23687279244D591C94
:103A680021601A702B682046198CFEF7B7FA2B686C
:103A78002046D98BFEF7B2FA71892046FEF7AEFAD6
:103A8800B1892046FEF7AAFA2B682046598CFEF722
:103A9800A5FA2B682046998CFEF7A0FAF1892046F2
:103AA800FEF79CFA318A2046FEF798FA2A682368BE
:103AB80092F82620591C21601A70A3E535140308D2
:103AC80081140308901E0020FB830020BC83002083
:103AD8005C510020193503084A4C0020203300208F
:103AE8008C3500202278002084340020F84F0020F4
:103AF8002441002020460021FEF770FA20460021CC
:103B0800FEF76CFA20460021FEF768FA2368AF4DED
:103B180000265A1C22601E7023682A68591C92F8D5
:103B28002C2021601A7023682A68591C92F83620C4
:103B380021601A7023682A68591C92F8372021607E
:103B48001A7023685A1C22601E7023685A1C22604F
:103B58001E7023685A1C22601E702B682046598FDD
:103B6800FEF73CFA2B682046198FFEF737FA2368D0
:103B78002A68591C92F82E2021601A7023685A1C52
:103B880022601E702B682046598EFEF727FA2B6894
:103B98002046998EFEF722FA34E523688C4A8D492F
:103BA800D0788D4A5D1C2560187023684979581CA7
:103BB800206019702368D278591C21601A7021E599
:103BC8000023DFF84892DFF848B204930393059383
:103BD8000693984601214FF6FF7A07E008F101089D
:103BE800B8F10B0F01F0A28519F9011F4F1C4AFA11
:103BF80008F3F3D0DE07F1D5BBF8003043FA08F339
:103C0800D807EBD505A8FEF75FFDE7E72268734BF9
:103C180073491878551C2560107022685878551C0F
:103C28002560107022689B78501C20601370C9882A
:103C38002046FEF7D3F9E5E423686A4A6449107818
:103C4800654A5D1C2560187023688978581C2060B7
:103C5800197023689278591C21601A70D2E4DFF831
:103C6800B4E10027FEB2714600232268501C206090
:103C780016702268501C20601370226811F8010F1A
:103C88000133551C062B25601070EED10137062F25
:103C98000EF1060EE6D1544900232268501C20601C
:103CA80017702268501C20601370226811F8010FE9
:103CB8000133551C0B2B25601070EED123684B4A3D
:103CC800581C07212060197023680021581C2060A7
:103CD8001970236892F8F020591C21601A7091E439
:103CE800434D2046298AFEF779F9698A2046FEF76E
:103CF80075F9A98A2046FEF771F983E4364B3D49E8
:103D0800B3F9003081FB0321DB17C3EBA10189B2B2
:103D18002046FEF763F975E42368374F591C3A7853
:103D280021601A703B78002B3FF46CAC0025EEB292
:103D380030461BF03DFB23684278591C2160304611
:103D48001A701BF035FB01892046FEF747F93B78CE
:103D580001359D42EBDB55E42368284A591C12784B
:103D6800216005A81A70FEF72BF823685A1C2260F8
:103D7800187047E4164D2046E989FEF72FF9A989FE
:103D88002046FEF72BF93DE41D4D20462988FEF715
:103D980025F969882046FEF721F9B5F90430154957
:103DA800DA1781FB0313C2EBA30399B22046FEF78F
:103DB80015F927E4134B20461968FEF7F7F8124B5C
:103DC80020461988FEF70AF91CE400BF24410020A8
:103DD800C4370020307A0020D4370020BC370020B8
:103DE800AC430020F84F002027480020444700201B
:103DF8001C52002067666666AD3D00200A3C002024
:103E0800D0400020C8400020CC4000208460030837
:103E18002041002003480020AA4D23682A68591C25
:103E2800127821601A702B6822689978531C2360D5
:103E3800002311702A6821681A4401335279481CFA
:103E4800032B20600A70F5D123682A68591C127A5E
:103E580021601A7023682A68591CD27821601A7068
:103E680023682A68591C127921601A702B68204629
:103E78005989FEF7B3F82A682368527A591C2160D9
:103E88001A702A68D2E0904D00232268286803EB54
:103E98004301561C405C266010702A6820680A445A
:103EA800461C5278266002702A6820680A4401334A
:103EB8009278411C0A2B21600270E6D1FFF7A2BB61
:103EC800824B03F1700522681978501C206011702C
:103ED80022685978501C2060117022689978501C0B
:103EE800206011702268D978501C206011702268F7
:103EF8001979501C2060117022685979501C206073
:103F08001170226899790733501CAB4220601170F8
:103F1800D9D1FFF777BB6E4D05F1800655F8041F20
:103F28002046FEF743F8AE42F8D1FFF76BBB236893
:103F3800684A591C527D21601A70FFF763BB664BB3
:103F480003F15A0522685979501C206011702268C3
:103F58001978501C2060117022685978501C206014
:103F6800117022689978501C206011702268D978E5
:103F7800501C20601170226819790633501C9D422C
:103F880020601170DED1FFF73DBB544D544E05F152
:103F9800200795F90210534B93F906208A4203F142
:103FA800080301F0A5839E42F6D10835AF42F0D14F
:103FB800FFF728BB00212046FDF7F8FFFFF722BBDB
:103FC80023680122991821601A70FFF71BBB236828
:103FD800454A464990785D1C2560187023685278D8
:103FE800581C20601A7023680A79591C21601A70BD
:103FF800FFF708BB082237492046FDF7BFFFFFF748
:1040080001BB3B4D20462988FDF7E8FFA9882046DB
:10401800FDF7E4FF29892046FDF7E0FFFFF7F2BA34
:104028002368344A581C1178206019702368527824
:10403800591C21601A70FFF7E5BA264D23682A7AC1
:10404800591C21601A70A98B2046FDF7C7FF298BE0
:104058002046FDF7C3FF698B2046FDF7BFFF2368A5
:10406800EA7C591C21601A70A98C2046FDF7B6FF1E
:10407800E98C2046FDF7B2FF2368AA7F591C21600E
:104088001A70236895F82020591C21601A70698CD1
:104098002046FDF7A3FF2368EA7A591C21601A70AD
:1040A800E9682046FDF782FF23682A7C591C2160B5
:1040B8001A70236895F82120591C21601A70FFF79F
:1040C800A1BA00BF2841002024410020082F002069
:1040D80040470020E47A002000300020107B0020B8
:1040E8008C5500206C550020E4370020901E0020DD
:1040F800202B0020F83C0020BB4D05F14006B5F808
:1041080080102046FDF76AFF236895F88220591C25
:1041180021601A70236895F883200435591CAE4233
:1041280021601A70EBD1FFF76DBA05A8FDF748FEBC
:1041380000283FF467AABDF814102046FDF74EFF8B
:1041480023689DF81620591C21601A7023689DF871
:104158001720591C21601A7023689DF81820591CD3
:1041680021601A7023689DF81920591C21601A7063
:1041780023689DF81A20591C21601A70BDF81C107C
:104188002046FDF72BFFFFF73DBA984B9B8AB3F506
:10419800006F01F2A683B3F5806F01F2FB83B3F5DC
:1041A800007F34BF01270227914D05F10C0655F811
:1041B800041B91FBF7F1204689B2FDF70FFFB542CA
:1041C800F5D18C4D8C4F05F10C06B5EC010AD7EDF5
:1041D800077A80EE270A30F0B7FE81B22046FDF755
:1041E800FDFEAE42F1D1854D05F10C0655F8041BD4
:1041F800204689B2FDF7F2FEB542F7D1FFF702BAC1
:1042080010227F492046FDF7B9FEFFF7FBB9236866
:104218007C4D01269A1922601E701AF019FC00289C
:1042280041F09383784B2268511C216010702268FA
:1042380041F2B410511C185C216041F278111070E1
:1042480059582046890AFDF7B1FEA96A204649084F
:10425800FDF7ACFEFFF7D6B923686C4D591C012257
:1042680021601A702368AA78591C21601A7016F008
:1042780083FC2368664A67495E1C26601870B1F99A
:104288000010B2F90000FEF7CDF823685A1C22602E
:10429800187029882046FDF7A1FEFFF7B3B921F071
:1042A8006DFDFF28054601F05E830EA8002300F887
:1042B800243D21F035FD2268574B511C21601570B3
:1042C80022681978501C2060117022685978501C97
:1042D8002060117022689978501C20601170226843
:1042E8009DF81410501C2060117099882046FDF725
:1042F80075FEFFF787B9494FFB78002B01F0E48280
:1043080023680822591C21601A7023680122991811
:1043180021601A702368424D591C2A7921601A704D
:104328002368AA78591C21601A7029882046FDF74D
:1043380055FEE9892046FDF751FE2368FA79591C94
:1043480021601A702368EA78591C21601A70FFF7F7
:1043580059B92368334A344D1178344A581C2060BF
:10436800197011682046FDF721FE2368304A591C50
:10437800127A21601A7029882046FDF72FFEA98835
:104388002046FDF72BFE29892046FDF727FE20460B
:104398000021FDF723FE00212046FDF71FFEFFF751
:1043A80031B9244D05F16006A9882046FDF716FEAF
:1043B800E9882046FDF712FE29892046FDF70EFE02
:1043C8002368AA7A591C21601A702368EA7A591C52
:1043D80021601A7055F80C1B2046FDF7E7FDB54221
:1043E800E2D1FFF70FB900BF44470020D8400020B2
:1043F8000841002010500020804D0020743C00200F
:10440800B03C0020A071002014570020FA7700204B
:104418000A360020103600203C560020F84F0020B5
:104428001C520020F83C0020202B00206082002035
:10443800E47A0020482E0020A94D20462988FDF75F
:10444800CDFD69882046FDF7C9FDA9882046FDF7FE
:10445800C5FDFFF7D7B8A34952232268501C206036
:10446800137011F8013F002BF7D1FFF7CBB8236881
:104478009D4D591C2A7921601A7023686A79591C44
:1044880021601A7029882046FDF7A8FD2368AA79BB
:10449800591C21601A7069882046FDF79FFD236822
:1044A800EA79591C21601A70FFF7ACB88F4D904E0D
:1044B800DFF86082DFF860929FED8E8A05F12007B1
:1044C8000EE0FCEEE77ACDED017ABDF80410204647
:1044D8000435FDF783FDBD4206F118063FF492A8A6
:1044E800717C0029F3D098F80030D5ED007A012BC3
:1044F800E7D1D9F80030DB0441F1BC81F5EE407A10
:10450800F1EE10FA41F05B8240F2DC51DFE72368FC
:1045180000255A1C226029461D702046FDF746FDDD
:1045280029462046FDF742FD29462046FDF73EFD77
:10453800FFF768B80723B2FBF3F3C3EBC301521AC2
:104548001DD1DBB203F1FF395FFA89F9002B3FF483
:1045580059A8DFF8A4B109F101091746731CC8F876
:10456800003096F90010644B002593F902208A4226
:1045780003F1080301F057820135042DF5D14FF0FE
:10458800FF331A46FFF740B8731CC8F80030357877
:10459800FF2D01F07B82FE2D01F031824046FDF7B0
:1045A800DBFC98E80C009B1A002B07DD531CC8F8AD
:1045B8000030137813B90C2D41F2A982272DDED8CB
:1045C8004E4A012322F815001A46FFF71DB8731C3E
:1045D800C8F8003030780328D1D8431E484D4949DF
:1045E800DBB203EB430305EB430308705D78002857
:1045F8003FF408A8531EDBB2AB42C0D10022C1F879
:104608000620C1F802208A726BB1581CD8F8003015
:1046180008444A1C0133C8F8003013F8011C02F89A
:10462800011F8242F6D1384B1B78002B3EF4EAAFCB
:104638002CF08DFC01231A46FEF7E6BF731CC8F860
:10464800003033780A2B01F0A8814046FDF790FC32
:104658004046FDF78DFC4046FDF78AFC01231A46CB
:10466800FEF7D2BF3346721CC8F80020274D13F856
:10467800022B6A70C8F8003073782B70F31CC8F8E6
:104688000030B378AB704046FDF766FCD8F80030D0
:1046980028811A46591CC8F8001012F8021B6971C3
:1046A800C8F800205B78AB7101231A46FEF7ACBF4F
:1046B800731CC8F8003033780A2B01F06581502B41
:1046C80040F09C864046FDF747FC114D2880404647
:1046D800FDF742FC012368801A46FEF795BF00BF2C
:1046E800AC43002054600308C8430020C03C0020AD
:1046F8005C51002000004042107B00208C77002095
:10470800F8610308347B002034230020A8400020EF
:10471800B8230020405200201C500020A5F10B00B7
:10472800EF283FF62CAF01A353F820F0AD56000850
:104738008745000887450008874500088745000821
:104748008745000887450008874500088745000811
:104758008745000887450008874500088745000801
:1047680087450008874500088745000887450008F1
:1047780087450008874500088745000887450008E1
:104788008745000887450008874500083356000814
:10479800874500081956000887450008F75500089E
:1047A800874500088745000887450008CB5500085D
:1047B800874500086555000887450008F15400083A
:1047C80087450008C554000887450008E9560008D1
:1047D8008745000863540008874500083D450008E0
:1047E8008745000887450008874500088745000871
:1047F8000D36000887450008315400088745000831
:10480800874500081554000887450008BD5300086F
:104818008745000887450008874500088745000840
:104828008745000887450008874500088745000830
:10483800715300088745000823530008874500087E
:10484800874500083D51000887450008874500084E
:104858008745000887450008874500088745000800
:1048680087450008D150000887450008E95100082D
:104878008745000835500008874500086F52000832
:1048880087450008A35000087B510008175000080E
:1048980087450008874500088745000887450008C0
:1048A80087450008874500088745000887450008B0
:1048B80087450008874500088745000887450008A0
:1048C8008745000887450008874500088745000890
:1048D8008745000887450008874500088745000880
:1048E8008745000887450008874500088745000870
:1048F8008745000887450008874500088745000860
:10490800874500088745000887450008874500084F
:10491800874500088745000887450008874500083F
:10492800874500088745000887450008874500082F
:10493800874500088745000887450008874500081F
:10494800874500088745000887450008874500080F
:1049580087450008874500088745000887450008FF
:1049680087450008874500088745000887450008EF
:1049780087450008874500088745000887450008DF
:1049880087450008874500088745000887450008CF
:1049980087450008874500088745000887450008BF
:1049A80087450008874500088745000887450008AF
:1049B800874500088745000887450008874500089F
:1049C800874500088745000887450008874500088F
:1049D800874500088745000887450008E54F000817
:1049E80087450008CF4F0008A14F000887450008F9
:1049F800874500088745000887450008874500085F
:104A0800874500088745000887450008874500084E
:104A1800874500088745000887450008874500083E
:104A2800454F000887450008074F000887450008DC
:104A3800594E0008F74D0008DB4D0008874500086F
:104A4800C14D000887450008974D0008854D0008AE
:104A5800254D000887450008FD4C000887450008DB
:104A680087450008DB4C0008A74C0008934C000859
:104A7800654C00083F4C00081D4C0008874500089D
:104A8800054C000887450008874500088745000849
:104A980087450008874500088745000887450008BE
:104AA80087450008874500088745000887450008AE
:104AB800874500088745000887450008EB4B000834
:104AC8008745000887450008814B0008874500088E
:104AD80087450008874500080F4B000887450008F0
:104AE8008745000887450008F54A0008C64B1B782B
:104AF800DB073FF544AD01F021FC01F0FBFD01238C
:104B08001A46FEF781BD4046FDF726FAD8F8003070
:104B1800ADF814001A46591CC8F8001012F8021B08
:104B2800C8F800208DF816105A788DF81720DA1C6E
:104B3800C8F800209A788DF818201A1DC8F80020A7
:104B4800DA788DF819205A1DC8F800201B798DF8DD
:104B58001A3005A80023ADF81C30FDF757F9AB4B08
:104B6800AB4A1D68401B4FF0010361F10001C2E927
:104B780004011A46FEF748BD731CC8F800303378A4
:104B88000F2B3FF6FCACB21CC8F80020C3EBC303E4
:104B9800A04A7178D154F11CC8F800101344B278B7
:104BA8005A70321DC8F80020F2789A70721DC8F841
:104BB80000203279DA70B21DC8F8002072791A71B3
:104BC800F21DC8F80020B2795A7106F10802C8F837
:104BD8000020F2799A7127F0E5F901231A46FEF7C9
:104BE80013BD4046FDF7B8F98B4DE8814046FDF707
:104BF800B3F90123A8811A46FEF706BD4046FDF722
:104C0800ABF9864900EB8000420001230A801A466E
:104C1800FEF7FABC4046FDF79FF9814D28824046D1
:104C2800FDF79AF968824046FDF796F90123A882B4
:104C38001A46FEF7E9BC3346721CC8F8002013F880
:104C4800020BC8F80030F31C7178C8F80030B2784D
:104C580022F010FB00287EF4D5AC90E43346721C99
:104C6800C8F800206F4A13F8021B1170C8F800300A
:104C7800694A73789370F31CC8F80030674BB278B0
:104C88009A7001231A46FEF7BFBC674B674918683C
:104C98004E222FF085FF01231A46FEF7B5BC324697
:104CA800731CC8F80030624B12F8021B1970C8F860
:104CB800002072785A70F21CC8F80020B2789A70F6
:104CC8004046FDF749F95B4A0123D0801A46FEF7B2
:104CD8009BBC4046FDF740F9564D28804046FDF7FD
:104CE8003BF968804046FDF737F90123A8801A464A
:104CF800FEF78ABC504F3B78002B3EF483AC4F4EF6
:104D080000254046FDF728F91EF084FF3B78A6EC05
:104D1800010A01359D42F4DBFEF774BC0D2A7FF4CD
:104D28002EAC731CC8F800303578072D3FF627AC39
:104D3800434F40460C26FDF70FF906FB05F6BD1953
:104D4800A8804046FDF708F9E8804046FDF704F9D9
:104D5800D8F8003028811A46591CC8F8001012F8F3
:104D6800021BA972C8F800205B78EB724046FDF779
:104D7800DBF80123B8511A46FEF746BC4046FDF75A
:104D8800EBF8304A012310801A46FEF73DBC731C2D
:104D9800C8F800303078060600F181871A4B1B7876
:104DA800DD073EF52FAC032828BF002001F0AAFA42
:104DB80001231A46FEF728BC134B1B78D8073EF58B
:104DC80021AC02F07DF801F095FC01231A46FEF7AC
:104DD8001BBC0D4B1B78DA073EF514AC1A490A7850
:104DE800012342F004020A701A46FEF70DBC064B76
:104DF8001B78D9073EF506AC144A4FF4C871012355
:104E080011801A46FEF700BC33560020C4760020F5
:104E1800901E0020082F0020C4370020D43700201F
:104E28001C520020F84F002024410020F47D030884
:104E3800BC370020AC430020AD3D00201C2D0020D5
:104E4800482E0020C2210020F8770020EC430020E3
:104E5800092A7FF794ABCF4F3346721C3D68C8F8D8
:104E6800002013F8022B2A70C8F800307378AB7052
:104E7800F31CC8F80030B378642BA8BF6423321D34
:104E88006B71C8F80020F378642BA8BF6423721DE7
:104E9800AB71C8F800203379EB71B31DC8F8003046
:104EA8007379642BA8BF6423F21D2B72C8F8002005
:104EB800B379EB7006F10803C8F80030F3792B7169
:104EC8004046FDF749F8D8F80420D8F80030688142
:104ED800D11A00290DDD591C3868C8F80010521A7B
:104EE800002A1978417204DD9A1CC8F800205B7802
:104EF80043701FF0FFFC01231A46FEF785BBA64B43
:104F08001868F31C02462136991EC8F8001013F8D9
:104F1800031C1170591EC8F8001013F8021C5170B8
:104F2800C8F8003013F8011C91700333B34202F142
:104F38000302E9D127F062FCFEF764BBC2F3470520
:104F4800122D3FF61CABBDB10EAB0DF1120703EBF2
:104F580045093E46A9F126094046FCF7FDFF26F81B
:104F6800020FB145F8D18D4B37F8022F23F8022FE5
:104F7800BE42F9D1112D09D8894A6B00023B13446E
:104F88000021223223F8021F9A42FBD185490122CF
:104F980013460A70FEF738BB731C8349C8F8003003
:104FA8000A783378002A00F0E985042A7EF42AABCF
:104FB8007E4A9B00138002F0B7FC7D4A0123906172
:104FC8001A46FEF721BB7B4D002340462B60FCF7B9
:104FD800ABFF012328601A46FEF716BB3346721C46
:104FE800C8F8002013F8025BC8F80030F31C70788A
:104FF800C8F80030B178002D00F0DC85012D7EF472
:1050080001AB1EF057F82B462A46FEF7FDBA731C73
:10501800C8F800303378002B00F0A7854FF4004023
:105028002AF0CEFE01231A46FEF7EEBA731CC8F822
:105038000030594D604F33787B7140462E68FCF73D
:105048008BFF308440462E68FCF786FFD8F8042092
:10505800D8F80030F083D11A072900F39385D11AC4
:10506800032900F32786D21A002A06DD591C2A686C
:10507800C8F800101B7882F8263001F09DFA22F05B
:1050880079FD4E4B28681B68002B00F0638527F0DC
:105098001DF801231A46FEF7B7BA3346721CC8F842
:1050A8000020474A13F8021BD170C8F80030454A5F
:1050B80073785371F31CC8F80030434BB278DA7038
:1050C80001231A46FEF7A0BA404B1B68002B3EF49A
:1050D80099AA20F053FEFF283EF494AA4046FCF714
:1050E8003BFF3F2840F2F485394E00253570D8F84B
:1050F8000030D8F80420B080D21A012A7EF782AA9C
:105108001A46591CC8F8001012F8021BB1700EA8F4
:10511800C8F8002000225D7800F8242D20F000FE59
:105128009DF81430AB423EF46DAA284620F01CFED0
:10513800FEF768BA274B1B78012B3EF663AA324666
:10514800731CC8F80030244D12F8023BAB70F31CF6
:10515800C91AC8F8002001297278C8F8003040F34D
:105168002F854046FCF7F8FE012328801A46FEF7F3
:105178004BBA1A4B1B7813F001017FF400AA731C79
:10518800C8F8003030781DF0CFFE01231A46FEF72C
:105198003BBA00BF284100202441002036330020BC
:1051A800383300205C3300200A3C002018780020A7
:1051B800901E0020F42F0020F84F0020E03C002033
:1051C800C4370020307A0020D43700203856002019
:1051D8003C56002050820020FA77002033560020E9
:1051E8003346721CC8F80020CD4F13F8022BBA7052
:1051F800C8F80030CB4A73781370F31CC8F8003035
:10520800C94DB3782B71331DC8F80030F378092BDA
:10521800A8BF09234046AB70FCF79EFED8F80030C3
:10522800D8F804202880D11A012907DD4046FCF768
:1052380093FED8F80030D8F80420E8819A4240F06C
:10524800248501F0B9F9D8F80030D8F804209A423A
:105258003EF4D8A95A1CC8F800201B78EB7001232B
:105268001A46FEF7D1B94046FCF776FE4046FCF7F1
:1052780073FE4046FCF770FE4046FCF779FED8F80E
:105288000030AA4D1946581C2A68C8F8000011F8C1
:10529800020B82F82C00C8F80010597882F83610F2
:1052A800D91CC8F800109B7882F837304046FCF7C4
:1052B8005FFE4046FCF75CFE4046FCF759FE404660
:1052C8002E68FCF749FE708740462E68FCF744FEBE
:1052D800D8F80030D8F804203087D11A01290DDD1C
:1052E800591C2A68C8F800101B7882F82E304046EE
:1052F800FCF73EFED8F80030D8F80420D31A032B68
:1053080009DD40462E68FCF727FE708640462E6869
:10531800FCF722FEB08628680CE6731CC8F800303B
:105328003778112F3FF62BA9B31CC8F80030804DF1
:10533800737805F817304046FCF70EFE40F6CA03AE
:105348009842A8BF184640F2EE23984205EB47055D
:10535800B8BF18460123A0F2EE211A46192091FB86
:10536800F0F16970FEF750B93346721CC8F8002096
:10537800704D13F8022B2A71C8F8003073786B71DE
:105388004046FCF7E9FDD8F8003028805A1CC8F8D8
:1053980000201B78AB714046FCF7DEFDD8F80030E2
:1053A80068805A1CC8F800201B78EB7101231A4644
:1053B800FEF72AB9731CC8F800305F4B32785F4F8C
:1053C8001A7000233B604046FCF7AEFDD8F8002079
:1053D8003B685B495B4D0343501C3B60C8F80000C9
:1053E80013780B724046FCF7B7FD28604046FCF77F
:1053F800B3FD68604046FCF7AFFDA8604046FCF787
:10540800ABFD4046FCF7A8FDFEF7FCB84E4B06F195
:1054180008020136C8F8006016F8011C03F8011FDD
:10542800B242F6D1FEF7EEB83346721CC8F8002037
:10543800464A13F8020B9070C8F800307078507024
:105448008B423EF4DFA8F31CC8F80030404BB2781A
:105458001A7101231A46FEF7D7B8731CC8F8003032
:1054680033780E2B3FF68BA8B21CC8F80020707852
:1054780003283FF684A83749062202FB03F28B185B
:10548800F51C5871C8F80050B0788854321DC8F817
:105498000020F2785A70721DC8F8002032799A708C
:1054A800B21DC8F800207279DA70F21DC8F8002021
:1054B800B2791A7101231A46FEF7A6B8731CC8F808
:1054C800003035781F2D3FF65AA8052A7FF457A8D3
:1054D8004046FCF729FD204B43F8250020F0AAF9A7
:1054E80001231A46FEF790B81B4D05F140064046C9
:1054F800FCF732FDD8F80030A5F88000591C1A4690
:10550800C8F8001012F8021B85F88210C8F80020AD
:105518005B7885F883300435AE42E8D1FEF772B87F
:10552800F84F0020B83700201C52002024410020EA
:105538008C350020C8430020F83C00206082002001
:10554800E47A0020202B0020E37A0020E4370020B2
:10555800901E00200030002044470020731CCA4DD4
:10556800C8F8003033782B724046FCF7F5FCA88366
:105578004046FCF7F1FC28834046FCF7EDFCD8F8E0
:1055880000206883531CC8F800301278EA74D8F8F1
:105598000420D31A032B00F35383D8F80030D11A10
:1055A800052900F31983D21A002A7EF72BA85A1C62
:1055B800C8F800201B7885F8213001231A46FEF729
:1055C80023B8731CC8F80030B04832780270C91A82
:1055D80000297EF717A8B31CC8F80030727800328B
:1055E80018BF0122012342701A46FEF70DB8404643
:1055F800FCF7B2FCA64D28604046FCF7ADFC68609D
:105608004046FCF7A9FC0123A8601A46FDF7FCBF39
:10561800A04D00232B604046FCF786FC2A68012336
:1056280002432A601A46FDF7EFBF731CC8F8003022
:105638003578132D3EF6A3AFB31CC8F80030707848
:105648002CF0F4FB00283EF49AAF934B027803F851
:105658002520F21CC8F8002003EB8505B2786A7093
:10566800321DC8F80020F278AA70721DC8F8002010
:105678003279EA7003F1500202E004339A4208D00A
:1056880019780029F9D19878D9788842F5D24FF05D
:105698000109824A89F00109012382F800901A461B
:1056A800FDF7B2BF7E49102A13464FF0000228BF0B
:1056B80010230A604A608A60CA600A74002B3DF4AD
:1056C800A1AFD8F80020013913440132C8F80020EE
:1056D80012F8010C01F8010F9A42F6D1FDF792BFBA
:1056E800731CC8F80030684B32785A75FDF78ABFCA
:1056F80023685A1C2260197029882046FCF76EFC22
:105708002368EA78591C21601A7023682A79591C81
:1057180021601A702368AA79591C21601A702368BD
:105728006A79591C21601A70FEF73FBCDFF894A112
:105738004FF000084FF0A80908F10108C8F120024D
:1057480009FA02F2A8F120032AFA08F6164329FA00
:1057580003F31E43B8F1280F06F001024FF00003CF
:105768000CD01343E8D05FFA88F01FF05FF80028E8
:10577800E2D0414605A8FCF7A7FFDDE7494B1B78B7
:10578800DA0700F1EB800026474FB04602E0013609
:10579800282E0ED031463846FCF7A6FF0028F6D052
:1057A800314605A8FCF7A0FF00285ED108F10108E2
:1057B800EDE73E4B3E4EB3F850102046FCF70EFC8A
:1057C8003C4B1988204689B2FCF708FC3A4B1A680A
:1057D800530103F02001C2F340030B43C2F38001DD
:1057E80043EA4103C2F3C00143EA8103C2F3401113
:1057F80043EAC10102F0100211432046FCF7EEFB18
:1058080003A904222046FCF7B9FB236831782B4A08
:10581800581C2060197011886429A8BF642120468B
:10582800FCF7DCFB962D00F0A48000212046FCF755
:10583800D5FB2168B8F1190348BFA8F11203A3F3F7
:10584800C4034A1C226020461A460B7004A9FCF7C0
:1058580095FB23681A4A581C112120601970116899
:105868002046FCF7A3FBFDF7CDBE414603A8FCF795
:105878002BFF9BE7F4EEC87AF1EE10FA80F235813F
:105888004FF47A71FEF723BEE47A0020F83C00203A
:10589800202B002060820020843400202C0200206D
:1058A8004A4C002033560020E480002020030020CA
:1058B8005B4C0020142D0020C4400020182D00202F
:1058C8001C41002090E33FF42368B978CD4A581C66
:1058D8002060197023681278591C21601A70FEF72D
:1058E80019BD0827FEF760BC5A1C1946C8F80020E5
:1058F800C54811F8022B0272C8F800105B78437291
:10590800042A0BD9FF2A3DF4F1AF216800204A1C74
:10591800012322601A460870FDF776BEBB49097854
:10592800994203D8022AF0D1FF2BEED12268012335
:10593800D11821601370BAF1000F3DF463AEB44A78
:10594800CAF800201A46FDF75FBE95F82420B14B2F
:10595800002A40F092803046FEF765BC059B43F074
:10596800010305930FE723685A1C22601870FDF79E
:1059780049BE23680322591C21601A702368727873
:10598800591C21601A7054E74046FCF7E5FAA24D0D
:10599800FEF79CBE0427FEF707BCB31CC8F800300E
:1059A8009E4B72781A70F21CC8F80020B2785A70B0
:1059B800321DC8F80020F2789A70FDF723BEF4EE85
:1059C800C87AF1EE10FA3EF59FAD9FED957AF4EEA8
:1059D800C77AFDEEE77AF1EE10FA17EE901A00F2A8
:1059E800A7806FF4F973303903FB01F140F2E73314
:1059F80091FBF3F101F2DB5189B2FEF768BDB31CEC
:105A0800C8F800307578022D3EF6B9AD4046FCF76F
:105A1800A3FA844A02EB45024FF0FF33A2F856007E
:105A28001A46FDF7F1BD0BEBC50A40468AF802108D
:105A3800FCF792FAD8F800302BF835001A46591CB2
:105A4800C8F8001012F8021B8AF80310C8F80020E2
:105A58005A788AF80420DA1CC8F800209A788AF85C
:105A680006201E1DC8F800600137DB788AF805306B
:105A7800B9457EF473ADFDF7C5BD5978022951D0FB
:105A880003290CBF04203046FEF7CDBB4046FCF787
:105A98006FFAD8F80030634D1A46591CC8F8001040
:105AA80012F8021B85F85510C8F800205B7885F8B5
:105AB80054304046FCF750FAA5F850004046FCF731
:105AC8004BFA4046FCF748FA98E80C009B1A012B61
:105AD800A5F852007DF796AD4046FCF73DFA012344
:105AE800A5F85A001A46FDF78FBDFDEEE77A40F299
:105AF800E73317EE901A303903FB01F140F2CF7308
:105B080091FBF3F101F2E93189B2FEF7E0BC454BB4
:105B180000301D4418BF0120012385F85E001A4695
:105B2800FDF772BD042A34BF02200320FEF77BBBB9
:105B380040F2F313A1F5836103FB01F140F2E7336F
:105B480091FBF3F101F2DD5189B2FEF7C0BC424688
:105B5800FDF711BF344B354A354836491A600123E1
:105B680002600A601A46FDF74FBD33490A680123EF
:105B780022F400420A601A46FDF746BD04220A7064
:105B8800FFF716BA4046FCF7E7F978814046FCF77C
:105B9800E3F9B88140462E68FCF7DEF97084404688
:105BA8002E68FCF7D9F9D8F80030D8F80420B0846A
:105BB800FFF755BA26F0ADFC01231A46FDF724BDC0
:105BC8001E4BB0781988012311FB02F11A4691FB8C
:105BD800F0F12980FDF718BD5A1CC8F800201B7881
:105BE800EB724046FCF7A0F9D8F80030E8605A1C80
:105BF800C8F800201B782B74D8F80030D8F8042097
:105C0800D1E400BFB8370020901E0020AD3D002031
:105C180065F4020814570020B4370020F9800020EA
:105C280000E082448C770020007500205D050008A4
:105C380054750020BC7500201C4100200A36002045
:105C48004046FCF789F9A8844046FCF785F9D8F85E
:105C58000030D8F80420E884D11A03297FF79FACD4
:105C68001A46591CC8F8001012F8021BA977C8F880
:105C780000205B7885F820304046FCF76DF9D8F8AD
:105C88000030D8F80420688489E45A1CC8F8002039
:105C98001B78003318BF0123FB71FFF7D2BA00F05D
:105CA8007F00032828BF00201DF020FA01231A4690
:105CB800FDF7AABC4046FCF74FF9F8814046FCF7CF
:105CC8004BF9D8F80030D8F804203882FFF7CBB960
:105CD800C50800F0070301350133EDB2034E28462D
:105CE8001946737019F00AFBFFF700BA3C560020FA
:105CF80038B50B4C23688BB15A68821A002A0546BE
:105D080004DA0CE05A68AA1A002A07DB9A682260AB
:105D180018461A6890472368002BF3D138BD38BD60
:105D2800203400200B4B002210B4027203F1DC0473
:105D3800012102E0072A09DC9979890702D5197936
:105D4800815401329C4203F11403F3D15DF8044BF2
:105D5800704700BF188603081F230370704700BFF1
:105D680030B401230225152414212222057244701F
:105D78004171C27003700371837030BC704700BFFB
:105D88002DE9F0410B78057BDB43DFB200F113020C
:105D980000F11D0302F8015F9342FBD1DFF890E0A8
:105DA80000F12701002203F8012F9942FBD11421A9
:105DB8000524002647FA04F303F00103002B1E44D0
:105DC80014BF4FF019084FF00A0814F0010FF6B28B
:105DD80014BFAC464FF0000C0023CA1810FA82F228
:105DE8000133434582F814C0F7D15A1E92B20132EA
:105DF800013C8B18621C9BB201D01946DAE716F0F9
:105E0800010F14BF19240A240022991810FA81F1ED
:105E18000132A2420D75F8D113449BB25A1C0344B7
:105E2800002192B21975AEF800200261BDE8F08138
:105E3800B81E00202DE9F04FDFF890A0BAF8023024
:105E48000B3383B01FFA83F901F1060B4FF00108F9
:105E58004FF0000C002711F801EB3E464C4601229A
:105E6800A4F10B039BB2019105E001339BB2017BC6
:105E780029759C4208D0C518002AF6D1C5180133E7
:105E88009BB29C422A75F6D103190136092F019954
:105E980083F814C0F6B20CD0092E15D008FA07F30F
:105EA80013EA0E0F14BF012200220C34A4B20137EA
:105EB800D6E709F1780959451FFA89F9CAD1AAF82C
:105EC80002C003B0BDE8F08F0022EEE7B81E002044
:105ED8002DE9F047DFF85C80B8F8043004331FFA86
:105EE80083FC01F109094FF0010E11F8017B6446AA
:105EF8000026231F0EFA06F29BB23A40C2B1B0F850
:105F08000CA0C51801339BB29C4285F814A0F5D1AA
:105F180001360434082EA4B2EBD10CF1200C49450B
:105F28001FFA8CFCE1D10023A8F80430BDE8F08703
:105F38009246E6E7B81E002010B50168047B0A689F
:105F48000223A3401A420AD0054A4068002414706C
:105F5800026822F001021204120C02604B6010BDAC
:105F6800362300202DE9F0478C4B1B78DB070746CA
:105F780044D58B4B8B4D1C788B4E012C59D01CD3A0
:105F8800022C07D189498A4A09881288914201D985
:105F980001241C70EB7AE3B12B89D3B1854B1B78B4
:105FA800BBB10BF049FD002800F09B802B7B83429E
:105FB8002CBF0121002131700CE07C497E4A098800
:105FC80010886A7B801A8842E2DAEB7A0024002B78
:105FD800E2D131782A79632A06D8022C774E00F06C
:105FE800BA803378002B5DD1754AAB7A8C4238BFC2
:105FF8000C461470002B4CD1BDE8F0876B4B694DF3
:1060080019885B88E878CB1A83EAE3728142A2EBAD
:10601800E3721DD32B788B421AD3614B1C78E01E98
:10602800012861D96749097802294FD0012C5E4EB1
:10603800A5D15F4A5D491288687B0988121A914286
:1060480039DD5D4A12888A42A4D200241C70A1E777
:10605800B1EB400FE1DC524B1C78E11E012940F204
:106068009480022ADEDC57494F4E0878DFF84481D5
:10607800DFF844C1DFF838E1002103240228347036
:106088001C7088F80010ACF80010AEF8001081D130
:106098001FE0012C71D0022C0BD10720BDE8F0477E
:1060A8002BF0ECBC7068381A474B984258DD727078
:1060B8009AE7BDE8F08702241C706BE7022AD2DD5C
:1060C8004049097802294FF0040464D13949364E11
:1060D80009783E48022ACCBF00220122C280818072
:1060E8004BE70221317075E7022A9BDC95F800C066
:1060F80091FBFCFC0CF1010CBCF1080FDFF8B4A01B
:10610800304EA87895F801E096F800802A4CDFF820
:10611800A090254EA8BF4FF0080C8AF800C01FFABF
:106128008CFA10FB0AF01EFB0AFE80B2DFF88CA086
:106138002080A9F800E000244FF0640EB8F1020FA7
:1061480034701C70CAF804408AF801E07FF439AF53
:106158000FFA8CF1BDE73078A0B90123776033706E
:10616800C2F164021A4B00FB02F083FB0023C01744
:10617800A0EBA3506430707036E70820BDE8F04704
:106188002BF07CBC7368F81A8EE7032C96D10D4966
:10619800097802299AD0044EFCE600BF3356002045
:1061A800D8220020A8400020E8220020D43E002069
:1061B800DC220020EA3E0020DA220020E022002033
:1061C80054780020CC3D00207F969800D03D0020D8
:1061D8006BCA5F6B2DE9F0470569C3681D4028D07D
:1061E8000F4606464FF000484FF00009B5FA85F310
:1061F80028FA03F2D2431B3B32611540042B16D810
:10620800DFE803F03129211903007B6A002B32D023
:1062180003F1FF3A1FFA8AFAC7F824903C6A34B1AE
:1062280023682046514698476468002CF8D1002D11
:10623800DCD1BDE8F0873868716B036889B298478C
:10624800002DD3D1F5E77868B16B036889B2984718
:10625800002DCBD1EDE7B868F16B036889B2984798
:10626800002DC3D1E5E7F868316C036889B2984717
:10627800002DBBD1DDE7F36A1FFA83FACEE700BF32
:106288001C4C08B5012102200AF09CFD237803F07C
:106298000502052A2AD003F00903092B08D000219A
:1062A80001200AF08FFD002108460AF08BFDFEE769
:1062B800114A124B11681A680B68114C4FF6FE70A0
:1062C80003400B601388206823F001031B041B0C98
:1062D800138018B12A2200238271C37102224E2131
:1062E8000AF0CCF920680AF057FDD8E71DF0A6FDA2
:1062F8002378D0E7F02A0020402300204423002000
:106308003C2B0020022828BF022010B4084C094B5F
:10631800207000EB8002C0EBC20207495DF8044B15
:10632800013003EB4203C0B20B602BF08DBC00BF01
:106338005B4C00200E8100202441002008B512F09B
:1063480043FFFBF74DFBBDE8084012F025BF00BF37
:106358002DE9F04F013085B0C3B203938E4D8F4FB6
:106368008F4C904E0A2302933220DFF8409226F099
:10637800FBFF4FF4FA7A4FF0100C4FF47A70D9F80B
:106388000430C3F30803002B40F0C880EFF31183F7
:10639800002B40F0C3802968A26800BF2B6899428F
:1063A800F9D1D7F800E000FB0EF39B1AB3FBFEF31C
:1063B80000FB01314FF0010E0191D9F80430C3F30D
:1063C8000803002B40F08E80EFF31183002B40F080
:1063D80089802B68A16800BF2A689342F9D1D7F851
:1063E80000B000FB0BF2521AB2FBFBF200FB0323D6
:1063F800019A9B1AB3F57A7FDFD3BAF1010ABED1AD
:10640800039B002B40F0C4804FF47A7ADFF89C910C
:1064180050464FF0100CD9F80430C3F30803002B92
:1064280040F09980EFF31183002B40F094802968A5
:10643800A26800BF2B689942F9D1D7F800E000FBA9
:106448000EF39B1AB3FBFEF300FB01314FF0010E74
:106458000191D9F80430C3F308033BBBEFF3118370
:1064680023BB2B68A16800BF2A689342F9D1D7F8EB
:1064780000B000FB0BF2521AB2FBFBF200FB032345
:10648800019A9B1AB3F57A7FE3D3BAF1010AC2D114
:10649800029B013B02937FF467AF4349434B444857
:1064A800444A0860DA6005B0BDE8F08FEFF3118860
:1064B8008CF31288A1682368DB0344BFC6F800E0A8
:1064C800A1682B6832685FFA88F888F31188D7F8D2
:1064D80000801A4400FB08F35B1AB3FBF8F300FBD7
:1064E8000233CDE7EFF311888CF31288A168236893
:1064F800DB0344BFC6F800E0A1682B6832685FFA86
:1065080088F888F31188D7F800801A4400FB08F34C
:106518005B1AB3FBF8F300FB023369E7EFF3118270
:106528008CF31288D4F808E02368D90303D5012333
:106538003360D4F808E02B683168D2B282F311884E
:106548003A68194400FB02F3A3EB0E03B3FBF2F322
:1065580000FB01312EE7EFF311828CF31288D4F897
:1065680008E02368D90303D501233360D4F808E091
:106578002B683168D2B282F311883A68194400FB5B
:1065880002F3A3EB0E03B3FBF2F300FB01315DE76B
:10659800184626F059FD37E7C4760020C876002053
:1065A80010E000E0C0760020FC9F002000ED00E035
:1065B800EFBEADDE0400FA0538B5434B5A89998918
:1065C800914224BF00225A81198ADA89914224BF54
:1065D8000022DA81DA788AB3072A2FD03B493C4D6A
:1065E80091F85300012400210A282C709C70D9715D
:1065F8003DD00C2865D0DFED377A8ABB364C9FED4D
:10660800370AA278002918BFF0EE407A062A04D883
:10661800334901EB820191ED000A217959B3013A1E
:10662800032A4DD8F7EE007A87EE800A2EF08CFC0C
:106638002388984228BF1846208038BDD97921B1CF
:1066480098780428B8BF04209870204890F8530020
:106658000A280CD00C28CED1DFED227A002ACDD022
:10666800072ACBD00A282CD1DFED1F7AC6E70A20EB
:10667800DFED1E7AC1E79B78154A07EE103A1178CC
:10668800B8EEC77A27EE277A07EE901AF8EEE77A7F
:1066980067EE877AB4EEE70AF1EE10FA10DDC0EE85
:1066A800077AFDEEE77A17EE903A102BA8BF102371
:1066B800012BB8BF0123DBB28B4238BF0B461370E6
:1066C80038BDDFED0B7A99E7F84F0020804D0020A8
:1066D800B83700206F1203391C5200206F1203389C
:1066E800946003080AD7A3390F506E3A5304E93867
:1066F8006F12833A2DE9F047A84FA94E12F064FDB6
:10670800BE421ED2DFF81483DFF81493444625886E
:1067180062197DB14A450DD2052D0BD933886188A0
:10672800C3F30B03994200F0DD80144625886219F3
:10673800002DEFD17168304614360AF080FFBE4252
:10674800E4D3984A1378A3F1170102290FD996497F
:1067580011F83300002840F0F180D800014449784E
:1067680029B1924911F83330002B00F00F81904B7A
:106778005A78022A40F2DC8000228E495A701A7830
:106788008D48022A016000F2CF8002EB82018B4B18
:10679800C2EBC10203EB4203998C5A8C884C91429C
:1067A800236001D300225A84864B9A78042A00F089
:1067B800E48032B91A88B2F5F07F84BF4FF4F072E2
:1067C8001A80814DFFF7F8FE2B68804A1A40002A8C
:1067D80000F0DF80D80700F1CB80590400F1C380B6
:1067E8001A0700F1BB809B0400F1B1802AF0EAF996
:1067F80010B977482AF020FE40200AF057FF802081
:106808000AF054FF4FF400700AF050FF4FF40030C4
:106818000AF04CFF4FF000700AF048FF4FF080601C
:106828000AF044FF1EF066F80021302269482FF074
:1068380048FB206825F08AFE674B276803F1500162
:1068480002E0043399426DD01A78002AF9D19C7875
:10685800D8788442F5D26149614B0D796149624823
:106868000A70624E624C8460C822642111FB0521C3
:10687800002259609A60DA601A615A619A61DA6195
:1068880083F8202083F82120376016F0C5FC594B87
:106898009FED595A1B88594A9FED596A50795949B1
:1068A80006EE903AF8EEE66A1388C5EE265A07EE29
:1068B800103A53881279C1ED005A07EE903AB8EEB3
:1068C800C77A514BF8EEE77A18725A7227EE067AB1
:1068D80067EE867ABDE8F04783ED017AC3ED007A6A
:1068E80012F05ABC63799B077FF41FAF716894F864
:1068F80004A030460AF0A3FE3388BAEB133F04D055
:106908001436BE42FFF402AF1BE773887068AA1FF3
:10691800C3F30B039A4204F10601A8BF1A462EF0EE
:106928003FF9EDE7012296E700221A70234B33E77F
:10693800204902EB420201EB820120E7D8000C1843
:106948006468002C7FF40AAF1724147006E72F48F8
:106958000AF0ACFE40200AF0A9FE47E72C480AF0EE
:10696800A5FE2B683FE72B480AF0A0FE2B6837E707
:1069780029480AF09BFE2B682FE79A8AB2F57A7F9E
:10698800BFF41FAF4FF47A729A821AE71823137074
:10699800EDE643F001032B601CE700BF0CC60308BB
:1069A80098C10308F83C0020908003086884030815
:1069B8005B4C00201A820020284100200E81002014
:1069C800244100201C52002060820020096000023F
:1069D800107B0020D81F002084340020C8430020EA
:1069E800F04800202C020020B81E00200C200020B7
:1069F800CA370020C4210020C0C9FB48901E0020CF
:106A080017B7D138C82100200443002009400002EC
:106A180001600002092000020860000202F0030879
:106A28000000040808B512F0CFFBFAF7D9FF12F0FE
:106A3800B3FBFFF75FFE0120BDE808402BF004B967
:106A48002DE9F047B54C82B0636820469847002886
:106A580000F0BF80B24B1B780122042B84F83C2045
:106A680000F0BA80B4F91610B4F91820B4F91A3045
:106A780021636263A363AB4B1B88002B69D0AA4DCB
:106A8800D4ED0C7AD5ED004A95ED050A95ED015A3D
:106A980095ED067AD5ED035A95ED026AF8EEE76AA8
:106AA800D5ED047AA4EEA60AA5EE267A67EEC07A9A
:106AB800A5EEC07AE6EE267A85ED057AC5ED067A6A
:106AC8002EF042FAD4ED0D6AD5ED094A95ED0E0A7D
:106AD80095ED0A5A95ED0F7AD5ED0D7AD5ED0C5A4C
:106AE80095ED0B6A2063F8EEE66AA4EEA60AA5EE19
:106AF800267A67EEC07AA5EEC07AE6EE267A85EDAC
:106B08000E7AC5ED0F7A2EF01FFAD4ED0E6AD5ED88
:106B1800124A95ED170A95ED135A95ED187AD5EDA9
:106B2800167AD5ED155A95ED146A6063F8EEE66AA3
:106B3800A6EEA40AA6EE857A67EEC07AA0EE657A7C
:106B4800E6EE867A85ED177AC5ED187A2EF0FCF90F
:106B5800A063764FA17F764816F0E0FA3B88002BB9
:106B68007CD1744EB568744B1B685B0742D4B5F989
:106B78000070216B636BA06B704A714E92ED026AD4
:106B8800D2ED006AD2ED015AC91B2163B5F9027032
:106B9800DB1B6363B5F904703568C01B07EE900A08
:106BA800B8EEE75A07EE901AB8EEE77A07EE903A91
:106BB800F8EEE77A36EE056A36EE877A77EEA57A4A
:106BC8000135A06382ED026A82ED007AC2ED017A96
:106BD800356002B0BDE8F0875A4BB4F91600B4F935
:106BE8001810B4F91A2018802063598061639A80BC
:106BF800A26340E7544F3B88322B7ED0002B5BD1F9
:106C080052480378002BB2D0DFF848E1716AB26AC3
:106C18008EFB01730027C9170770C1EB23118EFB88
:106C28000203D217C2EB2312F36A29806A80A08A72
:106C380047498EFB03E2DB17C3EB22131B1AAB8019
:106C4800CF6012F0C1FAFAF7CBFE12F0A5FAFFF7FF
:106C580051FD01202AF0F8FFB56888E7354E226B10
:106C6800B568B3F5C87F4FF0000323632B803988DC
:106C780018BFF068B7F8008008BF0020B1F5C87FDA
:106C880018BF3369616B02440B440020B8F5C87F14
:106C98006063F260336168803AD0D4F838E0716993
:106CA800A0637144B8F1010FA880716154D008F154
:106CB800FF38A7F8008056E7716A226B0023236328
:106CC8002B80B7F800E00A44BEF1320F616B6363B2
:106CD8006B807262A26B6BD0F06A0190B06AA3639A
:106CE80001440198B1620244BEF1010FAB80F26227
:106CF80063D00EF1FF333B8082E7154B2988D868B3
:106D08006A88AB88318330627283B3830021D4E709
:106D1800A36B7361A063A880C9E700BFD8400020B7
:106D2800CC3D00202438002028380020EC430020E7
:106D380008410020B81E00201C500020F842002006
:106D4800F4420020D03D0020D41F0020D11F002095
:106D5800C43700201F85EB51DFF80CC1DFF8F8E0DD
:106D6800C8328CFB02A9C833D217C2EBE9128CFBDC
:106D780003A9DB17C3EBE913C8316B802A808CFBAE
:106D8800013CA28ACB17C3EBEC139B1AAB80CEF85D
:106D98000C0012F019FAFAF723FE12F0FDF9FFF7CA
:106DA800A9FC40462AF050FFB7F80080B5687EE796
:106DB800A363B162F262AB809BE7234A234812685F
:106DC8002349037012F4003281F800E032D11346EF
:106DD8002049C85C0B2803F10C030ED00132182A95
:106DE800F7D1338B2B80728B1B4B6A80B18B326A45
:106DF800A980B7F800E0DA607BE71848D0F800C04F
:106E08005300BCF1000F09D003EB020E01EB8E0E0C
:106E18009CF801C09EF801E0E645E2D21344DFF891
:106E28004CE00F4A01EB830100230160AEF800300B
:106E38001360D6E70B4A1278032A01D01A46C7E72F
:106E48002AF000FEB568CCE7F42F0020D61F0020FA
:106E5800D01F0020BC750308C43700204021002043
:106E68002C220020547800201F85EB512822002076
:106E780038B50C4C0C4DAC4206D26168204614342F
:106E88000AF0DDFBAC42F8D3084A094B094C146000
:106E9800002209491A705A7008480860BDE838404D
:106EA8001EF0C8BC98C103080CC603082441002082
:106EB8005B4C00200E810020284100201A8200200F
:106EC80008B5FFF7D5FF12F07FF9FAF789FDBDE89D
:106ED800084012F061B9054B10B51A6B044C2178C3
:106EE800501C09B91A6310BD0246F8E7B81E002005
:106EF80036230020F0B50C292BD8DFE801F06F2AE3
:106F08002A2A4C2A2A2A2B2A2A2A0700046AB2F893
:106F18000CE097881668674D24F480540462036A6D
:106F28004468C16923F4005343EA0E3321F4E6416F
:106F3800A84243EA073341EA062100F0B58005F587
:106F48000065A84200F0B08092684460C1610264A4
:106F58000362F0BD046A96899588D2F800E0554F1F
:106F680024F480740462036A4468C16923F40073DA
:106F780043EA062321F07301B84243EA052341EAB4
:106F88000E017ED04C4DA8427BD092684460C1610E
:106F9800C2630362F0BD046A96899588D2F800E05E
:106FA800444F24F010040462036A4468816923F0A2
:106FB800200321F0807143EA061321F4E641B84228
:106FC80043EA051341EA0E2148D03B4DA84245D07B
:106FD80092684460816182630362F0BD046A9389A8
:106FE800B2F804E01768334E24F001040462056A1D
:106FF8004468816943EA0E0321F4803125F00205D3
:107008009BB221F07301B04243EA050341EA07014C
:1070180014D0294DA84211D005F54065A8420DD0DD
:1070280005F58065A84209D005F58065A84205D018
:1070380092684460816142630362F0BDD689158A13
:10704800578A23F0080333433D43D68824F4407419
:1070580023F00403ADB233432C43E9E7D589178AFB
:10706800D68823F0800343EA051324F44064558A44
:1070780023F0400344EA870443EA061344EA8504FC
:10708800A6E7D589178AD68823F4006343EA05233F
:1070980024F44054558A23F4806344EA071443EAED
:1070A800062344EA051470E7158A24F4804444EA68
:1070B800851449E7002C0140003401402DE9F04FC8
:1070C800F022002183B07848784CDFF80492784D9C
:1070D800784E794FDFF8FC812EF0F3FE7748784937
:1070E800DFF8F4E1DFF8F4C100221359834200F01D
:1070F800C180B3F1804F00F0BF80AB4200F0C88080
:10710800B34200F0C780BB4200F0C680734500F070
:10711800C580634500F0C480434500F0C380DFF8B4
:10712800C0A153457ED00AF5806A534508BF09239C
:1071380079D01432F02AD8D15C4C624D624E604F3F
:1071480004F1F00802E01434A04568D0A379002BBC
:10715800F9D023794FEA131909F1FF39B9F1050F6D
:1071680003F00F03EFD835F8190040FA03F2D207FD
:10717800E9D54FF0010A0AFA03F3013B18402DF054
:107188008DFA16F809305149184411EBC002DAD0CB
:1071980051F83000DFF84CE1217A00F138439B0ABE
:1071A8001EF8033003F01F0E5B09022B0AFA0EFAD1
:1071B80069D0032B62D0012B03D17B694AEA030310
:1071C8007B6193880093B3FA83F3C3F11F039BB2E7
:1071D800DA0800EB820203F00703D2F820E09B00F4
:1071E8004FF00F0C0CFA03FC2EEA0C0EC2F820E04C
:1071F800D2F820E001FA03F343EA0E03136269466A
:107208000023022214348DF804208DF805308DF8FF
:1072180006308DF8073022F0B5FCA04596D103B0B2
:10722800BDE8F08F082309EBC3034FF0010B93F877
:1072380020A00AF01F034FEA5A1ABAF1020F0BFAFC
:1072480003F30BD0BAF1030F0ED0DA457FF471AF18
:10725800D1F814A043EA0A034B616AE7D1F818A0F1
:1072680043EA0A038B6164E7D1F81CA043EA0A03E6
:10727800CB615EE70023D6E70123D4E7FB694AEA3E
:107288000303FB619DE7BB694AEA0303BB6198E717
:107298000223C8E70323C6E70423C4E70523C2E79C
:1072A8000623C0E70723BEE790410020188603089D
:1072B800000400400008004000100040002C01407D
:1072C800001002402888030834880308FC7E002048
:1072D800946003080040014000140040003401405D
:1072E800004401403C88030801490248FEF772BF88
:1072F800584200200048014001490248FEF76ABF91
:10730800304200200040014001490248FEF762BFB8
:10731800084200200034014001490248FEF75ABFE4
:10732800084200200034014001490248FEF752BFDC
:10733800E04100200004004002494FF08040FEF781
:1073480049BF00BFB841002001490248FEF742BFCB
:1073580090410020002C014001490248FEF73ABF45
:1073680090410020002C01402DE9F04104684E4D69
:10737800A30AAB427AD00AD94C4DAB425FD0023552
:10738800AB4277D0053DAB425DD0BDE8F081B3F5A7
:10739800801F67D04A3DAB4259D14FF0700E02268C
:1073A80047794FEA970C002968D0B00063468519E1
:1073B8000227D4F80C809F400CEB4503BFB23C4D2C
:1073C80003F1040C47EA080745F8231045F82C2078
:1073D800E760EFF31181502282F31288821905EBDE
:1073E800C2021369002B34D013620433821905EBEF
:1073F800C202576917B11F6053690433821905EB3C
:10740800C202976917B11F6093690433821905EBAB
:10741800C202D76917B11F60D36904330027CAB203
:107428001F6082F31188304405EBC000036A9BB9E2
:10743800E3684FF6FE721340E360BDE8F0814FF059
:10744800C00E0426ACE74FF0980E0326A8E7BDE867
:10745800F08105EB0E03C9E7E36843F00103E3603D
:10746800BDE8F0814FF0480E012699E74FF0200E55
:10747800002695E74FF0E80E052691E7BF0802239E
:1074880006FA03F0BB40DB43E768094D9BB23B407B
:1074980087190CEB470CE3600CF1040345F82C103A
:1074A80045F8232095E700BF4B001000500010005E
:1074B8009041002030B503685C4D18885C4CB4FBE3
:1074C800F2F20139013AAB4294B283B089B282B286
:1074D80066D05848834263D0B3F1804F60D0A0F59E
:1074E800983083425CD000F58060834258D052487F
:1074F80083425BD000F5806083427DD022F44072E5
:1075080000F58C3092B283421A80D9621C850ED065
:10751800484A93420BD002F54062934207D002F5E5
:107528008062934203D002F58062934201D1002227
:107538001A8601225A611A883C4992B242F0010225
:107548008B421A8062D0B3F1804F61D03B4A93429C
:1075580060D002F5806293425ED002F500629342E9
:107568005CD002F5806293425AD002F59032934281
:1075780058D002F54062934256D002F58062934299
:107588001ED002F58062934208BF092219D002A8D2
:107598004FF0012340F8043D22F0BEFA03B030BD9D
:1075A800254822F07002834292B2A3D101201A80AA
:1075B800D9621C8558611A8892B202431A80C5E7BD
:1075C80008221F4B03EBC20301A893F821408DF852
:1075D8000440012300228DF805308DF807308DF81E
:1075E800062022F099FA1B2CD8D1164B019301A83A
:1075F80022F092FA03B030BD01201A80D9621C85AE
:1076080058611A8892B202431A809CE70022D8E790
:107618000122D6E70222D4E70322D2E70422D0E7E8
:107628000522CEE70622CCE70722CAE7002C014054
:1076380000A24A0400340140001000400004004049
:107648009460030819010001204B98422DD0B0F135
:10765800804F2CD0A3F5943398422AD003F5806349
:10766800984228D003F50063984226D003F580633A
:10767800984224D003F59033984222D003F5406312
:10768800984220D003F58063984207D003F58063C1
:10769800984208BF092202D00020704708220C4BEC
:1076A80003EBC20393F8200070470022F7E701229A
:1076B800F5E70222F3E70322F1E70422EFE70522C8
:1076C800EDE70622EBE70722E9E700BF002C0140BF
:1076D800946003082DE9F04F013085B0C3B20393DD
:1076E8000B4602918B4C8C4E002B00F09A80322076
:1076F8008A4D8B4FDFF82C9225F036FE4FF4FA7A3C
:107708004FF0100C4FF47A70D9F80430C3F3080323
:10771800002B40F0DE80EFF31183002B40F0D9807E
:107728002968A26800BF2B689942F9D1D7F800E010
:1077380000FB0EF39B1AB3FBFEF300FB01314FF085
:10774800010E0191D9F80430C3F30803002B40F06F
:107758008780EFF31183002B40F082802B68A168AB
:1077680000BF2A689342F9D1D7F800B000FB0BF2AA
:10777800521AB2FBFBF200FB0323019A9B1AB3F5E2
:107788007A7FDFD3BAF1010ABED1039B002B40F008
:10779800BD804FF47A7ADFF88C9150464FF0100C88
:1077A800D9F80430C3F30803002B75D1EFF3118324
:1077B800002B71D12968A26800BF2B689942F9D1C2
:1077C800D7F800E000FB0EF39B1AB3FBFEF300FBB7
:1077D80001314FF0010E0191D9F80430C3F30803C9
:1077E80013BBEFF31183FBB92B68A16800BF2A68AC
:1077F8009342F9D1D7F800B000FB0BF2521AB2FB52
:10780800FBF200FB0323019A9B1AB3F57A7FE3D3BB
:10781800BAF1010AC4D1029B013B0293002B7FF409
:1078280066AF05B0BDE8F08FEFF311888CF31288CE
:10783800A1682368DB0344BFC6F800E0A1682B6891
:1078480032685FFA88F888F31188D7F800801A44FC
:1078580000FB08F35B1AB3FBF8F300FB0233D2E733
:10786800EFF311888CF31288A1682368DB0344BF07
:10787800C6F800E0A1682B6832685FFA88F888F3D8
:107888001188D7F800801A4400FB08F35B1AB3FB91
:10789800F8F300FB023370E7EFF311828CF31288E0
:1078A800D4F808E02368D90303D501233360D4F85A
:1078B80008E02B683168D2B282F311883A6819441B
:1078C80000FB02F3A3EB0E03B3FBF2F300FB013161
:1078D8007FE7EFF311828CF31288D4F808E023686D
:1078E800D90303D501233360D4F808E02B68316845
:1078F800D2B282F311883A68194400FB02F3A3EB71
:107908000E03B3FBF2F300FB013118E7184625F02C
:107918009BFB3EE710E000E0C0760020C476002024
:10792800C876002000ED00E0204B5B68C3F3080335
:1079380030B4BBB9EFF31183A3B91D4B1D4C1868C4
:10794800A16800BF1A689042F9D11B4B1C684FF41C
:107958007A7202FB04F3591AB1FBF4F130BC02FB52
:1079680000107047EFF31182102383F31288114936
:107978008C680B6813F4803F104B02D0012018600C
:107988008C680B49D2B20D68186882F311880A4BCB
:1079980019684FF47A72284402FB01F31B1B30BCB0
:1079A800B3FBF1F302FB0030704700BF00ED00E0CD
:1079B800C476002010E000E0C8760020C0760020E1
:1079C8002DE9F84F8046FFF7AFFF254E2549DFF830
:1079D800A0E0254A254D844610274FF47A740120EB
:1079E800DEF80430C3F30803D3B9EFF31183BBB94E
:1079F8000B68D2F808A000BFD1F800904B45F7D12A
:107A0800D6F800B004FB0BF9A9EB0A09B9FBFBF99E
:107A180004FB0393A3EB0C034345E1D3BDE8F88FC4
:107A2800EFF3118A87F31288D2F808B01368DB03E2
:107A380044BF2860D2F808B00B68D5F800905FFA08
:107A48008AFA8AF31188D6F800A0994404FB0AF34D
:107A5800A3EB0B03B3FBFAF304FB0933DAE700BF2C
:107A6800C8760020C476002010E000E0C076002030
:107A780000ED00E02DE9F04FDFF830C1474A4849F2
:107A8800484E494D8046102718F1FF38C0F08480D1
:107A9800DCF80430C3F30803002B5CD1EFF3118347
:107AA800002B58D10B68946800BF08688342F9D14D
:107AB800D6F800904FF47A7000FB09FEAEEB040E86
:107AC800BEFBF9FE00FB03EEDCF80430C3F3080349
:107AD8004FF47A740120FBB9EFF31183E3B90B6813
:107AE800D2F808A000BFD1F800904B45F7D1D6F8DE
:107AF80000B004FB0BF9A9EB0A09B9FBFBF904FB7D
:107B08000393A3EB0E03B3F57A7FBDD2DCF8043000
:107B1800C3F30803002BDFD0EFF3118A87F3128831
:107B2800D2F808B01368DB0344BF2860D2F808B065
:107B38000B68D5F800905FFA8AFA8AF31188D6F8AC
:107B480000A0994404FB0AF3A3EB0B03B3FBFAF37D
:107B580004FB0933D5E7EFF3118487F31288D2F8D1
:107B680008901368D80303D501232B60D2F8089036
:107B78000B682868E4B284F31188D6F800A04FF4A3
:107B88007A7400EB030E04FB0AF3A3EB0903B3FBBF
:107B9800FAF304FB0E3E97E7BDE8F08F10E000E033
:107BA800C4760020C8760020C076002000ED00E0F2
:107BB80030B4EFF31183102282F312880649074C80
:107BC8000A680748013200250A602560DBB20268AE
:107BD80083F3118830BC7047C4760020C07600203B
:107BE80010E000E00F4B1B88014643B90E4B0F4ACB
:107BF8001B7810680BB981F0010109F0D9B80C4B5A
:107C08005A691AB118B91A68106058747047094A45
:107C180018681188084A92FBF1F201210260597430
:107C2800704700BF9C7600209E760020A07600203A
:107C3800A4760020BC76002020A107001D4B70B55B
:107C48009C68236D626BDD69C2B1A36B2BB12B07F6
:107C580002D5236D08221A6270BD2A06F7D5A26ADA
:107C6800616A8A4220D0511CA069A162825C2069A5
:107C7800266D81423285EAD3A362E8E7A906E4D5F6
:107C8800E26A22B1988C216B80B29047DDE7E16906
:107C98009B8C6069DBB24E1CE6614354E169E36882
:107CA800994228BFE261D0E7226D136823F0800370
:107CB8001360CCE7F42A00201D4B70B55C68236D77
:107CC800626BDD69C2B1A36B2BB12B0702D5236DA3
:107CD80008221A6270BD2A06F7D5A26A616A8A422A
:107CE80020D0511CA069A162825C2069266D814266
:107CF8003285EAD3A362E8E7A906E4D5E26A22B1AD
:107D0800988C216B80B29047DDE7E1699B8C6069B4
:107D1800DBB24E1CE6614354E169E368994228BF2F
:107D2800E261D0E7226D136823F080031360CCE78B
:107D3800F42A00202DE9F04FBF4B1E788BB0002E9F
:107D480040F0BC80BD4BBE4C1D78DFF814A3DFF8B3
:107D58001493DFF8148305F00105A4F10A0B54F815
:107D68000A3CBBB1CC2707FB06B7184608F026F833
:107D780080B154F80A0C08F019F814F8023C8BB9D1
:107D8800242831D0F5B154F80A3C184608F016F802
:107D98000028EED10136032E04F1CC04DFD10BB05C
:107DA800BDE8F08F012B23D0022B2BD0032B37D02B
:107DB800042B67D0052B40D0062B4FD054F80A2C43
:107DC8001346D2E754F80A3C23281A4600F0878164
:107DD8009C4991F822108142C7D19B4BCAF8009068
:107DE800C3F80C801346C0E7012304F8023CCAE735
:107DF8004D2854F80A2C0CBF0223002304F8023C37
:107E08001346B2E700233C2804F8023C45D03E283C
:107E1800D4D10122032304F8012C04F8023CB2E770
:107E2800C02814D80022042304F8050C04F8040C14
:107E380004F8062C04F8023CA5E714F8063C14F8EC
:107E4800052C9A422FD814F8043C834203D000230F
:107E580004F8023C97E7062304F8023C14F801EC06
:107E6800BEF1000F00F08081BEF1010F00F0C48167
:107E780001360023032E04F8023C04F1CC047FF4FD
:107E88006EAF8CE714F8043C04F8030C5840052343
:107E980004F8040C04F8023C75E7032204F8013CDA
:107EA80004F8022C6FE714F8042CF9184240013347
:107EB80004F8042C04F8063C887264E7634B1868DD
:107EC80000283FF46CAF09F0F1FADFF8A0A1604D8B
:107ED800DFF89C91DAF8000007F070FF00283FF403
:107EE8005EAFDAF8000007F061FF09281BD03F28D1
:107EF80019D02B68002B66D1042800F0AC810C281F
:107F080000F0E6807F28E5D0A0F12002D2B25E2AF8
:107F1800E0D80BB92028DDD05A1C09F803002A60E4
:107F280023F014FBD6E72C68002C5AD1494B26467F
:107F380003F59478002E08BF1E4608334345F9D14F
:107F4800002E00F07C81A3F1080B3068DBF80020DC
:107F5800075D135D9F42204402EB040140F06D81F0
:107F6800671E4F4422460BB9FD2A5CD907F8013F2A
:107F780001322A6010F8013F11F801EF9E45F2D056
:107F88000AB1B34512D0344823F0E8FAB34508D310
:107F980056F8080B23F0E2FA092023F0D7FA5E45D9
:107FA800F6D92E4823F0DAFA2A680024944291D2AE
:107FB800661E4E4416F8010F23F0C8FA2B680134E8
:107FC8009C42F7D386E70C2800F082800A2851D01B
:107FD8000D284FD07F2800F0FC80FF2B3FF67AAFAA
:107FE80092E71C4F4FF0000B07F594785E4602E0CD
:107FF800083747450DD0224639684846F9F736FF15
:108008000028F5D1BB46002EF2D13E460837474539
:10801800F1D1002E99D1BBF1000F3FF45BAF0E48B0
:1080280023F09CFAB4E7511C202009F802002960CB
:1080380009F801300A46A4E77046002033560020AC
:1080480016440020107B002000ED00E03C2D0020AD
:10805800442E002074630308408B0308488B0308F0
:10806800FC9F0020EFBEADDE0400FA05402D002085
:10807800442D002023F0E8FA23217F482DF038FF13
:10808800002800F0E680A0EB0900286088B1431EB4
:1080980019F80310202940F0EC8009EB030204E0F2
:1080A80012F8011D202948D10346581E002BF7D18C
:1080B8002B604FF48072002148462DF002FF6F4B71
:1080C8001B78002B3FF46BAE6D4823F047FA01E7AD
:1080D8006C4823F043FA6A4823F040FAFAE66A4902
:1080E8006A48C9786A4ADFF8DCE15363003118BF8F
:1080F80001210170674991634021D36382F84010E0
:1081080082F84150644965480B603832CEF8002047
:108118005A4A0123137023F058FB594823F01EFADA
:108128004FF4006027F04CFE5D4B93F82230232B70
:1081380000F0978014F8023C3EE62B60594C002270
:1081480004F5947809F8032002E0083444457CD00B
:10815800216848460FF094F80028F6D0444574D2B8
:10816800636898470023A3E74F4BADF822E00FCB95
:108178000DF1280C02AF87E80F004CF824ED14F835
:10818800051C14F8033C069404EB010E62463946BC
:108198004FF0010C06A8CDF81CE0ADF820308DF8A2
:1081A80024C0FBF71FFAE8B9019F002304F8023C3A
:1081B800002F3FF4EFAD54F80A0C29F071F901369D
:1081C80054F80A0CB847032E04F1CC047FF4C7AD69
:1081D800E5E5013B002235482B6009F8032023F030
:1081E800BDF977E6029A324B03923946A4F10A00A8
:1081F800029309F02FFED7E714F8053C14F8032C76
:108208000694234407936E2A4FF0000308930993BA
:10821800ADF820207FF42CAE06A8F9F7A9FE06A831
:10822800F9F79AFE074606A8F9F796FE06A8F9F7A1
:1082380093FE204B1F6058601AE62246A0E61E48AF
:10824800A3F1080B23F08AF9A2E61C4823F086F96B
:1082580088E728681AE708480EF059FC0BB0BDE813
:10826800F08F174A14F8023CC2F80C80CAF8009044
:10827800A2E5034662E700BF442D002070460020B7
:10828800488B0308508B03085B4C0020AC2300206C
:10829800B81E00207DFA0008402D00207C8B0308C2
:1082A800107B00207463030800610308788B0308BF
:1082B800008400202C230020408B03085C8B0308DB
:1082C80000ED00E03C2D00202DE9F04F2DED068B50
:1082D800AB4BAC4A1C7897B000F59C4120318146E5
:1082E8000B911160002C00F0D986A74A12689042C1
:1082F80040F28380A54A06921668A549A54A0591C9
:10830800013C1C70A44B049206F480560893002E7E
:1083180040F08180A14B1B78022B01F00981042BCE
:1083280001F09D81012B01F051819D4B9945089BDE
:108338009B7800F28485002B40F08585994B079344
:10834800069B1E6816F4805740F07686DFF894A2E4
:10835800049BB3F90610059B5D8BA942B4BF0025A9
:108368000125914B1B6813F080535ED0079A127851
:1083780012F001025FD00598408C884241F3C18217
:10838800002D5ED1894C94F88C10002959D1884869
:108398008849006890F82D0000240C604C608C60BF
:1083A800854900284ED10870002A4FD0F1064DD5D6
:1083B800824A1278D20649D4002F47D1002B45D1E2
:1083C800740243D47E4B1B78002B02F04D827D4B08
:1083D8009B78002D42F0E0823BB17B4A7B4B1268D0
:1083E8001B689B1A002BC2F2E38210206F4C29F005
:1083F80045FB012384F88D3028E0644B06931E6802
:10840800644B634A049306F48056634B05920893C1
:10841800002E3FF47FAF00216348FAF765F9002882
:108428007FF478AF19F0D8FC74E770029ED4079AED
:10843800127802F001025D4C002184F88C10002DA6
:10844800A5D05D4901200870002AAFD1604B1A7889
:10845800002A79D10599049C488BB4F90070898B5E
:10846800B4F90240B842B4BF8026002646F0400363
:10847800B942D8BF33469B0843F08006A042B8BF34
:108488003346049F43F04006A142C8BF33469B08C9
:10849800B7F90440B7F9066043F08007A042B8BFB7
:1084A8003B4643F04007A142C8BF3B469B0843F008
:1084B80080073E4C8642C8BF3B4643F0400794F8CD
:1084C8008EE08E42B8BF3B469E4501F09584A4F8E5
:1084D800902084F892203A4984F88E300E78002E45
:1084E80001F053835F2B01F0E3836F2B01F0498484
:1084F800079B1B78DA0727D494F8921021BBB4F9AC
:108508009030322B20DD94F88E200120572A84F8F1
:10851800920001F09487069B1B685F0741F1A182D6
:108528005A2A41F09E8294F89430002B42F0B08190
:1085380094F8963083F0010384F89630002B42F0CB
:10854800F5810C2029F09AFA224B0993224B234DEE
:108558000A93069B1B685C0700F1EB860DF1500936
:108568001F4E0B950022C9F804203446149240F699
:10857800330B4FF0190840F28337049D37E000BFF2
:108588001C34002034330020183400201C500020F4
:10859800E47A002024780020F04800200A3C0020DB
:1085A800404B4C0033560020A43700203C1F0020CD
:1085B800244100205C3C002094210020F877002012
:1085C8002C020020E4370020C476002080420020DE
:1085D800C3460020C440002028410020204100203C
:1085E80084340020D43400200434544520D0A178A9
:1085F800E378994218FB0170F6D26178043118FBD0
:10860800037335F911105945A8BF5946B1F5617F73
:10861800B8BF4FF461718142E6DD9942E4DC21780C
:108628002729E1D848460434FAF74EF85445DED1F4
:10863800664A0B9D1378664A99E8030082E80300AE
:10864800002B40F02E86634B1A78002A00F0A8858C
:1086580001215F48FAF748F8002840F0E482089BB7
:10866800DB78002B40F0DF822B881FB227F0010750
:108678001FFA87F84345A5F8008001F00880564F97
:108688004FF002090E204FF0140B4FF0FF0A87F845
:10869800009087F801B087F802A029F0EFF9494661
:1086A8004B48B5F80080FAF71FF8002841F0CF8250
:1086B80028F002039BB243452B800BD0464B022087
:1086C8001421FF2218700E2059709A7029F0D6F9DB
:1086D800B5F80080414B424A197850680C9318F05D
:1086E800030F08BF81F00201C1F340010B9208F0AB
:1086F8005FFB24213648F9F7F7FF30B9079A13785A
:10870800590744BF23F004031370099B1B6813F037
:108718000A0F1BD005212E48F9F7E6FF002801F0C3
:10872800C6802F887B0741F1458229480621F9F741
:10873800DBFF002801F0A880780641F13382072189
:108748002348F9F7D1FF002840F0C4870C212048BE
:10875800F9F7CAFF2A88002800F0458342F480739D
:108768009A422B8009D01C4B022214211A700E2029
:10877800FF2259709A7029F081F91A4B1B78082B3F
:1087880000F03D830E2B00F03A83069BD3F800805F
:1087980018F4806F60D0144B1B79002B00F02582F1
:1087A80014210B48F9F7A0FF002840F0238225F098
:1087B800A9FC012029F0B0F800284AD0DFF82CA045
:1087C80000274FF0CC0BA14615E000BF4052002017
:1087D800A4370020704600201C3100208C76002031
:1087E80090760020F83C0020DC3E00200C4400205D
:1087F800DFB2022F2CD80BFB07F87B1C5AF8084075
:10880800002CF5D1032290F9023002940192C2782B
:10881800E24951F8222000921846224623460121B7
:1088280028F0FEFE034607EB470000EB0010099313
:1088380053B121460AEB8000CC222DF042FB099B64
:108848004AF808300137FFB228F0B4FB0028D0D12D
:108858004C46069BD3F80080079B93F800A0D04BAA
:108868001AF0010A00F0408201221A700A9B04994A
:108878001B68B1F906105A89CA4801279142077046
:1088880080F21882C84B4FF07E521A60059BC74F82
:10889800B3F81890049B97F90420B3F9003038789E
:1088A80097F801C0002AA3EB090714BF01224FF073
:1088B800FF32002FB8BF7F42B7F5FA7FA8BF4FF449
:1088C800FA77B84280F2F3813F1A07EE907AF8EE11
:1088D800E77AB74F4B45C7ED007A03DAF1EE677ACE
:1088E800C7ED007A049BB3F902E0AEEB0903002B55
:1088F800B8BF5B42B3F5FA7FA8BF4FF4FA7398424A
:1089080080F2D2811B1A07EE903AF8EEE77AF14529
:10891800C7ED017A03DDF1EE677AC7ED017A049BB2
:10892800B3F90400A0EB0903002BB8BF5B42B3F511
:10893800FA7FA8BF4FF4FA736345CCBFA3EB0C03CF
:10894800002302FB03F207EE902AF8EEE77A484587
:10895800C7ED027ABCBFF1EE677AC7ED027A18F468
:10896800805800F07E81B1F5FA6F924BA8BF4FF4A2
:10897800FA61B1F57A7F1A78B8BF4FF47A71A1F528
:108988007A71002A41F033818B4ADFF844E282FB96
:108998000130CB17C3EB6013581C6FF0630C3EF922
:1089A80010003EF913E00CFB0313A0EB0E0003FBD1
:1089B80000F382FB0312DB17C3EB62139E440FFA2A
:1089C8008EFE07EE90EAB8EEE78A87ED038AB8F1E3
:1089D800000F40F0A5832B885A0640F1FB807749A9
:1089E800774A91ED018AD2ED019A92ED026A91EDF2
:1089F800034A92ED030A91ED029A92ED007AD1EDC5
:108A0800005AD7ED011A97ED002A6E4A6E4938EEE2
:108A1800445A79EEC63A77EE007A65EE233A75EE57
:108A2800C96A75EE890A37EE401A66EEA76AB0EE93
:108A3800633AA0EE813A13F00303B0EE665A78EE7B
:108A4800044A79EE867AA0EE815AF0EE638AA4EEA3
:108A5800A73AD4EEA78AA4EEE75A33EE263AF0EE08
:108A6800687AF0EE674AF6EE008A35EE88AAE0EEFC
:108A7800C14A28EEC33A35EE635A77EE293A77EEC3
:108A8800E67AAAEE233A25EE285A76EE403A34EEF4
:108A980049AAE0EE817A74EEA64AAAEE235A34EE89
:108AA800094A37EE697A64EEA84A63EE036AE4EE8F
:108AB800074A75EEC85A36EE006A67EEA87AB0EE35
:108AC800667A95EE057AE5EE056AE5EE867AB1EE08
:108AD800648AF0EE665AF0EE476AB1EE674AE8EE4D
:108AE800246A63EE270A67EEA43AE4EE275AB1EE49
:108AF800450AB0EE606AB0EE631AA4EE277A23EE58
:108B0800244AE7EEA76AA5EE246AA0EE031AE8EE67
:108B1800245AB0EE448A31EEA19AE0EE240AA5EE7A
:108B2800278A66EEA16A72EE028AE5EE033A61EEE2
:108B3800211A26EE096AA4EEA47AA0EE274A0CBFF1
:108B4800D7ED022ADFED212A82ED005AA2EE256A2E
:108B5800E0EEA86AE2EE081A73EEA33A27EE227A4C
:108B680034EE044AF0EE005AE3EEA26AA4EE226A5A
:108B7800A1EEA57AC7ED016AC1ED366A81ED356AC5
:108B880087ED006A81ED377A82ED013AC2ED027A0B
:108B9800C2ED034AF3B987ED027A1BE01487030894
:108BA80034560020CC21002048210020BC3700206A
:108BB800EC3E0020E02200201F85EB51D40100206C
:108BC800E40100201C0200203C1F002000000000DF
:108BD800D0430020BAF1000F40F024811CF07AF84D
:108BE80017B0BDEC068BBDE8F08F079B1B78D90743
:108BF8007FF5DDAD4FF40F7022F074F900283FF4D3
:108C080028AE09F0C9FA4FF40F7022F0D3F8002803
:108C18003FF41FAE09F0C0FA4FF40F7022F0CAF803
:108C28000028EED115E6099B1B6898077FF51CAD57
:108C3800B5F8008018F0010F7FF43AAD48F0010351
:108C480098452B803FF434ADC14B022214211A7091
:108C58000E20FF2259709A7028F010FFB5F8008096
:108C680026E5059B5A8B9142C0F20785B1F5FA6F4C
:108C7800D4BFC2EB0101C2F5FA614FF47A7303FB6A
:108C880001F1B4480378C2F5FA62B1FBF2F1002BA6
:108C98003FF47AAE4378B04A01FB03F182FB01232B
:108CA800C917C1EB63116FE6DFEDAC7A2FE6DFED94
:108CB800AB7A0EE6B1F5FA6F80F2E284187A8B1A75
:108CC80003FB00F3C2F5FA6293FBF2F3C3F164030A
:108CD80007EE903AF8EEE77A9FEDA17AA14B67EE9E
:108CE800877AC3ED007AD1E51B780693002B7FF4D1
:108CF800BDAD9D4A1268002A3FF4B8AD9B4A079261
:108D080012F8030CDFF8A0B21146D71E1BF056FD6F
:108D18009BF80090079A002800F04A86069BB9F154
:108D2800000F41F0568507F1080178791BF046FDE0
:108D3800002841F061858E49B87A1BF03FFD002874
:108D480000F04986B9F1020F41F05E858949F87B48
:108D58001BF034FD002841F053858749387D1BF00E
:108D68002DFD002800F04986B9F1040F41F05C851B
:108D78008249787E1BF022FD002841F05185804908
:108D8800B87F1BF01BFD002800F04986B9F1060FDB
:108D980041F042857B4997F823001BF00FFD00281E
:108DA80041F03685784997F828001BF007FD002820
:108DB80000F04986B9F1080F41F01A85734997F810
:108DC8002D001BF0FBFC00283FF450AD0922134690
:108DD80002EB820217446E4A7878B9788BF8003033
:108DE8001070517042E522F480739BB29A422B8036
:108DF8007FF4B9AC674B1B78082B7FF4C3AC2A8887
:108E080022F040039BB29A422B803FF4BEAC504BF9
:108E1800022214211A700E20FF2259709A7028F02D
:108E28002DFEB2E40C9B19780B9B01F00101186828
:108E380007F0BEFF17B0BDEC068BBDE8F08F13B985
:108E4800089A01239370544B089A1D7892F8214090
:108E580007931B201BF0EAFC012C05F00108814652
:108E680000F0688705F00205089A4C4E92F8203009
:108E7800DFF838A14A4F09959346052B00F2D487AD
:108E8800DFE813F0BF00B5000600FD00FF00F200A8
:108E9800012C04BF05238BF82030B8F1000F12D045
:108EA800059B3088B3F918100022134661F30F02AE
:108EB80060F31F4261F30F03049861F31F430360DB
:108EC800032342600993374DDBF814102A68914256
:108ED80080F04B8647F230510322CBF81C108BF8F8
:108EE8002020022026F06CFF18F076FF2968DBF8B6
:108EF8001C200A440421CBF818208BF82010012CE0
:108F080040F0D8872A68DBF81810914280F08C87E7
:108F18009AF8000020B91BF089FC002840F08487EB
:108F28003A6822F002023A602A687388642101FBD9
:108F380003234FF480600022CBF810308BF82020F8
:108F48008BF8032026F00CFF9BF8203095E700BF34
:108F58001C310020E02200201F85EB51000000009A
:108F68000AD7233C4821002038560020EA30002048
:108F7800F4300020F9300020FE30002003310020BA
:108F8800083100200D310020123100201731002057
:108F98003C560020F83C002033560020C8430020EF
:108FA8001C410020C4760020000000202C02002074
:108FB8001BF042FC012807D1BB4D72882B68642145
:108FC80001FB0233CBF81030B9F1000F02D0B379AE
:108FD800002B4BD1012C00F02787B34DDBF8101084
:108FE8002A689142C0F0738701238BF82030012C46
:108FF8003AD0F379012B46D01BF09EFB9BF820302A
:109008003BE7B8F1000FD3D1099D4FF48060B9F167
:10901800000F00F05C8326F0BBFE089A0023136162
:10902800002D3FF48DA9284628F028FD069B1E68D0
:1090380016F480573FF48AA91D219C48F9F754FB80
:1090480000287FF483A99A4B03F1500A03E0043304
:109058009A4500F0EF861A78262AF8D19978DA78B6
:109068009142F4D2FFF774B98F4D5DE71BF064FBB2
:1090780003224FF47A738BF82020CBF81C308A4DEA
:109088002FE7894D3BE71BF057FB032240F6B83327
:109098008BF82020CBF81C30834D22E7854F3B7896
:1090A800002B01F0B282844BDFF82482DFF824B26F
:1090B800DFF824A2059345465E46049099460EE0E3
:1090C80019F804109847032C28DC88B93B782AF84B
:1090D800020F01349C4205F1040580F24F81072CF0
:1090E800E1B23046DBF80430EADD984700B2EDE73C
:1090F80038F824206B88801A4FF47A719B1A01FB88
:1091080000F040F6CA0290FBF3F00844904240F2A7
:10911800EE23A8BF10469842B8BF184600B2D5E75C
:109128001D216248F9F7E0FA28B100F03FBE043685
:10913800B4423FF450AC31782629F8D1B278F378AC
:109148009A42F4D2089BDB78002B7FF444AC574852
:10915800F9F7CAFADFED597A002801F06D8238EE86
:10916800678A574A5749FDEEC87ACDED047ABDF9AA
:1091780010301B0382FB0302DB17C3EBA212C9F5F5
:109188007A731BB203FB02F343F30F334B4407EE2E
:10919800903AF8EEE77A0123C7ED037A0B701AE4E8
:1091A800DFF83891DFF838A1474F0B9209F15A08D8
:1091B8004FF0010B494619F8010C1BF0FFFA00B3F8
:1091C80099F8040099F8023099F803E000EB40019F
:1091D80007EB8101013BD1F8A02003EB4303534483
:1091E80093420ED097F8CC20C1F8A0300BFA00F0CB
:1091F80022EA00000B9B81F89CE0C1F8A43087F8B4
:10920800CC0009F10609C145D4D1304B264A1B7858
:109218000B930A9BDFF8CCA012681B680C93AAF189
:109228009C094FF0000B9046DAF8043083B31F789E
:1092380077B3DAF80820A8EB0202002A0CDB99F8C9
:10924800CC20012101FA0BF122EA010208F5FA719A
:1092580089F8CC20CAF808100B9ACAB19AF80020ED
:1092680059780432D2B2002940F051830599049804
:10927800098B30F9122001F1C800824240F3EC85D5
:1092880099F8CC109A7841FA0BF3D90740F1778610
:109298000BF1010BBBF1040F0AF10C0AC4D1FFF763
:1092A800D7B9034B24E000BFC4760020A4370020C0
:1092B8008434002044350020E47A002000007A44F9
:1092C800D34D6210C02100203C1F0020C14800205F
:1092D80058350020203300203A1F0020013000209C
:1092E80010610308D81F00200433A3423FF4ABA940
:1092F80019782329F8D19878DA789042F4D29F48DF
:10930800F9F7F2F900283FF49EA99D4B1B6813F466
:10931800003341F0558200229A4B1046995C14297B
:1093280002F10C0201F0088101301828F6D1FFF78C
:109338008AB9954C94F896305BB1079B1B78D8078F
:1093480007D5049BB3F90620059B5B8B9A4200F373
:10935800088611218948F9F7C7F9002800F0BF826B
:1093680094F89A302BB994F8943013B93223A4F8AE
:109378009830012384F89A30FFF7F0B8DDF81090A0
:10938800824A06928249126842F2010AA1FB091B2D
:1093980012EA0A0A4FEA9B1B00F09E827D4D7E4826
:1093A8007E4C7F492E780078267008701EB17C4963
:1093B8000E7886F00106744C0F2184F82410002BD7
:1093C80000F01884059D774BB5F826C0B5F824E061
:1093D800059D109318462D8B0078734B129594F8C1
:1093E80025500995714D0495A3FB00535B0803EBC9
:1093F8004303C31ADBB20F90CDF834C002F4805295
:109408000C9304F128000BF59673CDF8449097F867
:109418000080DDF82490DFF8ACC10994634C0E910C
:10942800139200210A930896CDF81CE0089B002BA4
:1094380000F03D83099B079D33F911201FFA82FE36
:10944800AE454FEA410303D30D9DAE4540F2748308
:109458005CF82120934580F03483E25EBAF1000F76
:1094680040F0498301314145E25200F10600DDDB5D
:109478000E9A099C4E4B84F824200F2A49460CBFAB
:1094880001220022DDF8449084F825101A7000F0BB
:10949800B883484B4049424ADFF82CB108931C4630
:1094A800042001230B70137026F08AFCDBF80030CF
:1094B800A1686268E3605B1A934284BF002384F862
:1094C8002130069B3C781E68002C01F0D680059A56
:1094D800394DB2F824E0178B344916F480562846E3
:1094E80040F0C88332460EE0437803EB830303EB76
:1094F800830303F2EE239BB20132A24221F8023B1E
:1095080000F102000ED015F81230002B00F018837D
:10951800022BE9D001320B8821F8023BA24200F16C
:109528000200F0D1109A137801331370FEF7EFBEE2
:10953800059A0499537DD27D013B31F913301AB154
:10954800C3F53B6308331BB2A3F57A7307EE903A71
:109558009FED1A7A1A4AF8EEE77A40F2FF3167EE81
:10956800877AFCEEE77ACDED077ABDF81C308B429E
:1095780028BF0B461380FEF7D8BE00BFA4370020D3
:10958800F42F0020BC7503083C1F00201C5000204D
:10959800D34D6210FC3200209C010020C1480020FD
:1095A8009D01002039340020ABAAAAAA2478002003
:1095B800043D0020F04800208C3500206F12833FC6
:1095C800187800203C340020C4760020DA4CD4F807
:1095D8008830A9EB0303002BFEF6A7AED74AD84B79
:1095E800527C059933F812308A7DDFEDD66A9FEDFB
:1095F800D66AC97D9BB207EE102A07EE903AB8EEFC
:10960800C77AF8EEE77A27EE267A67EE867A0B9A1B
:10961800C4F88820C7EE876A40F2FF32FCEEE67A8B
:10962800CDED077ABDF81C30934228BF134609B127
:10963800D31A9BB2C548C64D0178C64C35F811609F
:10964800226825F81130921B13440131C24D236062
:1096580001F00F021B0902702B80FEF766BEFEF7B1
:1096680063F9BE4BBE4A1B68C31A93427EF75DAED0
:10967800B94B00221A80FEF758BE4146FFF701BBDE
:109688001B7AC3F1640307EE903AFFF723BB02216C
:10969800B448F9F729F800283FF40AA82F8018F0F1
:1096A800020F7FF417A848F0020343452B803FF4CC
:1096B80011A8AD4B022214211A700E20FF225970F6
:1096C8009A7028F0DBF9B5F80080FFF703B826F0A8
:1096D80047FBA2E4A54AB2F90030002BB8BF5B42B1
:1096E800B3F5E17FBFF632A8B2F90230002BB8BF5C
:1096F8005B42B3F5E17FBFF629A89D4B93ED096A5C
:10970800D3ED076A93ED057AD3ED037A76EE866A90
:1097180077EE877A76EEA66AB7EE007A37EE666A53
:1097280077EEA77AB0EEC66AF0EEE75AB4EEE56ACD
:10973800F1EE10FAB4BFB0EE655AB0EE465AB5EE87
:10974800405AF1EE10FA40F0DC839FED8A7AB4EECD
:10975800E56AF1EE10FA44BF9FED876A36EE477A64
:10976800B7EE006AF4EEC66AF1EE10FAC8BFDFED94
:10977800836AF5EEC07AC8BF36EEC77AF1EE10FA02
:1097880048BFB1EE477AF6EE007A27EE677ADFED4A
:109798007A7A77EE276ABDEEE66A16EE103A20333B
:1097A800402B40F28186DFED766A764ADFED747AE7
:1097B800C2ED006AFDEEC76AC2ED017A16EE903A74
:1097C8002033402BC2ED027A49D8DFED6C7AB4EE33
:1097D800E77AF1EE10FA41F343809FED6B6ADFED13
:1097E8006B6A01E0B0EE677AB4EEE67AF1EE10FA51
:1097F80077EE467AF6DC9FED667AF4EEC77AF1EEFC
:1098080010FA41F141809FED606ADFED626A01E084
:10981800F0EE477AF4EEE67AF1EE10FA37EE867A51
:10982800F6D4DFED557AB4EEE77AF1EE10FA40F3AC
:10983800D686DFED527A37EEC77A27EE076ADFED74
:10984800565ADFED566ADFED567AE6EE256A67EE80
:10985800065AE6EE267AA5EEA77AF0EE477A514B3D
:10986800C2ED037A1A6812F4003240F095864E4B26
:109878001046995C0A2902F10C0200F08585013036
:109888001828F6D1FEF762BF27F040039BB2BB420F
:109898002B803EF454AF344B022214211A700E2050
:1098A800FF2259709A7028F0E9F8FEF748BF2B8814
:1098B80023F00407BFB2BB422F803EF436AF2A4BD9
:1098C800022214211A700E20FF2259709A7028F073
:1098D800D5F82F88FEF729BF34490E7866E594F845
:1098E8009430002B3EF43AAE079B1B7813F001032B
:1098F8007EF434AE012284F8943084F89520FEF783
:109908002DBE0D4C012184F88C10FEF79ABD01295B
:1099180000F0588599F8CC20012303FA0BF30BF1DA
:10992800010B1343BBF1040F89F8CC300AF10C0A80
:109938007FF47AACFEF78CBE3C1F00203C760020FA
:109948005C7600200000C842000080440B3C0020E8
:10995800103C00200C3C002018780020A81E002095
:1099680060E31600A43700201C310020D0400020FE
:10997800F4010020A7DFA834DB0FC93FDB0F494003
:1099880000000000D4010020DB0FC940E4CB1641E1
:10999800DB0F49C0E4CB16C192E741B99730083CC8
:1099A80015A82ABEF42F0020BC750308C148002062
:1099B800511D78791AF002FF00283FF4BCA9B9F1CB
:1099C800010F40F0198707F10D01B87A1AF0F6FE79
:1099D800002840F01987C149F87B1AF0EFFE0028EB
:1099E8003FF4BBA9B9F1030F40F00A87BC49387DA1
:1099F8001AF0E4FE002840F01787BA49787E1AF07A
:109A0800DDFE00283FF4BBA9B9F1050F40F0088737
:109A1800B549B87F1AF0D2FE002840F0FD86B34958
:109A280097F823001AF0CAFE00283FF4BBA9B9F141
:109A3800070F40F0ED86AE4997F828001AF0BEFEF1
:109A4800002840F0D586AB4997F82D001AF0B6FEED
:109A580000283EF40BAFB9F1090F3EF407AFFFF74A
:109A6800B5B95D2A00F090825B2A00F0D2855E2AA3
:109A780000F08C86562A00F08E86972A00F0D88649
:109A8800A72A00F077869C4D2B889E0740F04286D7
:109A9800A2F1B703072B00F2B182DFE813F0A102AD
:109AA800AF02AF02AF029302AF0285028502079BA5
:109AB800002B3FD05CF8212093454FEA4103FFF487
:109AC800CCAC8E4A8D4DD25C05EB030E002A00F01B
:109AD800B180022A47D19EF8012002EB820202EBF4
:109AE800820202F2EE2292B2032933DD12B2BAF1F7
:109AF800000F3FF4B7AC0C9D20F81520B9F1000F0A
:109B080003D10F9D022D7FF6ADACB0F8029002880C
:109B1800B0F804E04A449644794A0FFA8EFE82FB74
:109B28000E52784DA2EBEE7225F803E012B24FF018
:109B3800010997E41A464B000A9D4CF821508DE420
:109B4800D3B2022B04D9032B7FF4E4AC7346D3E4DD
:109B58003B46D1E4012505FA01FE0E9D25EA0E05D6
:109B680012B20E957AE4E25ABEE7674A1278002AE2
:109B78007FF4B0A9B8F1000F3FF4ACA9012C40F074
:109B880053819BF82030FFF778B931465F48F8F7E2
:109B9800ABFD002800F0D18084F8936018F00AFC2F
:109BA800FEF7A6BC47F04003BB422B807FF473AEA0
:109BB800FEF7C5BD47F004039F422B800AD0544BE3
:109BC800022214211A700E20FF2259709A7027F071
:109BD80055FF2F884F4B504AB3F904304F4982FB49
:109BE8000302DB17C3EBA2030B80FEF79EBD5B7875
:109BF800FFF751B84A4B4B4A109201221A704A4B50
:109C080004931B214148F8F76FFD00287FF441AC0D
:109C1800464BDFF81CB108931946DBF80030CA68D8
:109C28008B609B1AC82B00F2F884069B1E6806F40A
:109C3800805677E4CAB2022A40F2C183032A92D13D
:109C4800129A139D079E002D08BF32464CE728F054
:109C580001039BB243452B803FF421AD0E2087F8CA
:109C6800009087F801B087F802A027F007FFB5F841
:109C7800008014E500220FE0437803EB830303EB35
:109C8800830303F2EE239BB20132A24221F8023B86
:109C980000F102003FF446AC15F812301BB1022B5C
:109CA800EAD00B88F0E7D3B2032BFAD83B46EBE7B0
:109CB800B2F5FA7FFEF648AC94F89230002B7EF4A9
:109CC80043AC079B1B7801210B4084F8921000F0ED
:109CD800D38318F081F8FEF737BC00BFF9300020B5
:109CE800FE30002003310020083100200D31002013
:109CF8001231002017310020204100208C3500202F
:109D080056555555AC1F002084210020A43700204B
:109D18001C310020D040002067666666C221002002
:109D2800043D00203934002024780020F048002029
:109D3800C47600200025FFF797B8079BC14A1B7817
:109D48001060D8077EF5D8ABBF4B1B78002B3EF4CC
:109D5800FBAB089BDB78002B7EF4F6AB94F89330D2
:109D68000133DBB2032B84F893307EF6EDABB74BAF
:109D78005B7813B9002D7EF4E7AB18F02DF8FEF7E9
:109D8800B7BBB2F5FA7FFEF6DFAB94F89230002B42
:109D98007EF4DAAB079A1278012184F89210D10781
:109DA80000F12A8418F006FBFEF7CEBB089BDB788F
:109DB800002B7FF4C0A9DFEDA67AA64938EE678AA2
:109DC800C9F5FA63FDEEC87A1BB2CDED047ABDF988
:109DD8001020120381FB0201D217C2EBA11203FB70
:109DE80002F343F30F334B4407EE903AB8EEE78A99
:109DF80087ED038AFFF79FB9974A96491068B4F927
:109E08009020C66981FB06018911F617701A00F5C2
:109E1800FF407F3082423EF75EAB891B0A4412B294
:109E2800A4F89020FEF757BB099D002D3EF488AAA0
:109E3800FFF7F9B8894A059BD588049A1B8BB2F9B4
:109E480006105A1B914240F389802B449942B4BFB3
:109E580000250125FEF785BAC8398A4242DA99F801
:109E6800CC109A7841FA0BF3DB073FF511AA52425E
:109E780001200D9227F0E8FE7B1E0D9A162B00F2AA
:109E88008581DFE813F006021A02EE013F022E0276
:109E98005302D901C401AF019A01860183013F022F
:109EA80075015302D901C40161014D0139016802EC
:109EB80023010F01AB460899DBF80020CB69099D07
:109EC80013448B61002D3EF43BAAFFF7ACB81AF09F
:109ED80033FC032140F6B8328BF82010CBF81C2055
:109EE800FEF7FFBF99F8CC30012202FA0BF223EA01
:109EF800020308F5FA7289F8CC30CAF80820FFF78F
:109F0800C7B9B4EEE56AF1EE10FA8CBFB0EE654A57
:109F1800B0EE464AC4EE054A9FED512A9FED515ACC
:109F2800DFED511ADFED512A9FED513ADFED513A3D
:109F38009FED514AA4EE825AE4EEE12AA4EE857A16
:109F4800A4EEA23AB0EE475AB0EE637AA4EE837A52
:109F5800A4EE874A84EE057AFFF7F9BB0125FEF7E0
:109F680000BA00214548F8F7BFFB00287FF4F1A9A3
:109F7800322384F89600A4F89830FFF7EAB9002A4B
:109F88000CBF0120022074E73D4B002201203D490F
:109F98003D4C0B603D4B09933D4B22703D4D0A9360
:109FA80027F052FEFEF7D5BA394A374B0A921146C6
:109FB800394A0A6002225A70344B09931AF09AFC03
:109FC800FEF7C7BA324A304B0A921146334A0A6042
:109FD80000225A702D4B09931AF08CFCFEF7B9BA7F
:109FE8002B4A294B0A9211462D4A0A6001225A70BF
:109FF800264B09931AF07EFCFEF7ABBA9E2A00F0B6
:10A008008D849D2A00F08284AE2A00F07784AD2AE0
:10A0180000F06C84EF2A00F06684FD2A00F0518479
:10A02800FB2A00F08C84FE2A00F08684F72A00F0D0
:10A0380080847B2A00F03E84144B0993144B0A93C6
:10A04800FEF787BA84420020C1480020E437002088
:10A0580000007A44D34D6210407A0020AC430020BF
:10A0680099FB243F69A2163E39094E3DE3B59E3E51
:10A0780088FA163E45FE7F3FA7DFA834A4370020A4
:10A088000E810020244100205B4C0020C4400020A9
:10A098002841002020410020328200201A8200201E
:10A0A80026820020D9F8D000B64B90F836109B785D
:10A0B80011446429A8BF642121EAE17180F83610AF
:10A0C800002B40F0518422F099FB23E4D9F8D0000A
:10A0D800AC4B90F837109B781144FE29A8BFFE219D
:10A0E80021EAE17180F83710002BECD016201AF025
:10A0F800E7FBD9F8D000E6E7D9F8D000A14B817882
:10A108001144C829A8BFC82121EAE17181709B7850
:10A11800002BD8D014201AF0D3FBD9F8D000D2E7FE
:10A12800D9F8D000974B41781144C829A8BFC82155
:10A1380021EAE17141709B78002BC4D013201AF0FA
:10A14800BFFBD9F8D000BEE7D9F8D0008D4B017815
:10A158001144C829A8BFC82121EAE17101709B7880
:10A16800002BB0D012201AF0ABFBD9F8D000AAE728
:10A17800844B0C989B78417911446429A8BF6421C9
:10A1880021EAE1714171002B40F01A84D9F8D0001E
:10A1980099E7D9F8D0007B4B017A9B781144C829FC
:10A1A800A8BFC82121EAE1710172002B8BD00B20D6
:10A1B8001AF086FBD9F8D00085E7D9F8D000714BA2
:10A1C800C1799B781144C829A8BFC82121EAE17147
:10A1D800C171002B3FF477AF0A201AF071FBD9F850
:10A1E800D00070E7D9F8D000664B81799B7811448C
:10A1F800C829A8BFC82121EAE1718171002B3FF469
:10A2080062AF09201AF05CFBD9F8D0005BE7D9F8F7
:10A21800D0005C4B417993F802E01144C829A8BFEB
:10A22800C82121EAE1714171BEF1000F40F08A8333
:10A23800112F7FF464AF46E7D9F8D000514B01796C
:10A2480093F802E01144C829A8BFC82121EAE171A6
:10A258000171BEF1000F40F09583102F7FF463AFBA
:10A2680031E70C99474B0F790D931744642FA8BF1A
:10A27800642727EAE7770F711AF03CFB0D9B9B7860
:10A28800002B83D0032039461AF01AFBD9F8D000E6
:10A2980019E70C983B4B01781144FA29A8BFFA2119
:10A2A80021EAE17101709B78002B3FF46FAF012028
:10A2B8001AF006FBD9F8D00005E70C98314B8178E5
:10A2C80011446429A8BF642121EAE17181709B7857
:10A2D800002B3FF45BAF02201AF0F2FAD9F8D00055
:10A2E800F1E60C98274BC1799B78114481F308015A
:10A2F800C171002B3FF44AAF05201AF0E1FAD9F8F2
:10A30800D000E0E60C981F4B817993F802E01144E5
:10A318006429A8BF642121EAE1718171BEF1000FAF
:10A3280040F01A830D2F7FF424AF2FE7D9F8D0001F
:10A33800144BC17893F802E01144C829A8BFC8217A
:10A3480021EAE171C170BEF1000F40F011830F2FB7
:10A358007FF4FDAEB7E60C980A4B41781144B1F58D
:10A36800967FA8BF4FF4967121EAE17141709B78FE
:10A37800002B3FF40BAF15201AF0A2FAD9F8D00041
:10A38800A1E600BFFA770020C449D1F800E04200F6
:10A39800BEF1000F08D0171803EB87079EF801E0FD
:10A3A8007F787745BEF4D2A91044BD4FBD4A03EB70
:10A3B800800300200B6038801060FEF7C7B9129A3E
:10A3C800FFF792BB04999B7831F91220B2F5617FAF
:10A3D8004FF4966191FBF3F3C0F2E68040F6330147
:10A3E8009142A8BF11460C2FA1F5617191FBF3F1C1
:10A3F80000F0FC81182F7FF48DAAC9B2C8290B463A
:10A40800A8BFC823D9F8D020D77DD8B2B8423FF426
:10A4180081AADF1BA44BD07548BF0737FF109B7874
:10A428000137FFB23BB9002F3FF474AA384627F032
:10A438000BFCFFF76FBA18201AF042FAF3E79B4AB1
:10A448009B4B099210461A689A494FF47A73B3FBEA
:10A45800F2F3C3EB431203EB82030268DB00A1F8BB
:10A46800A83053077EF572A8934B944D0A221A80A0
:10A47800934B0A93FEF76DB89249096811F40031BD
:10A4880040F09881904B08465D5C0F2D01F10C015E
:10A498006DD001301828F7D1FA3A0023A4F890209B
:10A4A80084F89230FEF750B8B4EEE77AF1EE10FA7D
:10A4B80040F3D381DFED855A9FED856A01E0F0EE28
:10A4C800676AF4EEC66AF1EE10FA76EEE57AF6DC23
:10A4D800DFED806AF4EEE67AF1EE10FA40F1B3812E
:10A4E800DFED7A5A9FED7C6A01E0F0EE667AF4EED1
:10A4F800C67AF1EE10FA77EEA56AF6D4DFED777A30
:10A50800F4EEE76AF1EE10FA40F3BB80DFED747AFF
:10A5180077EEE66A66EEA65A9FED725A9FED726A6A
:10A52800DFED727AA5EE856A26EEA55AE5EE867A03
:10A53800E5EE276AFFF739B95849D1F800E042003B
:10A54800BEF1000F08D0171803EB87079EF801E04B
:10A558007F787745BEF477A80244514F514803EB02
:10A56800820300220B603A800260FEF76CB84B4908
:10A578000F68450037B12E1803EB86067F7876788A
:10A58800BE4289D20544464E464803EB8503002562
:10A598000B60358005607FE7554B1B78032B00F077
:10A5A80021810022FFF763B90C2F40F015810027A5
:10A5B8003946504B0E915B78BB423FF4ABA93A4BFE
:10A5C8000D93384618F092FD0D9B0E999B781BB1A0
:10A5D800C9B20C201AF074F90137FFB223E7DFED96
:10A5E800467AB4EEE77AF1EE10FA44BFDFED397A35
:10A5F80037EEC77AFFF721B9404A2C491360304B30
:10A6080009912E4D0A93FDF7A4BF3D4A0592FEF726
:10A61800B7BE3C4B01220220B9E43B4A069B1E68A8
:10A62800136823F004031360089A012306F4805684
:10A6380082F82130FEF776BF38EE678A334B34490B
:10A648001870FDEEC87AC9F5FA63CDED047ABDF944
:10A658001020120381FB0201D217C2EBA1121BB218
:10A6680003FB02F343F30F334B4407EE903AF8EE43
:10A67800E77AC7ED037AFEF7AEB906F48056FEF71F
:10A6880051BFDFED1D7AF4EEE76AF1EE10FA44BF30
:10A69800DFED107A77EEE66A3CE700BF4021002044
:10A6A800282200202C220020FA770020C440002015
:10A6B8000C500020804D0020EA430020204100205B
:10A6C80028410020F42F0020BC750308DB0FC94087
:10A6D800E4CB1641DB0F49C0E4CB16C1DB0FC93F01
:10A6E800DB0F494092E741B99730083C15A82ABECC
:10A6F800547800205B4C0020DB0FC9BF8442002047
:10A70800E47A00205C8100201C410020C021002048
:10A71800D34D62100023BB2A149300F0C880B72AD7
:10A7280000F0C180BE2A00F09680BD2A7FF466AC96
:10A738004FF6FE71A64AA748D689099090893344F6
:10A748000144D38191810EF03FFDF7F749F90EF0EE
:10A7580023FDFBF7CFFF012027F076FAB4F89030FD
:10A768009D4A0A92FA3B0022A4F8903084F892207D
:10A77800FDF7EFBE994A974B09931378984D43F02C
:10A7880004031370944B0A93FDF7E3BE954B022222
:10A798000320FFF7FCBB0EF017FDF7F721F90EF0C9
:10A7A800FBFCFBF7A7FF012027F04EFA94F88E2058
:10A7B800FFF763B98C490978032947D0194661E640
:10A7C800894B1B78032B7EF4A6AD27F03BF9FDF7E8
:10A7D8003ABF1A46FEF7FCBA182F7FF49BA800214F
:10A7E8000B460FE627F02EF9FDF7B0BFCFB2E0E633
:10A7F80008221346FEF7ECBA01221346FEF7E8BA20
:10A8080003221346FEF7E4BA02221346FEF7E0BA23
:10A8180007221346FEF7DCBA06221346FEF7D8BA1B
:10A8280005221346FEF7D4BA04221346FEF7D0BA1F
:10A838006E4B684A09924FF4C8721A80664B684D8D
:10A848000A93FDF786BEF0EE676A57E627F0FAF836
:10A85800B4F9902020E602216CE7F0EE667A37E63C
:10A86800F0EE477AFEF7C7BF002D3DF4BEAD604C51
:10A8780094F88D30002B3DF4E9AD27F0E3F8002380
:10A8880084F88D30FDF7E2BDB0EE677AFEF7C9BFF8
:10A89800504B0993504B84F8941084F89500504D10
:10A8A8000A93FEF747BD19464FF6FE7342E719466D
:10A8B80002233FE74FF4FA61022018F035FBFFF757
:10A8C800BBBB0021012018F02FFBB4F89030414A9F
:10A8D8000992963B404AA4F8903000230A9284F8E3
:10A8E8009230FDF736BE00210846ECE7FF21002034
:10A8F8001FF0EEFB94F88E20FFF78CBB012100209F
:10A908001FF0E6FB94F88E20FFF781BB0021FF20A3
:10A918001FF0DEFB94F88E20FFF776BB00210120A4
:10A928001FF0D6FB94F88E20FFF76BBB0B20FDF7CA
:10A9380009BE00210420C6E700210320C3E7002147
:10A948000220C0E711200E930D9219F0B9FFD9F833
:10A95800D0000E9B0D9A6BE40D200E930D9219F00A
:10A96800AFFF0E9B0D9ADDE4172019F0A9FF0DE447
:10A978000F200E930D9219F0A3FFD9F8D0000E9B6B
:10A988000D9AE4E410200E930D9219F099FFD9F86E
:10A99800D0000E9B0D9A60E4002B3FF468AF154978
:10A9A800154A09684FF47A7000FB031313605EE7D9
:10A9B8000F4C17F011FA002384F88D30FDF746BDCF
:10A9C8000E2019F07DFFD9F8D000FFF77CBB00BF3F
:10A9D800C4370020C440002028410020F877002018
:10A9E80020410020AA81002054780020EC43002058
:10A9F8003C1F0020C4760020804200202DE9F04F43
:10AA08002DED0E8BDFF8A8A393B0DAF8043004908C
:10AA180050469847002875D0BAF8A85000228AF8FE
:10AA28005120002D41F07684DAF84830BAF93C60BC
:10AA3800BAF93800DAF82050BAF93A10DAF82440AE
:10AA4800DFF870B3F71A87EAE772A2EBE772B2F59C
:10AA5800804FDAF82820DCBFCAF848603346401B2C
:10AA6800091B9B1ACAF82C00CAF83010B4489AF887
:10AA78005210CAF8343012F051FBDBF8003099005C
:10AA880041F16085DAED0C5ADFF82C93DAED0B7A98
:10AA9800AC4999ED406AD9ED416A99ED427AD9F805
:10AAA8000C210968A84B0293B8EEE58ADAED0D5A35
:10AAB800F8EEE77AF8EEE58A013277EE867A38EE34
:10AAC800268A78EE878A8A42C9ED407A89ED418ADA
:10AAD800C9ED428AC9F80C2102F088821F78142F28
:10AAE80003F0DF810023D9F814410393062C01F207
:10AAF800B781DFE814F0CB1551158E148D16250992
:10AB08006215EE14904BDFF8B0921C780293072C74
:10AB180001F0F98199F82831069353B15F1E89F83D
:10AB28002871012C01F0C48413B0BDEC0E8BBDE874
:10AB3800F08F864A5279002A01F05982844A1278A5
:10AB4800013AD2B2072C89F8282102F01083002399
:10AB580007938049D9F83421D1ED006A7E490591DF
:10AB680004999FED7E6AD9ED4C9A7D4BDFF84CB283
:10AB78001B6899ED4BDADFF848829FED7A9ADFED92
:10AB88007AAA9FED7ACA9FED7AAADFED7ABA9FED8D
:10AB98007ABA7A4F7A4ECDF80CB08A1A07EE902A14
:10ABA800F8EE677AB7EE007AC6EE278A0024C9F86D
:10ABB800341125469B4677EE69CA6CEEA6CAF4EEB8
:10ABC800C7CAF1EE10FA88BFF0EE47CA6D4B98ED90
:10ABD800008A2344D3ED007AF5EE407AF1EE10FABC
:10ABE80017D0694B234493ED007A78EE476AB0EEAC
:10ABF800E66AF4EEC67AF1EE10FA08D5F5EEC06A08
:10AC0800F1EE10FACCBF37EE878A37EE678A83ED0C
:10AC1800008A5E4B1A88930739D0022D37D09BF8EB
:10AC28002E105B4B07EE901A234493ED007A4B42AB
:10AC3800F8EEE76A07EE903A26EE877AF8EEE77ABA
:10AC4800B4EEE77AF1EE10FA0AD407EE901AF8EEAD
:10AC5800677AF4EEC77AF1EE10FA88BFF0EE477A19
:10AC68004C4B4D4903EB450331F91500B3F90C3052
:10AC7800C31A07EE103AB8EEC77AD007E7EE497A5A
:10AC880041F14B81454B93ED008A27EE888A059B5D
:10AC980099F86821234493ED01EA78EE4EDA002A08
:10ACA80000F0DA803E4BD9F86C2104991B688A1AA7
:10ACB8009A4240F3D1809BF84830022B02F0A682DA
:10ACC800022D04F0D385374B1B6899077AD4364B8D
:10ACD80086ED00CA1B689342C0F2AE80F7EE007A98
:10ACE800F4EEE79AF1EE10FA40F1B68005992F4B91
:10ACF800D1ED017A93ED007AF0EEE77AF4EEC77AB7
:10AD0800F1EE10FA40F1A880D1ED027AF0EEE77A80
:10AD1800B4EEE77AF1EE10FA40F39E80D1ED037AB3
:10AD2800F0EEE77AB4EEE77AF1EE10FA40F39480A9
:10AD38001C4B1B689B077FD51749164B63E000BF68
:10AD4800AC4D002098380020CC3D0020F84F002062
:10AD5800B8370020107600200C50002000247449D9
:10AD680024410020CDCCCC3DAE47813F00000000FF
:10AD78000000C84200003443610BB63B683C002029
:10AD88005C3C002004760020602100202041002047
:10AD98006C210020C4370020D0400020EC75002032
:10ADA80018760020C4400020147600202076002069
:10ADB800804D00201C5000201C200020503C00200A
:10ADC80054210020D34BD449DFF8C8E331F915C02A
:10ADD8009EED008ADFF8C0E386ED00CA03EB45006C
:10ADE80028EE098AB0F90C00A0EB0C0007EE900AD7
:10ADF800F8EEE77ADEF8000027EE888A904278EECF
:10AE08004EDABFF66BAFB3F90C20B1F900E0C348D6
:10AE1800AEEB020E00688EEAEE72A2EBEE72824290
:10AE28001ADAB3F90E30B1F90220D21A82EAE273C3
:10AE3800A3EBE27398420FDDB94B1A88002389F817
:10AE48006831002A43F08B86B64AB74B11781868E8
:10AE580081F0010105F0ACFFB44B234493ED000AE7
:10AE6800039B2DEE000A022D20EE2D0AA3EC010A09
:10AE7800039304F0AD84AE4BD6ED006A93ED007AEF
:10AE8800AC4BD3ED007AAC4B93ED006AAB4B67EE5D
:10AE9800277A234427EEAC7AD3ED007A67EE277A37
:10AEA800F0EE665AEDEEA75AB1EE467AB4EEE57AC0
:10AEB800F1EE10FA08DCF4EEC65AF1EE10FA8CBF87
:10AEC800B0EE467AB0EE657A99ED4C6AF7EE007A04
:10AED800B4EEE76AF1EE10FAACBF0123002343B1E8
:10AEE800F0EEE66AF0EEC77AF4EEE67AF1EE10FAE2
:10AEF80001D586ED007A022D04F0D283904A914B59
:10AF080052F825001B68B0EE4E0A98478E4A8F4BC0
:10AF180052F825001B6898479BF8373023B18C4BB3
:10AF28001B88002B01F0EE80B0EE4C8A894B38EE7E
:10AF3800400A234493ED008A83ED000A9BF84830C9
:10AF480030EE480A20EE288A002B33D0824B1B783B
:10AF580013F0010300F0BF86F7EE007AF4EEE79AEB
:10AF6800F1EE10FA99F86831C1F2C185002B01F0B1
:10AF78007981D9F86C31049AD31A784A12689A42BE
:10AF880018DD774BD3ED007AF0EEEDDAF4EEE7DA80
:10AF9800F1EE10FA42F14B81614B1A88002389F8CF
:10AFA8006831002A00F0A3866E494A6912B10A681E
:10AFB80013604B746C4B99F87821234493ED000A85
:10AFC8002DEE000A20EE088A87ED008A32B9039B2D
:10AFD80086ED00CA03ED01CA87ED00CA0135032DCD
:10AFE80008F1040807F1040706F1040604F1040453
:10AFF8007FF4ECAD029B1A78072A01F08E85012AAE
:10B0080002F0A3800023059399F88021002A41F0DB
:10B018008382DFF888B1554BDBF800201968D50426
:10B0280091F82C0001F19A80DFF87481504AB8F841
:10B038001A30D2ED005A4F4A4F4CD2ED004AD4EDA7
:10B04800036A4E4AC9ED645A07EE103A4C4B92ED2A
:10B05800005AD3ED007AD3ED013A93ED026AC9EDB7
:10B06800625AB8EEC77A34EEE54A012236EEC77A5C
:10B0780089ED614AC9ED654A89F89821C7EE055AF4
:10B088000A8D534206EE903A3E4BDFED3F4A93ED70
:10B09800005A3E4B93ED004AB7EE007AF4EEC75AD9
:10B0A80035EE045AF1EE10FA88BFF0EE475A35EE45
:10B0B800275AF8EEE66AF4EEE45AF1EE10FA07EED3
:10B0C800902AB4EEE65AB8BFF0EE645AF1EE10FAE0
:10B0D800C9ED685AB8EE677A01F18683B4EEC75AAB
:10B0E800F1EE10FA88BFB0EE475A264BDFED284A3A
:10B0F800D3ED017A254B93ED014A77EE847A25EE5C
:10B10800245A77EEA37AF4EEE76AF1EE10FA52DCED
:10B1180048E000BFC4370020D04000201C76002043
:10B128009C7600209E760020A0760020C075002026
:10B13800FC7400200400002034760020CC75002028
:10B1480004750020007500205875002054750020F3
:10B15800204100208C210020335600201876002042
:10B1680024760020A4760020D875002024410020F1
:10B1780034360020B0370020EC3E0020B4430020D5
:10B188005C3C0020503C002000000000683C00208F
:10B198006F12833AEC750020147600201C500020B2
:10B1A800E47A0020B4EEE77AF1EE10FA8CBFF0EE04
:10B1B800676AF0EE476AEC4B4A8DD3ED027A9FED51
:10B1C800EB7A534204EE103A76EE277AB8EEC44A88
:10B1D80066EE876AF4EEC47AF1EE10FA0AD407EE46
:10B1E800102AB8EE474AB4EEE74AF1EE10FA88BFE3
:10B1F800B0EE674ADE4ADFEDDD7A527824EE274A60
:10B208000AB9B1EE444A002841F0B486B7EE003AD4
:10B21800D84D2A78002A02F05986D7499FEDD76A77
:10B22800D1ED024A91ED017AD1ED037A66EEA44A96
:10B23800E5EE074AE4EE274A63EE244AF4EEC64AEE
:10B24800F1EE10FAB4BFF0EE463AF0EE643A98BF69
:10B25800B0EE646A012ACDED0A4A02F08486D1ED87
:10B26800067AD1ED052A91ED077A66EEA77AE5EE22
:10B27800227AE4EE077A23EE277AB4EEC67AF1EE64
:10B2880010FAB4EEE37A8CBFF0EE467AF0EE477A25
:10B29800F1EE10FA98BFB0EE676AB4BFF0EE637AC9
:10B2A800F0EE477A022A8DED0B7A00F0DE8091ED00
:10B2B8000A7AD1ED092AD1ED0B3A26EE877AA5EE66
:10B2C800227AA4EE237A23EE077AB4EEC67AF1EE58
:10B2D80010FAB4EEE77A8CBFF0EE463AF0EE473A51
:10B2E800F1EE10FA98BFB0EE636AA8BFF0EE477AA5
:10B2F800032A8DED0C7A00F0B88091ED0E7AD1ED2D
:10B308000D2AD1ED0F3A26EE877AA5EE227AA4EE21
:10B31800237A23EE077AB4EEC67AF1EE10FAB4EE89
:10B32800E77A8CBFF0EE463AF0EE473AF1EE10FAC3
:10B3380098BFB0EE636AA8BFF0EE477A042A8DED95
:10B348000D7A00F09280D1ED123AD1ED112A91EDEB
:10B35800137A66EEA33AE5EE223AE4EE073A63EE94
:10B36800233AF4EEC63AF1EE10FAF4EEE73A8CBF5F
:10B37800B0EE467AB0EE637AF1EE10FA98BFB0EE0E
:10B38800476AA8BFF0EE637A052ACDED0E3A6CD075
:10B39800D1ED163AD1ED152A91ED177A66EEA33A5A
:10B3A800E5EE223AE4EE073A63EE233AF4EEC63AC3
:10B3B800F1EE10FAF4EEE73A8CBFB0EE467AB0EE52
:10B3C800637AF1EE10FA98BFB0EE476AA8BFF0EEC4
:10B3D800637A062ACDED0F3A47D0D1ED1A3AD1ED6E
:10B3E800192A91ED1B7A66EEA33AE5EE223AE4EECD
:10B3F800073A63EE233AF4EEC63AF1EE10FAF4EEA9
:10B40800E73A8CBFB0EE467AB0EE637AF1EE10FA06
:10B4180098BFB0EE476AA8BFF0EE637A072ACDED71
:10B42800103A22D091ED1E7AD1ED1D2AD1ED1F3AA6
:10B4380026EE877AA5EE227AA3EE847A27EE037A9F
:10B44800B4EEC67AF1EE10FAB4EEE77A8CBFF0EEFD
:10B45800466AF0EE476AF1EE10FA8DED117A98BF60
:10B46800B0EE666AA8BFF0EE477A77EEC67AF7EED6
:10B47800006AF4EEE67AF1EE10FAC9ED4C7A43F37D
:10B48800B08686EEA77A022ADDED0B7A64EE874A4B
:10B4980067EE877ACDED0A4ACDED0B7A2DD0DDED3A
:10B4A8000C7A67EE877A032ACDED0C7A25D0DDED8C
:10B4B8000D7A67EE877A042ACDED0D7A1DD0DDED81
:10B4C8000E7A67EE877A052ACDED0E7A15D0DDED76
:10B4D8000F7A67EE877A062ACDED0F7A0DD0DDED6B
:10B4E800107A67EE877A072ACDED107A05D0DDED60
:10B4F800117A27EE877A8DED117A2149096811F0C2
:10B50800805C01F0A982F6EE005AC9ED685A002A5B
:10B5180002F0D6841B4B99ED656A1B491B4E1C78BB
:10B528001B4F99F9983199ED645AB6F90660C878B5
:10B53800DBF80010D7ED004A0396BDEEC66A07EEA9
:10B54800103AB8F81A60134B079616EE107ABDEE4B
:10B55800C56A04F0010E01F4805601F0100401F4EC
:10B56800800108911B7817E0503C00206F12833A45
:10B57800F83C0020AD3D00202443002000000000DE
:10B58800A437002033560020F048002024780020FB
:10B598002043002040520020D9ED616AD9ED627A3B
:10B5A800B8EEC77A16EE101A002840F0FB87002C78
:10B5B80041F0AF83D44C9DED0A5A94ED006AD3480C
:10B5C80025EE866AA5EE076AB0EE675AA6EE265AF9
:10B5D800BDEEC56A16EE10CA16EE106ABC45A8BFC5
:10B5E8003E466145C8BF0E4606EE106AB8EEC66A0A
:10B5F800012A80ED006A00F0DC8094ED046A9DED7C
:10B608000B5A25EE866AA5EE076AB0EE675AA6EED3
:10B61800265ABDEEC56A16EE10CA16EE106ABC456B
:10B62800A8BF3E466145C8BF0E4606EE106AB8EE92
:10B63800C66A022A80ED016A00F0BB8094ED086AB0
:10B648009DED0C5A25EE866AA5EE076AB0EE675A9C
:10B65800A6EE265ABDEEC56A16EE10CA16EE106A98
:10B66800BC45A8BF3E466145C8BF0E4606EE106AF7
:10B67800B8EEC66A032A80ED026A00F09A8094ED5B
:10B688000C6A9DED0D5A25EE866AA5EE076AB0EEA6
:10B69800675AA6EE265ABDEEC56A16EE10CA16EE11
:10B6A800106ABC45A8BF3E466145C8BF0E4606EEB7
:10B6B800106AB8EEC66A042A80ED036A79D094ED60
:10B6C800106A9DED0E5A25EE866AA5EE076AB0EE61
:10B6D800675AA6EE265ABDEEC56A16EE10CA16EED1
:10B6E800106ABC45A8BF3E466145C8BF0E4606EE77
:10B6F800106AB8EEC66A052A80ED046A59D094ED3E
:10B70800146A9DED0F5A25EE866AA5EE076AB0EE1B
:10B71800675AA6EE265ABDEEC56A16EE10CA16EE90
:10B72800106ABC45A8BF3E466145C8BF0E4606EE36
:10B73800106AB8EEC66A062A80ED056A39D094ED1B
:10B74800186A9DED105A25EE866AA5EE076AB0EED6
:10B75800675AA6EE265ABDEEC56A16EE10CA16EE50
:10B76800106ABC45A8BF3E466145C8BF0E4606EEF6
:10B77800106AB8EEC66A072A80ED066A19D094EDF9
:10B788001C6A9DED115A65EE865AE7EE055AE6EEFB
:10B79800A57AFDEEE77A17EE904AA742A8BF27469A
:10B7A800A142D8BF394607EE901AF8EEE77AC0ED05
:10B7B800077ABEF1000F01F00280554A1268002A8C
:10B7C80041F00A80534A127882B1287858B14F4E16
:10B7D800514F0024E0B23B68B6EC010A984728783C
:10B7E80001348442F6DB4D4A12689047029B1A786E
:10B7F800072A01F081810025DBF80020510500F1BE
:10B80800F787474B1A68120701F10080454A1278FA
:10B81800BAB14549B8F81A20B1F90610914210DCBE
:10B82800424A1278012A01F0B784192A01F0B48437
:10B838000E2A06D0082A04D03D4C0022A260C9F87E
:10B84800402199F8AA4124B13A4B1A88960741F049
:10B85800618499F8B021002A41F0508098F81E6060
:10B86800002E00F01C86022E01F0B983032E41F051
:10B87800B28398F82010C1EB411001EB8001C90098
:10B8880089B298F81F700237FFB2002A00F05F866D
:10B89800002900F05C8628480668B1FBF6F10EB274
:10B8A800A9F8E061002F03F0648107EE906AF8EED2
:10B8B800E77AF7EE006A86EEA77A1D4C012FD9EDDC
:10B8C8007D6AD4ED007A77EEE67A67EE877AC9ED7D
:10B8D800797A3DD0D4ED017AD9ED7E6A77EEE67AB1
:10B8E800022F67EE877AC9ED7A7A31D0D4ED027AE1
:10B8F800D9ED7F6A77EEE67A032F67EE877AC9ED8E
:10B908007B7A25D01AE000BF24430020C03C0020E9
:10B91800F874002068550020345200203C52002062
:10B92800C44000202C02002024780020F83C00208D
:10B93800EC3E002020410020E03C0020D4ED037ABA
:10B94800D9ED806A77EEE67A67EE877AC9ED7C7A78
:10B95800029B1978092903F06582002E40F3A5851A
:10B968009FB399ED7D7AD9ED797A77EE877A012FB1
:10B97800C9ED7D7AC4ED007A21D099ED7E7AD9EDB2
:10B988007A7A77EE877A022FC9ED7E7AC4ED017A4A
:10B9980015D099ED7F7AD9ED7B7A77EE877A032FE8
:10B9A800C9ED7F7AC4ED027A09D0D9ED807A99ED94
:10B9B8007C7A77EE877AC9ED807AC4ED037A013F05
:10B9C800022FB8BF0227FBB20693002A069B18BFB6
:10B9D8000223CC4ADFEDCC6A1168029A887817787E
:10B9E8000A7807EE902AF8EEE77AB0EE007A67EE6A
:10B9F800A67AF4EEC77AF1EE10FA40F3F186DFED9D
:10BA0800C36A37EEC77AB0EE676AA7EE266AF0EE29
:10BA1800466A94ED007A9FEDBE6A27EE066AF0EE5C
:10BA2800C65A89ED546AC9ED575A98B107EE100AFB
:10BA3800B8EEC75A9FEDB47A66EE064A25EE075A65
:10BA4800B7EE007A37EE457A64EEA54AA4EE857A19
:10BA580026EE076A9FEDAF7A4A7926EE877A27EEB7
:10BA6800067ACAB1DFEDA86A9FEDAB6A65EEA65A01
:10BA780006EE902AF8EEE66A66EEA56AF4EEC66A65
:10BA8800F1EE10FA01F34D82F7EE005A75EEE66A10
:10BA980085EEA66A27EE067A0C2F9FEDA08ADFEDC9
:10BAA800A06A01F00780B4EEC87AF1EE10FA98BFE8
:10BAB800B0EE478AB4EEE68AF1EE10FAB8BFB0EEFF
:10BAC800668A89ED4E8A002B00F0DC80B0EE007AA1
:10BAD800F4EEC77AF1EE10FA05DD37EEC77ADFED3E
:10BAE8008B6AE7EE267A94ED017ADFED896A27EE14
:10BAF800267AF0EEC75A89ED557AC9ED585A98B1A9
:10BB080006EE900A9FED806AF8EEE66A27EE075A7D
:10BB180066EE866AB7EE006A36EE666A25EE255A44
:10BB2800A5EE266A27EE067ADFED7A6A8A7967EE4D
:10BB3800A67A67EE877AAAB107EE102AB8EEC77A16
:10BB48009FED716ADFED746A27EE257A27EE067A93
:10BB5800B4EEE67AF1EE10FA41F3E781DFED716AAF
:10BB680067EEA67A0C2F00F07E87DFED6C6A9FEDFA
:10BB78006C7AF4EEE67AF1EE10FA88BFF0EE667AA7
:10BB8800F4EEC77AF1EE10FAB8BFF0EE477A012B5F
:10BB9800C9ED4F7A76DD4B78DFED5B6A4A7A07EEBE
:10BBA800903AF8EEE77AB0EE007A67EEA67AF4EE0D
:10BBB800C77AF1EE10FA05DD37EEC77ADFED536A82
:10BBC800E7EE267A94ED027ADFED516A27EE267ABF
:10BBD800F0EEC75A89ED567AC9ED595A9AB106EE70
:10BBE800902A9FED496AF8EEE66A27EE075A66EE54
:10BBF800866AB7EE006A36EE666A25EE255AA5EE25
:10BC0800266A27EE067ADFED436ACA7967EEA67AD6
:10BC180067EE877AFAB107EE102AB8EEC77A9FED79
:10BC28003A6ADFED3D6A27EE257A27EE067AB4EE0A
:10BC3800E67AF1EE10FA01F38681B5EEC07AF1EEFC
:10BC480010FA02F16383B7EE006A36EE477AC6EE61
:10BC5800076A67EEA67A0C2F00F02487DFED2F6ABB
:10BC68009FED2F7AF4EEE67AF1EE10FA88BFF0EE47
:10BC7800667AF4EEC77AF1EE10FAB8BFF0EE477ABA
:10BC8800C9ED507A092F00F0DA8698F82140002C87
:10BC980040F08F86002289F8B02112F011FC0028AC
:10BCA80040F01384204B1B7823B9204B9B78002B42
:10BCB80041F04682049805F05BFE029B1C78072C35
:10BCC8007EF42FAFFBF730FE194B029A401B147815
:10BCD800D880FEF726BF99F86821002A3FF46AA9A0
:10BCE800144A89F868311288002A7FF45DA9124A3B
:10BCF800124B1178186881F0010105F059F8FFF727
:10BD080059B900BF284100200AD7233CD7A368416E
:10BD18006F12033B00004843A4707D3F00C0F94404
:10BD280000C0F9C40000C84270460020FA7700201D
:10BD3800D03D00209C7600209E760020A076002032
:10BD4800AC4A1178D9F81861AB4B9FEDAC7AF50085
:10BD58005A1982ED007A002978D0A948B0EE476ACE
:10BD6800F0EE476A0022F0EC017A013267EEA77A1A
:10BD780005EE902AB4EEE77AF1EE10FAF8EEE55AFD
:10BD8800B8BFB0EE677A8A4276EEA76AA7EEA56AD0
:10BD9800E9D1F5EEC06A5A19F1EE10FA82ED007A8F
:10BDA80054DDC6EE265A974A97490988F7EE007A75
:10BDB80075EEE75AD2ED007A65EEA77AFDEEE77ADE
:10BDC80017EE902A812A42F309828A42A8BF0A46BE
:10BDD80007EE902AF8EEE77A8C4AA81902EB80025F
:10BDE80092ED057AD2ED003A92ED066A92ED014A9B
:10BDF800D2ED046AD2ED034A92ED025AA3EEA77A75
:10BE0800A4EE276A66EEC76AA7EE646ABDEEC77A33
:10BE1800E5EE276A17EE100A812882ED056AC2ED61
:10BE2800066A42F3D8818142A8BF014607EE901AFC
:10BE3800F8EEE77AFCEEE77ACDED057ABDF8142046
:10BE480059198A8016B9132F03F0B381152F41F0C1
:10BE580033831D446E4BAA8823F81620D9F8144161
:10BE68006C4A013482FB04321119E217C2EBA102B9
:10BE7800C2EBC202A41AC9F814416748D9F81C21B8
:10BE8800049B664C01682478C9F81C319A1A11443D
:10BE98000160002C40F0D28007EE902A604DDFF858
:10BEA8009881604EB8EEE78A05F5F07405F51377CA
:10BEB800F5EC017A9AED070ADAF80832F8EEE77A33
:10BEC800204627EE800A9847A4F1E000DAF82831E6
:10BED8009847A4F17000DAF898319847D5F8EC0043
:10BEE800DAF8AC309847D6ED007AA8EC010AE0EE13
:10BEF800087A2434A742E6EC017AD9D1029B1C784F
:10BF0800072C7EF407AEFBF70FFD029A404B14781E
:10BF1800049A801A1880FEF7FDBD99ED577AB1F999
:10BF28000000D9ED586AB1F902E03F4AF4EEC76A59
:10BF380080EAE0738EEAEE71A3EBE073F1EE10FA9B
:10BF4800A1EBEE71B8BFF0EE476A8B42B8BF0B4663
:10BF580007EE103A1378B8EEC77A27EE097A002B65
:10BF680000F05781314B93ED005AB5EEC05AF1EE0F
:10BF780010FA40F36D852E4BD3ED004AF5EEC04A1A
:10BF8800F1EE10FA40F3648534EEC77A66EECA5AC9
:10BF980087EE246AC5EE856AB7EE007AB4EEC76A02
:10BFA800F1EE10FA88BFB0EE476AB5EEC06AF1EE5E
:10BFB80010FA76EE876AB8BFB0EE4C6A66EE266A6B
:10BFC800F4EEC76AF1EE10FA88BFF0EE476AF5EEB4
:10BFD800C06AF1EE10FAB8BFF0EE4C6A154B93ED5B
:10BFE800007A67EE877AA7EEA68AFEF750BE01228E
:10BFF800FEF7A8BD9E380020943B002000000000FA
:10C008001C200020A03800209C380020BC3A0020CA
:10C01800D03D002093244992E44200209438002027
:10C02800AC4D0020E8420020F8750020F47500208F
:10C03800FC750020F07500201050002007EE902AB3
:10C048009E4B9F4C9F49A04FCDF81490F8EEE78A7D
:10C05800039304F5B875984600268946029BDAEDE5
:10C06800077A1B78172B6DD094ED007AB8EEC78A43
:10C07800082B28EE278A07D1B0EE480A069328F045
:10C0880063FF069BA8F80000DBF8002092000BD5A0
:10C09800002E03F08283B0EE480ADAF8083205F180
:10C0A80070009847B0EE408AB0EE480ADAF82831B6
:10C0B800A5F170009847DAF8983128469847029B0E
:10C0C8001B78032BB0EE408A37D0D4F8F000DAF8AA
:10C0D800AC30B0EE480A9847D7ED007AA9EC010ACF
:10C0E800E0EE287A0136032E05F1240508F102084E
:10C0F80004F10404E7EC017AB0D1029BDDF8149056
:10C108001C78FDE6714B724A234493ED007AD2ED18
:10C11800007A704B67EE277AF7EE006AF4EEE67A5B
:10C12800F1EE10FA93ED007A88BFF0EE667A67EECA
:10C13800877A27EE888AFEF7F9BE28F005FFA8F867
:10C148000000C2E794ED007A0AEB4602B8EEC78A0F
:10C15800128FA8F8002028EE278A95E75E4BDFF8B3
:10C16800B0811A78D4075CBFB8F81820A9F88C21D8
:10C178005A4A5B4C1288D4ED037A07EE102AB8EEBF
:10C18800C77AF4EEC77AF1EE10FA41F24786554CB9
:10C19800238807EE103AB8EEC77AF4EEC77AF1EEC4
:10C1A80010FAC1F20580504A504C92ED006AD4ED65
:10C1B800006A99F99821C9ED646A76EE665A012AEF
:10C1C800C9ED626AC9ED615A89ED656A01F0E884D2
:10C1D800049BC9F89C31002437EEC77AFCEEE77A55
:10C1E800434D89ED687A17EE902AA9F88C2101222F
:10C1F80095ED005A89F898213E4A944241F23E86CC
:10C208003D4BD3ED007AD3ED013A93ED026AFEF788
:10C2180035BF3A4B93ED006AB4EEEA6AF1EE10FAD4
:10C2280040F17387F7EE005A75EEC65A3BEEC77AAF
:10C2380065EE8B5A324BA7EE256A93ED007A26EE0F
:10C24800076AB5EEC06AF1EE10FA40F20184CAEE50
:10C25800065AB7EE007AB0EE476AA6EEE56AF0EE47
:10C26800466AADE6274AD2ED007AB0EEC87AB4EE57
:10C27800E77AF1EE10FA7EF79DAE234AD2ED007A06
:10C28800B0EEED7AB4EEE77AF1EE10FA7EF792AE00
:10C298001E4AD8ED007A92ED007AF0EEE77AF4EED5
:10C2A800C77AF1EE10FA7EF585AE01220499C9F835
:10C2B8006C1189F86821FEF760BE00BFD03D0020F0
:10C2C800AC4D002010500020E842002078210020CA
:10C2D800E8750020E475002033560020B84300209C
:10C2E800EC3E0020BA430020B0370020A4430020D1
:10C2F800C04300208FD003005C3C00200076002063
:10C30800F475002028760020247600202C76002062
:10C31800E47A0020934C9448944B9549059326461B
:10C328001B68029003944F780478B6F906004FF41E
:10C338007A71B1FBF3F3C3EB431603EB8603DE001C
:10C34800B6B2B54201F04E87DAF87CE0BAF9382087
:10C35800DAF860300EF1010107EE902A1344012942
:10C36800CAF87C10CAF86030F8EEE77A01F047871F
:10C37800DAED1B5ADAED1D6A07EE101A37EEE56A98
:10C38800B8EEC75A012D86EE057A37EE257A77EE94
:10C39800C77A8AED1C7AE7EE866A8AED1B7AF0EE98
:10C3A800667ACAED1E6ACAED1D6A02F08883DAF859
:10C3B80090E0BAF93A20DAF864300EF1010107EE9C
:10C3C800902A13440129CAF89010CAF86430F8EE8C
:10C3D800E77A01F02F87DAED205ADAED226A07EEC4
:10C3E800101A37EEE56AB8EEC75A012D86EE057ABF
:10C3F80037EE257A77EEC77A8AED217AE7EE866AF4
:10C408008AED207AF0EE667ACAED236ACAED226ACE
:10C4180002F07D83DAF8A4E0BAF93C20DAF8683053
:10C428000EF1010107EE902A13440129CAF8A4105D
:10C43800CAF86830F8EEE77A01F01787DAED255A7E
:10C44800DAED276A07EE101A37EEE56AB8EEC75A32
:10C45800012D86EE057A37EE257A77EEC77A8AEDD2
:10C46800267AE6EE276A8AED257AF0EE667ACAED34
:10C47800286ACAED276A02F01583039BDFF8189132
:10C48800D880BAF8A820029B013A1C78AAF8A820FC
:10C49800059900224A608A60CA60FEF738BBA9F88D
:10C4A800E061002A3FF4F9AB324C0223FFF791BA5E
:10C4B800314B324A196812882A4BC96919805A8047
:10C4C80013B0BDEC0E8BBDE8F08F2D4C11F0B4FE0F
:10C4D8006378022B00F05086032B7FF4E3AB41F224
:10C4E800B813E35C002B41F0568341F2A403E35CEC
:10C4F800002B41F04B8341F2E803E35C002B41F051
:10C50800408341F22C13E35C002B3FF4CBAB1D4876
:10C5180014F0E2FAFFF7C6BB1B4B1C4D1A7812F059
:10C52800010F2A7840F02483002A00F01D8592002C
:10C5380017491848DFF864B0DFF8648028F030FB4A
:10C54800FFF73BB9084B0293DFF84C9095E4B9F834
:10C55800E061013E36B2002EA9F8E061A1DD054C8C
:10C56800FFF7FEB9D03D0020CC3D00200C50002044
:10C57800F84F0020EC3E0020407A0020182D0020C3
:10C58800145700204068002033560020AD3D00209D
:10C598001C2D0020C03C00201C2000201C50002026
:10C5A800E47A0020002C01F0A781BEF1000F42F0D0
:10C5B800EF82C44C002B42F0278194ED006A9DED78
:10C5C8000A5AC14825EE866AFDEEE44AA5EE076AD6
:10C5D800B0EE675AA6EE265A14EE901ABDEEC56A5A
:10C5E80016EE10EA16EE106ABE45A8BF3E46714523
:10C5F800C8BF0E4606EE106AB8EEC66A012A80ED7C
:10C60800006A00F0DF8094ED046A9DED0B5A25EE78
:10C61800866AA5EE076AB0EE675AA6EE265ABDEE00
:10C62800C56A16EE10EA16EE106ABE45A8BF3E4669
:10C638008E45B8BF0E4606EE106AB8EEC66A022AE4
:10C6480080ED016A00F0BE8094ED086A9DED0C5AF9
:10C6580025EE866AA5EE076AB0EE675AA6EE265A58
:10C66800BDEEC56A16EE10EA16EE106ABE45A8BF02
:10C678003E468E45B8BF0E4606EE106AB8EEC66A4C
:10C68800032A80ED026A00F09D8094ED0C6A9DED0E
:10C698000D5A25EE866AA5EE076AB0EE675AA6EE31
:10C6A800265ABDEEC56A16EE10EA16EE106ABE45A9
:10C6B800A8BF3E468E45B8BF0E4606EE106AB8EED5
:10C6C800C66A042A80ED036A7CD094ED106A9DED59
:10C6D8000E5A25EE866AA5EE076AB0EE675AA6EEF0
:10C6E800265ABDEEC56A16EE10EA16EE106ABE4569
:10C6F800A8BF3E468E45B8BF0E4606EE106AB8EE95
:10C70800C66A052A80ED046A5CD094ED146A9DED32
:10C718000F5A25EE866AA5EE076AB0EE675AA6EEAE
:10C72800265ABDEEC56A16EE10EA16EE106ABE4528
:10C73800A8BF3E468E45B8BF0E4606EE106AB8EE54
:10C74800C66A062A80ED056A3CD094ED186A9DED0C
:10C75800105A25EE866AA5EE076AB0EE675AA6EE6D
:10C76800265ABDEEC56A16EE10EA16EE106ABE45E8
:10C77800A8BF3E468E45B8BF0E4606EE106AB8EE14
:10C78800C66A072A80ED066A1CD094ED1C6A9DEDE6
:10C79800115A65EE865AE7EE055AE6EEA57AFDEEE1
:10C7A800E77A17EE904AA742A8BF2746A142D8BF0A
:10C7B800394607EE901AF8EEE77AC0ED077A002AB4
:10C7C8003EF4FBAF920041493F4828F0E9F9404A5E
:10C7D8001268002A3EF4F6AF1FF018F8FEF7F2BF11
:10C7E800F0EE676AFFF715B9B0EE665AFEF77DBC42
:10C7F800DAF80820002A3FF404A83649A1F14C00D1
:10C808009047354B1A6812077FF500A8334CD4EDD2
:10C81800027AB2EE0E7AF0EEE76AF4EEC76AF1EE4B
:10C8280010FA41D52E4B1A8853073DD52D4A2E486C
:10C83800B2F90420B9F8A61180FB0230D217C2EB76
:10C84800A002521A92B210B210F1B30FBCBF02F597
:10C85800B47210B2B328C4BFA0F5B47210B2234AA0
:10C86800234912790978002A4FF6FF7218BF01226E
:10C878000F077EF5CBAF1F4B196810FB02F2087E3D
:10C888001D4992B210FB02F281FB02311144D2170A
:10C89800C2EB211207EE102AB8EEC77A77EEC77AF4
:10C8A800C4ED027AFEF7B2BF0E4A0F49B2F904206E
:10C8B80081FB0231D217C2EBA102A9F8A621FEF72B
:10C8C800A5BF00BF24430020C03C00201C2D002031
:10C8D800F8740020CC4D0020C4400020EC3E00201D
:10C8E80020410020D040002067666666BC370020E3
:10C8F800F877002024410020898888889148924947
:10C90800D0F8EC00096844F62064A042A8BF20468D
:10C91800B0F57A7FB8BF4FF47A7080B211F0100F7B
:10C92800A9F8B201DBF8001000F03D84CB0441F116
:10C93800CC85864B1F687E8E7608854C854BD9F84A
:10C94800B411D4ED037AA3FB00308409642090FB72
:10C95800F4F01428BDEEE77A09EB410EA8BF1420C5
:10C9680001318842C9F8B41117EE10CADCBF0021A2
:10C97800C9F8B41109EB4101AEF8B8C1B1F9B83141
:10C9880007EE103AB8EEC77A77EEC77AFDEEE77A87
:10C99800CDED037ABDF90C3083EAE371A1EBE371C5
:10C9A800B14201F3ED866C4B4FF07E511960FEF7F2
:10C9B80055BF1E216448F5F797FE00283FF46AA981
:10C9C800664B1A8852063FF565A999F80422A242D7
:10C9D80042F04582604BD9ED827AD3ED016A99ED38
:10C9E800505ADFED5F5A9FED5F6A27EEC57A67EE12
:10C9F800887AA6EE887AE5EE267AB4EEE57AF1EE44
:10CA080010FA88BFB0EE657AB4EEC67AF1EE10FA85
:10CA1800F4EEE57AB8BFB0EE467AF1EE10FA88BFC8
:10CA2800F0EE657AF4EEC67AF1EE10FAB8BFF0EEE1
:10CA3800467A89ED4E7AC9ED507AFFF72BB9FDEEAB
:10CA4800C87A494917EE902A8E80CA80FFF71DB927
:10CA5800DFED466AFFF7C2BADBF8001048023EF580
:10CA680052ADFEF754BD9FED3E7ADFED3E6A3E487B
:10CA7800F4EEC77AF1EE10FA98BFB0EE677AFDEEE1
:10CA8800E77AB4EEE67AF1EE10FA17EE902AB8BF1C
:10CA9800B0EE667A012B89ED4F7A42803FF77BA88A
:10CAA800FFF7F3B8BDEEE77A2F4A17EE101A918018
:10CAB800FFF7D4B8B4EEC87AF1EE10FA98BFB0EE2A
:10CAC800478ABDEEC77AB4EEE68ADFF89CC0F1EE7D
:10CAD80010FA17EE102AB8BFB0EE668A89ED4E8AB2
:10CAE800ACF80020002B7EF4F1AFFFF7CEB8002B96
:10CAF8003EF460AAFEF73DBAFAF716FF029B1A4900
:10CB08001A78059B072AA0EB030088807EF473AE91
:10CB1800FAF70AFF0546FEF76FBEFAF705FF029A15
:10CB280007991278104B0393401A012A588000F095
:10CB38000E83072A7EF466AAFAF7F6FE0590FEF73A
:10CB480063BA00BF20030020A4370020244100203E
:10CB5800EC3E0020D34D621004000020204100204C
:10CB680000C0F94400C0F9C4D03D00200000000016
:10CB7800002A00F0F981D9ED583A99ED576AD9EDB4
:10CB8800627AF34999ED617AD1ED005A99ED554AE7
:10CB9800D9ED544AEF4CF048F4EEC63AF3EE046A85
:10CBA800F1EE10FA37EEA65A00F1808394ED026A8E
:10CBB80026EE446AF0EE674AE6EE074AF4EEC54A06
:10CBC80034EEE66AF1EE10FA48BFB0EE656A012A63
:10CBD80080ED006A00F0C88194ED066A26EE446A8A
:10CBE800F0EE674AE6EE074AF4EEC54A34EEE66A26
:10CBF800F1EE10FA48BFB0EE656A022A80ED016ACC
:10CC080000F0B28194ED0A6A26EE446AF0EE674AB3
:10CC1800E6EE074AF4EEC54A34EEE66AF1EE10FA9B
:10CC280048BFB0EE656A032A80ED026A00F09C8175
:10CC380094ED0E6A26EE446AF0EE674AE6EE074A7D
:10CC4800F4EEC54A34EEE66AF1EE10FA48BFB0EEEB
:10CC5800656A042A80ED036A00F0868194ED126A01
:10CC680026EE446AF0EE674AE6EE074AF4EEC54A55
:10CC780034EEE66AF1EE10FA48BFB0EE656A052AAE
:10CC880080ED046A00F0708194ED166A26EE446A1D
:10CC9800F0EE674AE6EE074AF4EEC54A74EEE66A35
:10CCA800F1EE10FA48BFF0EE656A062AC0ED056A93
:10CCB80000F05A81D4ED1A6A66EEC46AF0EE674A4B
:10CCC800E6EE874AB3EE046AF4EEC54A74EEC66A25
:10CCD800F1EE10FA48BFF0EE656A072AC0ED066A61
:10CCE80000F04281D4ED1E6ADFF874B2DFF8748276
:10CCF80026EEC44AE4EE077AF4EEC57A77EEC67AF1
:10CD0800F1EE10FA48BFF0EE657AC0ED077AFEF74B
:10CD180054BD904C9DED0A5A94ED006ABEF1000F87
:10CD280041F0568125EE866A8B48A5EE076AB0EE7B
:10CD3800675AA6EE265ABDEEC56A16EE10EA16EE3A
:10CD4800106ABE45A8BF3E467145C8BF0E4606EEEE
:10CD5800106AB8EEC66A012A80ED006A3FF432AD67
:10CD680094ED046A9DED0B5A25EE866AA5EE076AD6
:10CD7800B0EE675AA6EE265ABDEEC56A16EE10EA60
:10CD880016EE106ABE45A8BF3E467145C8BF0E469E
:10CD980006EE106AB8EEC66A022A80ED016A3FF410
:10CDA80011AD94ED086A9DED0C5A25EE866AA5EE44
:10CDB800076AB0EE675AA6EE265ABDEEC56A16EEA9
:10CDC80010EA16EE106ABE45A8BF3E467145C8BFB8
:10CDD8000E4606EE106AB8EEC66A032A80ED026AAD
:10CDE8003FF4F0AC94ED0C6A9DED0D5A25EE866A81
:10CDF800A5EE076AB0EE675AA6EE265ABDEEC56ADA
:10CE080016EE10EA16EE106ABE45A8BF3E467145FA
:10CE1800C8BF0E4606EE106AB8EEC66A042A80ED50
:10CE2800036A3FF4CFAC94ED106A9DED0E5A25EEDF
:10CE3800866AA5EE076AB0EE675AA6EE265ABDEED8
:10CE4800C56A16EE10EA16EE106ABE45A8BF3E4641
:10CE58007145C8BF0E4606EE106AB8EEC66A052AC6
:10CE680080ED046A3FF4AEAC94ED146A9DED0F5A60
:10CE780025EE866AA5EE076AB0EE675AA6EE265A30
:10CE8800BDEEC56A16EE10EA16EE106ABE45A8BFDA
:10CE98003E467145C8BF0E4606EE106AB8EEC66A31
:10CEA800062A80ED056A3FF48DAC94ED186A9DED75
:10CEB800105A25EE866AA5EE076AB0EE675AA6EE06
:10CEC800265ABDEEC56A16EE10EA16EE106ABE4581
:10CED800A8BF3E467145C8BF0E4606EE106AB8EEBA
:10CEE800C66A072A80ED066A3FF46CAC94ED1C6AAA
:10CEF8009DED115A65EE865AE7EE055AE6EEA57ADB
:10CF0800FDEEE77A17EE904AA742A8BF2746A1424E
:10CF1800C8BF0F4607EE907AF8EEE77AC0ED077AB9
:10CF28004DE49FED0E6AFEF7B5BDB5EEC07AF1EEA1
:10CF380010FA01F1E781B7EE006A36EE477AC6EEDD
:10CF4800076AFEF70DBEDFED056AFEF782BE00BF79
:10CF58002043002024430020C03C00200000C84299
:10CF68001C500020E47A0020DFF838B3DFF838835B
:10CF7800FEF723BCB5494A79002A3EF447A9B44ACA
:10CF88001278002A3EF442A90B78B249DFEDB24A82
:10CF980007EE903A0B88B8EE677A07EE902A06EE0D
:10CFA800103AF8EEE77AB8EE466A67EE277AB7EEF7
:10CFB800007A87EE863AB4EEE43AF1EE10FA88BFCA
:10CFC800B0EE643AB4EEC73AF1EE10FAB8BFB0EE7C
:10CFD800473AFEF71DB9A1494988FEF752BCB9F88E
:10CFE800B21101F57A7189B2FEF74BBC9C490391E5
:10CFF80007EE102A08461978B0F904009AED070AD6
:10D00800B9F81051B8EEC77AF7EE006A0022132972
:10D0180086EE879AC9F80C2101F08C81914A9249D1
:10D0280001EB85060024C9F80041C9F8044167EE00
:10D03800897A92ED001AD2ED053A92ED122A92ED14
:10D04800173AD2ED091AD2ED0E4A92ED016A92ED25
:10D05800064A92ED0A7AD2ED0F5AD2ED132AD2ED92
:10D06800186A92ED045AD2ED030A69EE288A29EE6D
:10D07800088AE1EE273AA2EE283AE1EE884AA6EEBF
:10D08800274AE7EE085A92ED167A92ED0D6A92ED6C
:10D09800021AD2ED0C1AC6ED003AE2EEA86A25EEA5
:10D0A800635A27EE437A92ED0B2AD2ED152AC6ED84
:10D0B800204AA0EEE34A26EE646AD2ED143A82EDE5
:10D0C800054AA1EE275AF0EE477AE1EEE45AA2EEBD
:10D0D800086AE2EEC36AE3EEA87A82ED065AC2ED68
:10D0E8000E5A82ED0F6A86ED403AC2ED176AC2ED1C
:10D0F800187AC9F80841039B6A1C02F01F0298803D
:10D10800A9F81021029BFDF7E9BC584B93ED006A82
:10D11800FFF797B8564A9FED577AD2ED087AF4EEA2
:10D12800C77AF1EE10FA00F2D0849FED537A534C8F
:10D13800D4ED037A77EE877AC4ED037AFEF789BBDC
:10D1480004980DF02FFDFEF7B5BD454B0393FAF794
:10D15800EBFB4B49D9F87C2109680590821AC9F87C
:10D168007C010398511A8280C180FDF74DBFFAF700
:10D17800DBFB0790FDF7EDBCA3784FF0010A072B06
:10D188003EF690ADDFE813F00F06270624050406E7
:10D19800A1058A05940530053A4A927B002A3EF497
:10D1A8004BABFEF74EBBCC003FF5C0ABFEF756BB12
:10D1B800B9F88C41944240F2D38499F8A441002CE8
:10D1C80040F0A786304A314D92ED007AD5ED007ACD
:10D1D80099F99821C9ED647A77EE676A012AC9ED51
:10D1E800627AC9ED616A89ED657A01F0F487049B7A
:10D1F800C9F89C31264A9FED207A92ED005A89EDB4
:10D20800687A012289F89821FEF7F6BF214B1B881E
:10D21800002B40F0CB84204A204B1178186803F08B
:10D22800C7FDD9F86C21049B9A1AFDF749BD1C4B20
:10D23800D8ED007A93ED007AF0EEE77AF4EEC77A4B
:10D24800F1EE10FA7DF7B6AEFDF7A6BEA8400020B5
:10D25800EA3E0020D43E0020713DAA3F2033002042
:10D26800D03D0020283B0020BC380020F475002069
:10D27800BC4200208FC2753C00000000EC3E00203C
:10D28800E03C00202C7E0020B0370020A443002082
:10D29800C04300209C7600209E760020A0760020C7
:10D2A8002C7600201C500020E47A002094ED016ABE
:10D2B80026EE646AB0EE674AA6EE074AB4EEC54A9F
:10D2C80034EE666AF1EE10FA48BFB0EE656A012ADC
:10D2D80080ED006A3FF448AE94ED056A26EE646A74
:10D2E800B0EE674AA6EE074AB4EEC54A34EE666A5F
:10D2F800F1EE10FA48BFB0EE656A022A80ED016AC5
:10D308003FF432AE94ED096A26EE646AB0EE674ADD
:10D31800A6EE074AB4EEC54A34EE666AF1EE10FA94
:10D3280048BFB0EE656A032A80ED026A3FF41CAE7E
:10D3380094ED0D6A26EE646AB0EE674AA6EE074AD7
:10D34800B4EEC54A34EE666AF1EE10FA48BFB0EEA4
:10D35800656A042A80ED036A3FF406AE94ED116A0B
:10D3680026EE646AB0EE674AA6EE074AB4EEC54AEE
:10D3780034EE666AF1EE10FA48BFB0EE656A052A27
:10D3880080ED046A3FF4F0AD94ED156A26EE646A08
:10D39800B0EE674AA6EE074AB4EEC54A74EE666A6E
:10D3A800F1EE10FA48BFF0EE656A062AC0ED056A8C
:10D3B8003FF4DAADD4ED196A66EEE46AB0EE674A76
:10D3C800A6EE874AB3EE046AB4EEC54A74EE466A1E
:10D3D800F1EE10FA48BFF0EE656A072AC0ED066A5A
:10D3E8003FF4C2ADD4ED1D6ADFF898B2DFF8988239
:10D3F80066EEE44AE4EE877AF4EEC57A77EEC67A0A
:10D40800F1EE10FAB8BFF0EE657AC0ED077AFEF7D4
:10D41800D4B9914DD9ED017A99ED006A29886A69E4
:10D4280077EEA77AF0EE006AB0EE677AA6EE267A73
:10D438004D1E09EBC501D6EE267A08391032F6EEF4
:10D44800003A27EE237A67EEA37A89ED207AC9EDB0
:10D45800217ADFF81C924E4609F1800091ED027A9C
:10D4680091ED036AD6ED036AD6ED027A52ED014AD0
:10D4780012ED025A37EE674A76EEC65A77EE277AE9
:10D48800E4EE845A013DA1F10801E5EE047A06F1C3
:10D49800080602F1080236EE267A00F10800E4EEEA
:10D4A800877AE5EE475A67EEA37A25EEA37AC0EDB0
:10D4B800007A80ED017AD1D1142F7EF4D1ACFAF73D
:10D4C80033FA039A654B801A5880D9F81441FEF74D
:10D4D800C7BCD9F81881B9F810E1614ACEF1200328
:10D4E800DBB20EEB481602EB86069A0801F06E8650
:10D4F800013215015B485C4906EB050C06F1100288
:10D5080012ED024A12ED035A12ED016A12ED047A85
:10D5180050ED024A50ED035A50ED016A50ED047A7D
:10D5280064EE244A65EE255A66EE266A67EE277A87
:10D538001032944541ED024A41ED035A41ED016A2A
:10D5480041ED047A00F1100001F11001D8D14748EB
:10D55800A5F110010E4400EB010C494413F003023D
:10D5680009D0B6EC017AFCEC017A67EE277A013A29
:10D57800E1EC017AF5D1BEF1000F40F05487142F89
:10D588007EF46EACFAF7D0F9039A344BD9F814410B
:10D59800801A5880FEF764BC2F4D3548AA68A989BF
:10D5A80026F0F8FA029B1F78142F01F07686D9F836
:10D5B80014410134C9F814412CE7D9F818412D4910
:10D5C8002D482E4BE200114414448A88196800EE55
:10D5D800102A643AC82AA8BFC822782AB8BF782275
:10D5E80007EE902AB8EEC07AF8EEE77A00EB8404EA
:10D5F80077EE670A77EE876A67EE877A20EEA67A73
:10D60800B8EE400AC7EE870A2046D4F81880E669C3
:10D61800256A94ED058A23F0C3F9029B84ED058AF7
:10D628001F78C4F81880142FE661256201F03F8640
:10D63800D9F818211249D9F81441013281FB021393
:10D64800A3EBE27808EB4803A2EB03080134C9F81E
:10D658001881C9F814413EE7A4380020D03D0020C5
:10D66800BC3800204C3A00202C2000203C3A0020F6
:10D678001C200020943B00208C4F00200C500020E0
:10D68800565555551C500020E47A0020954D2988A0
:10D698006B684FEA51084FEA88005FEAD10E09EB40
:10D6A800000209EB810400F0A18000F110010EF1E5
:10D6B800010E8D4E02EB0E1E2144103203F11007AD
:10D6C80004F1100050ED032A50ED043A16ED043A27
:10D6D80016ED032A50ED026A10ED016A16ED020AF2
:10D6E80016ED018A11ED044A11ED035A52ED044A70
:10D6F80052ED035A12ED027A52ED017A51ED020A07
:10D7080011ED011A73EE238A72EE221A46ED048A8D
:10D7180046ED031A70EE268A78EE061A46ED028A5E
:10D7280046ED011A74EE848A75EE851A42ED048A74
:10D7380042ED031A77EE208A77EE811A42ED028ACB
:10D7480042ED011A73EE633A75EE655A17ED035A06
:10D7580032EE623A74EE644A65EE631A17ED044AD3
:10D7680023EE052A64EE652AE3EE041A1032964584
:10D7780024EE843AA3EE842A06F1100607F1100776
:10D78800A5EE853A00F1100001F11001E4EE852ABA
:10D7980040ED071A00ED082A01ED073A41ED082A85
:10D7A80057ED055A17ED065A70EE666A38EE466A66
:10D7B80030EEC77A71EE677A26EE253A65EEE63ADC
:10D7C80025EE674A67EE054AE6EE053AA6EE853A83
:10D7D800A7EE254AE7EEA54A00ED063A40ED053AE0
:10D7E80001ED064A41ED054A7FF46CAF1FFA88F84F
:10D7F8001A4641463D4822F0F3FD6A6841462046F4
:10D8080022F0EEFD029B1A78142A7FF45EAE56E6EB
:10D81800DFF8E08098F800108E0801F0C085344DDC
:10D8280006F1010C4FEA4C1C05EB0C0E05F1200229
:10D83800A5F1700012ED076A52ED056A12ED037A40
:10D8480052ED017A52ED025A12ED084A52ED064A9B
:10D8580012ED045A26EE066A66EEA66A27EE077AE5
:10D8680067EEA77AA4EE046A20329645E4EEA46A2D
:10D8780000F11000A5EE057AE5EEA57AF1EEC65A9C
:10D88800B1EEE66AF1EEC76AB1EEE77A40ED085A02
:10D8980000ED076A40ED066A00ED057ACAD1ACF1E1
:10D8A80020022A4409EB061611F0030018BF0832BB
:10D8B8000FD052ED017A12ED027A67EEA77A01389D
:10D8C800E7EE077A02F10802B1EEE77AA6EC017AF0
:10D8D800EFD1142F01F0D3840134C9F81441FEF7B5
:10D8E80031BA00BFA43800202C2000201C200020C2
:10D8F8009C2000209E380020BD4C002B40F0FC8569
:10D9080094ED006A9DED0A5ABA4825EE866AFDEE46
:10D91800E44AA5EE076AB0EE675AA6EE265A14EE58
:10D92800901ABDEEC56A16EE10CA16EE106ABC450E
:10D93800A8BF3E466145C8BF0E4606EE106AB8EE5F
:10D94800C66A012A80ED006A3DF433AF94ED046A9B
:10D958009DED0B5A25EE866AA5EE076AB0EE675A6A
:10D96800A6EE265ABDEEC56A16EE10CA16EE106A65
:10D97800BC45A8BF3E468C45B8BF0E4606EE106AA9
:10D98800B8EEC66A022A80ED016A3DF412AF94ED42
:10D99800086A9DED0C5A25EE866AA5EE076AB0EE78
:10D9A800675AA6EE265ABDEEC56A16EE10CA16EEDE
:10D9B800106ABC45A8BF3E468C45B8BF0E4606EE69
:10D9C800106AB8EEC66A032A80ED026A3DF4F1AE29
:10D9D80094ED0C6A9DED0D5A25EE866AA5EE076A50
:10D9E800B0EE675AA6EE265ABDEEC56A16EE10CA04
:10D9F80016EE106ABC45A8BF3E468C45B8BF0E4619
:10DA080006EE106AB8EEC66A042A80ED036A3DF491
:10DA1800D0AE94ED106A9DED0E5A25EE866AA5EEFD
:10DA2800076AB0EE675AA6EE265ABDEEC56A16EE2C
:10DA380010CA16EE106ABC45A8BF3E468C45B8BF52
:10DA48000E4606EE106AB8EEC66A052A80ED046A2C
:10DA58003DF4AFAE94ED146A9DED0F5A25EE866A3B
:10DA6800A5EE076AB0EE675AA6EE265ABDEEC56A5D
:10DA780016EE10CA16EE106ABC45A8BF3E468C4585
:10DA8800B8BF0E4606EE106AB8EEC66A062A80EDE2
:10DA9800056A3DF48EAE94ED186A9DED105A25EE98
:10DAA800866AA5EE076AB0EE675AA6EE265ABDEE5C
:10DAB800C56A16EE10CA16EE106ABC45A8BF3E46E7
:10DAC8008C45B8BF0E46FDF752BEF0EEE76AB7EEDA
:10DAD800005A35EE665A9FED484ADFED485A9FEDE9
:10DAE800486A9FED487A99ED6B0AF1EEC54AE6EE71
:10DAF800845AF5EEC07AA6EEA56AF1EE10FAA6EE03
:10DB0800867A48BFDFED407A27EE247A48BF37EEA1
:10DB1800C77A27EE000A27F017FAB0F5617F00F3FD
:10DB28004A8607EE900AF8EEE76ADFED387A66EE85
:10DB3800A76A07EE904ABDEEE67AF8EEE77A17EEA6
:10DB4800102A2032402A41F28C849FED310A27F0B6
:10DB5800FBF900B207EE900AB8EEE77AFFF7E7BAEA
:10DB68002C4A02F1500403E00432944200F0D181BF
:10DB78001378262BF8D19578D3789D42F4D2FFF705
:10DB88001CBB254812F0A8FFFEF7BBBC234812F0C7
:10DB9800A3FFFEF7B0BC224812F09EFFFEF7A5BC1B
:10DBA800D9F89C41049B1C1BFEF716BB1D494B6909
:10DBB800002B3DF485A81C481C4B008893FBF0F013
:10DBC8000B684FF0010E186081F811E0FDF778B886
:10DBD800174B00930320A0703023052215491648DF
:10DBE80013F028FCFEF75EB803236370FEF75AB8FB
:10DBF80024430020C03C0020306E99BC2716983D75
:10DC0800843459BEA40DC93FDB0F4940D06D393A61
:10DC18000000000084340020FC670020B867002062
:10DC2800CC680020A4760020BC76002020A1070044
:10DC380045000208848B03088468002023690622B3
:10DC4800652BA27034D92278032A14BF6FF0FF0223
:10DC58006FF07F02A3F1650303EA020303F10103F6
:10DC680014BF4FF4807280229A42236120D23A680E
:10DC7800E768023203EB0708904581F00285C34A42
:10DC88006760D16FC4F80880490203FB01F30521DE
:10DC9800176042F81C3C42F8183CA170A268BC49C5
:10DCA80001200FF02FFF012841F0E1840623A37023
:10DCB8000021B8480FF0EEFE012841F0D884A3787F
:10DCC8000133DBB2A370FFF75ABA2278237DB24F33
:10DCD800DFF8BC92032A14BF4FF480784FF0800815
:10DCE800002B41D0012BFBD1AC4B62681968386816
:10DCF80000234FEA412E4FF0FF31B1FBFEF112EB4A
:10DD0800010B43F1000C0021614500F1020008BF3E
:10DD1800584538BF83465A46A149022010F024F8D6
:10DD2800032801F2668201A353F820F0ADBC000875
:10DD380045DD0008ADBC000845DD00086268A36841
:10DD48002669991AB14284BFE260216103283FF431
:10DD580075AF0133B3FBF8F208FB12320AB1434442
:10DD68009B1A0022636022753A68494602320020F5
:10DD78000FF0FAFF032801F23C8201A353F820F0C8
:10DD8800ADBC000819DE0008ADBC000845DC000881
:10DD980041F27013E35C002B3DF484AF7D4812F030
:10DDA8009BFEFDF77FBF00230AAE314618460922C5
:10DDB8000FF030FD01287DF475AF0A9B93F8FE2122
:10DDC800552A01F0198241F2B41202210123A1540B
:10DDD8006370FDF767BF0AAE41F2FC173146E059A0
:10DDE800002309220FF016FD01287DF45BAF002304
:10DDF8000A9A2370B2F80B30B3F5007F01F0D48390
:10DE080041F2B41203210123A1546370FDF74ABF04
:10DE1800636884F814A00133A36065E7614A624C23
:10DE2800D2ED006A614A94ED006A1278C9ED646A1D
:10DE380089ED656A002A00F0F18276EE665A99F952
:10DE48009821C9ED615A0132C9ED626A00F09486E1
:10DE5800049BC9F89C31002437EE677AFCEEE77A18
:10DE6800534D89ED687A17EE902AA9F88C21FF2284
:10DE780095ED005A89F89821FEF7BEB9DFED4D7A85
:10DE88004D4B99ED687AC3ED007AC3ED017AC3ED85
:10DE9800027A4A4BB0EE676AF0EE673A1968FDF706
:10DEA800EDB8F9F741FD029B03901F78142F05BFC9
:10DEB800434BD9F81441D9F814411C80FCF716BE1D
:10DEC800404B1C7804F0010EFDF773BC3E49DFEDB2
:10DED8003F7A0968C9ED4C7A11F0805C40F05E84A5
:10DEE800DBF8001011F4800C00F0F5824FF0000C04
:10DEF800B6EE007A67EE877AF4EEE57AF1EE10FA7C
:10DF0800C8BFF0EE675A40F34984C9ED685AFDF777
:10DF1800FEBA244A244CD2ED007A244A94ED007AC1
:10DF28001278C9ED647A89ED657A002A00F02284B6
:10DF380077EE676A99F99821C9ED616A0132C9EDEE
:10DF4800627A00F06987049BC9F89C3100249FED30
:10DF5800197A174D89ED687AFF2295ED005A89F8EC
:10DF68009821FEF749B973EEC67AB7EE007AF4EE57
:10DF7800C77AF1EE10FAC9ED4C7A41F3328184EE9A
:10DF8800A77A8DED0A7AFDF7B8BA00BFA868002015
:10DF980018570020846800201C690020246900208C
:10DFA8001C57002034360020A8430020405200208F
:10DFB800BC430020000000005C3C002024410020FD
:10DFC800D03D002033560020A437002000000080F8
:10DFD800002E00F0D58725EE866ACE48A5EE076AA2
:10DFE800B0EE675AA6EE265ABDEEC56A16EE10EADE
:10DFF80016EE106ABE45A8BF3E467145C8BF0E461C
:10E0080006EE106AB8EEC66A012A80ED006A3DF491
:10E01800D4AB94ED046A9DED0B5A25EE866AA5EE05
:10E02800076AB0EE675AA6EE265ABDEEC56A16EE26
:10E0380010EA16EE106ABE45A8BF3E467145C8BF35
:10E048000E4606EE106AB8EEC66A022A80ED016A2C
:10E058003DF4B3AB94ED086A9DED0C5A25EE866A43
:10E06800A5EE076AB0EE675AA6EE265ABDEEC56A57
:10E0780016EE10EA16EE106ABE45A8BF3E46714578
:10E08800C8BF0E4606EE106AB8EEC66A032A80EDCF
:10E09800026A3DF492AB94ED0C6A9DED0D5A25EEA3
:10E0A800866AA5EE076AB0EE675AA6EE265ABDEE56
:10E0B800C56A16EE10EA16EE106ABE45A8BF3E46BF
:10E0C8007145C8BF0E4606EE106AB8EEC66A042A45
:10E0D80080ED036A3DF471AB94ED106A9DED0E5A24
:10E0E80025EE866AA5EE076AB0EE675AA6EE265AAE
:10E0F800BDEEC56A16EE10EA16EE106ABE45A8BF58
:10E108003E467145C8BF0E4606EE106AB8EEC66AAE
:10E11800052A80ED046A3DF450AB94ED146A9DED38
:10E128000F5A25EE866AA5EE076AB0EE675AA6EE84
:10E13800265ABDEEC56A16EE10EA16EE106ABE45FE
:10E14800A8BF3E467145C8BF0E4606EE106AB8EE37
:10E15800C66A062A80ED056A3DF42FAB94ED186A6D
:10E168009DED105A25EE866AA5EE076AB0EE675A4D
:10E17800A6EE265ABDEEC56A16EE10EA16EE106A2D
:10E18800BE45A8BF3E467145C8BF0E4606EE106A9A
:10E19800B8EEC66A072A80ED066A3DF40EAB94ED28
:10E1A8001C6A9DED115A65EE865AE5EE075AE6EEB1
:10E1B800A57AFDEEE77A17EE902A9742A8BF174690
:10E1C8009142D8BF394607EE901AF8EEE77AC0EDCB
:10E1D800077AFDF7F2BA8222FDF732BEDFED4E7AFA
:10E1E800FDF7FABDBAF93830CAF8202007EE903AA0
:10E1F8000122F8EEE77ACAF86030CAF87C200023DA
:10E20800012DCAED1C7ACAED1B7ACAF8743001F0E8
:10E218001881B5427EF4CBA8BAF93A30CAF864300E
:10E2280007EE903A00220123F8EEE77ACAF8242094
:10E23800CAF890300023012DCAED217ACAED207A60
:10E24800CAF8883001F0F980B5427EF4E3A8BAF93B
:10E258003C30CAF8683007EE903A00220123F8EE05
:10E26800E77ACAF82820CAF8A4300023012DCAED9D
:10E27800267ACAED257ACAF89C307EF4FEA89FED6E
:10E28800278A032C38D04FB107EE907AF8EEE77A58
:10E29800F4EEC87AF1EE10FA01F17E81204ADFF837
:10E2A8009090039B1168DAF86820D88099F82001CB
:10E2B80002EB560292FBF6F60022CAF828608A6240
:10E2C8000A63CA6228B1174A126832F480637EF47E
:10E2D800D8A8154A126812F4003241F05580134C40
:10E2E8001146A35C012B02F10C0200F07D8501317F
:10E2F8001829F6D1FEF7C5B8B0EE480A26F024FE74
:10E3080000B2C0E7F7EE006AFDF72ABCF7EE006A34
:10E31800FDF79FBCC03C0020000002430000000045
:10E32800407A00201C410020F42F0020BC7503080F
:10E338001C2000206D4C6E4E94ED004A94ED057A39
:10E34800D4ED014A94ED066AD4ED046A94ED035ABB
:10E35800D4ED025A67EE897A06EB8502A4EE277A95
:10E36800A4EEA76A66EEC76AA5EE476AE5EEA76A55
:10E3780020EE070A84ED056AC4ED066A82ED007A8C
:10E3880029EE088A26F0E0FD69EE288AD4ED0E5AB7
:10E39800D4ED176A94ED091AD4ED121A94ED0F5AB8
:10E3A80094ED187A94ED0A2AD4ED132A94ED0D6AA7
:10E3B800D4ED167A94ED0C3AD4ED0B3A94ED154A57
:10E3C800D4ED144AE1EE085A002206EB8501E8EE86
:10E3D800A16A00B2C9F80021A2EE085AC9F80421BE
:10E3E800C9F80821A8EEA27A26EE656A67EEE67AF1
:10E3F800A3EE655AA3EE886AA6EEC47AE8EEA47A7C
:10E4080084ED0E5AC1ED205A84ED0F6AC1ED406AC1
:10E4180084ED177AC4ED187AFEF76DBE76EEC65A0B
:10E42800F0EE466A0BE59E00314B03EBC8185FEA35
:10E438009E0300EB060C4E4401F0598001331B018A
:10E4480008EB030508F110020CF1100006F11001A9
:10E4580012ED024A12ED035A12ED016A12ED047A26
:10E4680050ED024A50ED035A50ED016A50ED047A1E
:10E4780064EE244A65EE255A66EE266A67EE277A28
:10E488001032954241ED024A41ED035A41ED016ACD
:10E4980041ED047A00F1100001F11001D8D1103BD0
:10E4A80098440CEB03001E441EF0030E3FF467A8CB
:10E4B800B8EC017AF0EC017A67EE277ABEF1010E2A
:10E4C800E6EC017AF4D1FFF75AB80A4B1F68B7F99E
:10E4D8003260FEF732BAB6EE007AF4EEC75AF1EEC1
:10E4E80010FA3FF705ADFDF712B800BF283B002032
:10E4F800BC3800202441002094ED006A9DED0A4AB2
:10E50800BA4825EE866AFDEEE43AA4EE076AB0EE54
:10E51800674AA6EE264A13EE901AB4EEC45AF1EEF4
:10E5280010FAB0EE446A88BFB0EE646ABDEEC66AFF
:10E5380016EE10CA16EE106ABC45A8BF3E466145E5
:10E54800C8BF0E4606EE106AB8EEC66A012A80ED0C
:10E55800006A3DF42EA994ED046A9DED0B4A25EE60
:10E56800866AA4EE076AB0EE674AA6EE264AB4EEBB
:10E57800C45AF1EE10FAB0EE446A88BFB0EE646A8D
:10E58800BDEEC66A16EE10CA16EE106ABC45A8BFE4
:10E598003E468C45B8BF0E4606EE106AB8EEC66A0F
:10E5A800022A80ED016A3DF404A994ED086A9DED04
:10E5B8000C4A25EE866AA4EE076AB0EE674AA6EE14
:10E5C800264AB4EEC45AF1EE10FAB0EE446A88BF97
:10E5D800B0EE646ABDEEC66A16EE10CA16EE106A90
:10E5E800BC45A8BF3E468C45B8BF0E4606EE106A2D
:10E5F800B8EEC66A032A80ED026A3DF4DAA894ED03
:10E608000C6A9DED0D4A25EE866AA4EE076AB0EE07
:10E61800674AA6EE264AB4EEC45AF1EE10FAB0EEF6
:10E62800446A88BFB0EE646ABDEEC66A16EE10CAC8
:10E6380016EE106ABC45A8BF3E468C45B8BF0E46CC
:10E6480006EE106AB8EEC66A042A80ED036A3DF445
:10E65800B0A894ED106A9DED0E4A25EE866AA4EEE8
:10E66800076AB0EE674AA6EE264AB4EEC45AF1EE3F
:10E6780010FAB0EE446A88BFB0EE646ABDEEC66AAE
:10E6880016EE10CA16EE106ABC45A8BF3E468C4569
:10E69800B8BF0E4606EE106AB8EEC66A052A80EDC7
:10E6A800046A3DF486A894ED146A9DED0F4A25EEA0
:10E6B800866AA4EE076AB0EE674AA6EE264AB4EE6A
:10E6C800C45AF1EE10FAB0EE446A88BFB0EE646A3C
:10E6D800BDEEC66A16EE10CA16EE106ABC45A8BF93
:10E6E8003E468C45B8BF0E4606EE106AB8EEC66ABE
:10E6F800062A80ED056A3DF45CA894ED186A9DED44
:10E70800104A25EE866AA4EE076AB0EE674AA6EEBE
:10E71800264AB4EEC45AF1EE10FAB0EE446A88BF45
:10E72800B0EE646ABDEEC66A16EE10CA16EE106A3E
:10E73800BC45A8BF3E468C45B8BF0E4606EE106ADB
:10E74800B8EEC66A072A80ED066A3DF432A894ED51
:10E758001C6A9DED114A65EE865AE7EE045AE6EE0C
:10E76800A57AB4EEE75AF1EE10FAC8BFF0EE647A73
:10E77800FDF70FB877EEC76AF0EE477AFFF7DABB16
:10E78800BB8E9FED1B7A07EE903AF8EEE77A194BAD
:10E7980067EE877AC3ED007AFDF760B8B7EE007AC6
:10E7A80077EE677AF4EEE75AF1EE10FA88BFF0EEEA
:10E7B800675AFFF7AABB07EE904ADFED0F6AF8EE3B
:10E7C800E77A66EEA65A9FED0D5A9FED0D6A9FED0A
:10E7D8000D7AA5EE856A26EEA55AA5EE867AE5EEAF
:10E7E800076A26EEA70AFFF7B2B900BFC03C0020AF
:10E7F8006F12833A0400002084F9223F92E741B95E
:10E808009730083C15A82ABE94ED006A9DED0A4A87
:10E81800DC4825EE866AFDEEE43AA4EE076AB0EE1F
:10E82800674AA6EE264A13EE906AB4EEC45AF1EE91
:10E8380010FAB0EE446A88BFB0EE646ABDEEC66AEC
:10E8480016EE10EA16EE101ABE45A8BF39467645F0
:10E85800C8BF314606EE101AB8EEC66A012A80ED26
:10E86800006A3DF4AFAF94ED046A9DED0B4A25EEC6
:10E87800866AA4EE076AB0EE674AA6EE264AB4EEA8
:10E88800C45AF1EE10FAB0EE446A88BFB0EE646A7A
:10E89800BDEEC66A16EE10EA16EE101ABE45A8BFFF
:10E8A8003946B645B8BF314606EE101AB8EEC66A04
:10E8B800022A80ED016A3DF485AF94ED086A9DED6A
:10E8C8000C4A25EE866AA4EE076AB0EE674AA6EE01
:10E8D800264AB4EEC45AF1EE10FAB0EE446A88BF84
:10E8E800B0EE646ABDEEC66A16EE10EA16EE101AAD
:10E8F800BE45A8BF3946B645B8BF314606EE101A20
:10E90800B8EEC66A032A80ED026A3DF45BAF94ED67
:10E918000C6A9DED0D4A25EE866AA4EE076AB0EEF4
:10E92800674AA6EE264AB4EEC45AF1EE10FAB0EEE3
:10E93800446A88BFB0EE646ABDEEC66A16EE10EA95
:10E9480016EE101ABE45A8BF3946B645B8BF3146BF
:10E9580006EE101AB8EEC66A042A80ED036A3DF482
:10E9680031AF94ED106A9DED0E4A25EE866AA4EE4D
:10E97800076AB0EE674AA6EE264AB4EEC45AF1EE2C
:10E9880010FAB0EE446A88BFB0EE646ABDEEC66A9B
:10E9980016EE10EA16EE101ABE45A8BF3946B6455F
:10E9A800B8BF314606EE101AB8EEC66A052A80EDE1
:10E9B800046A3DF407AF94ED146A9DED0F4A25EE05
:10E9C800866AA4EE076AB0EE674AA6EE264AB4EE57
:10E9D800C45AF1EE10FAB0EE446A88BFB0EE646A29
:10E9E800BDEEC66A16EE10EA16EE101ABE45A8BFAE
:10E9F8003946B645B8BF314606EE101AB8EEC66AB3
:10EA0800062A80ED056A3DF4DDAE94ED186A9DEDA9
:10EA1800104A25EE866AA4EE076AB0EE674AA6EEAB
:10EA2800264AB4EEC45AF1EE10FAB0EE446A88BF32
:10EA3800B0EE646ABDEEC66A16EE10EA16EE101A5B
:10EA4800BE45A8BF3946B645B8BF314606EE101ACE
:10EA5800B8EEC66A072A80ED066A3DF4B3AE94EDB7
:10EA68001C6A9DED114A65EE865AE7EE045AE6EEF9
:10EA7800A57AB4EEE75AF1EE10FAC8BFF0EE647A60
:10EA8800FDEEE77A17EE901A8F42A8BF0F468E4226
:10EA9800D8BF3E4607EE906AF8EEE77AC0ED077AEF
:10EAA800FDF78DBE01297FF7EAAB07EE10EAB8EE55
:10EAB800C77AC7EE876AB1EEE68AFFF7E2BB01299B
:10EAC80040F3BF8407EE10EAB8EEC77AC7EE876A4C
:10EAD800B1EEE68A032C14D04FB107EE907AF8EE27
:10EAE800E77AF4EEC87AF1EE10FA00F15585DAF813
:10EAF800603003EB560393FBF6F3CAF82030FFF7B8
:10EB080088BBB0EE480A26F01FFA00B2E4E70129F4
:10EB180040F3938407EE10EAB8EEC77AC7EE876A27
:10EB2800B1EEE68A032C14D04FB107EE907AF8EED6
:10EB3800E77AF4EEC87AF1EE10FA00F12D85DAF8EA
:10EB4800643003EB560393FBF6F3CAF82430FFF75F
:10EB58007BBBB0EE480A26F0F7F900B2E4E70A49B1
:10EB68004A69002A3CF478A90A6813604B74FCF7D8
:10EB780073B9064CFCF7ECBED9F89C41049B1C1BEE
:10EB8800FFF76AB9C03C0020A4760020EC3E0020C4
:10EB9800002E00F0A483E94C9DED0A4A94ED006A2A
:10EBA80025EE866AA4EE076AB0EE674AA6EE264A04
:10EBB800B0EE446A33B1B4EE445AF1EE10FAC8BF6D
:10EBC800B0EE646AFDEEE44ABDEEC66A14EE906AE1
:10EBD80016EE101A8E4214EE90EA00F3D984B94268
:10EBE800A8BF394606EE101AD548B8EEC66A012AFB
:10EBF80080ED006A3CF4E1AD94ED046ADDED0B4A6A
:10EC080025EE866AA4EE876AF0EE674AE6EE264AA3
:10EC1800B0EE646A002B00F0B184B4EEE45AF1EE71
:10EC280010FA40F3AB843146B942A8BF394606EE24
:10EC3800101AB8EEC66A022A80ED016A3CF4BDAD2E
:10EC480094ED086ADDED0C4A25EE866AA4EE876A23
:10EC5800F0EE674AE6EE264AB0EE646A002B00F052
:10EC68008384B4EEE45AF1EE10FA40F37D84314621
:10EC7800B942A8BF394606EE101AB8EEC66A032A8A
:10EC880080ED026A3CF499AD94ED0C6ADDED0D4A15
:10EC980025EE866AA4EE876AF0EE674AE6EE264A13
:10ECA800B0EE646A002B00F05584B4EEE45AF1EE3D
:10ECB80010FA40F34F843146B942A8BF394606EEF0
:10ECC800101AB8EEC66A042A80ED036A3CF475ADE2
:10ECD80094ED106ADDED0E4A25EE866AA4EE876A89
:10ECE800F0EE674AE6EE264AB0EE646A002B00F0C2
:10ECF8002784B4EEE45AF1EE10FA40F32184314649
:10ED0800B942A8BF394606EE101AB8EEC66A052AF7
:10ED180080ED046A3CF451AD94ED146ADDED0F4AC0
:10ED280025EE866AA4EE876AF0EE674AE6EE264A82
:10ED3800B0EE646A002B00F0FA83B4EEE45AF1EE08
:10ED480010FA40F3F4833146B942A8BF394606EEBB
:10ED5800101AB8EEC66A062A80ED056A3CF42DAD95
:10ED680094ED186ADDED104A25EE866AA4EE876AEE
:10ED7800F0EE674AE6EE264AB0EE646A002B00F031
:10ED8800CD83B4EEE45AF1EE10FA40F3C78331466E
:10ED9800B942A8BF394606EE101AB8EEC66A072A65
:10EDA80080ED066A3CF409AD94ED1C6ADDED114A6C
:10EDB80065EE865AE4EE875AE5EEA67A002B00F057
:10EDC800A583F4EEC57AF1EE10FA40F19F8332463E
:10EDD800BA42A8BF3A46964607EE90EAF8EEE77AB6
:10EDE800C0ED077AFCF7E9BCD9F8245148003DB1D9
:10EDF800421804EB82026D785278AA42BDF441AB06
:10EE0800014404EB81040021C9F82441A9F80C123B
:10EE1800C9F81012FDF735BBD9F89C41049B1C1B9F
:10EE2800FFF795B894ED000A039226F08DF845494E
:10EE3800DFF848E1D1F8EC10434B8EFB012EC917DF
:10EE4800C1EBAE1107EE901AF8EEE77A1880FDEEE6
:10EE5800E77A039A17EE901A5980FCF77EBD07EE01
:10EE6800904ADFED3A6A9FED3A7A89F80442F8EE63
:10EE7800E77A67EEA67A77EE876ABDEEE66A16EE5F
:10EE8800102A2032402A40F29282DFED326A324B59
:10EE9800BDEEE77AC3ED016A17EE102A2032402A48
:10EEA80000F282829FED2D7AF4EEC77AF1EE10FA25
:10EEB80040F3FD83DFED2A5A9FED2A6A01E0F0EE68
:10EEC800477AF4EEC67AF1EE10FA37EEE57AF6DC18
:10EED800DFED257AB4EEE77AF1EE10FA40F1DA8345
:10EEE800DFED1F5A9FED216A01E0B0EE677AB4EEBC
:10EEF800C67AF1EE10FA77EE257AF6D49FED147AF9
:10EF0800F4EEC77AF1EE10FA40F39F829FED137A80
:10EF180077EE677A67EEA75A9FED155A9FED156A47
:10EF28009FED157AA5EE856A27EEA55AA5EE867A95
:10EF3800E5EE077AC9ED827AFDF751BD244300203A
:10EF4800C03C002020030020D03D002035FA8E3C34
:10EF5800DB0FC93F0000000004000020DB0F494020
:10EF6800DB0FC940E4CB1641DB0F49C0E4CB16C127
:10EF780092E741B99730083C15A82ABED34D6210D4
:10EF880025EE866AA5EE076AB0EE675AA6EE265AFF
:10EF9800BDEEC56A16EE100A814200F39E81B842A2
:10EFA800A8BF384606EE100AB8EEC66ABCF1000FD4
:10EFB80000F0BC83D148012A80ED006A3CF4FDAB27
:10EFC80094ED046A9DED0B5A25EE866AA5EE076A54
:10EFD800B0EE675AA6EE265ABDEEC56A16EE106A5E
:10EFE800B14200F37881BE42A8BF3E4606EE106AE1
:10EFF800B8EEC66ABCF1000F00F06D83022A80EDFE
:10F00800016A3CF4DAAB94ED086A9DED0C5A25EEE2
:10F01800866AA5EE076AB0EE675AA6EE265ABDEED6
:10F02800C56A16EE106AB14200F35381BE42A8BF0A
:10F038003E4606EE106AB8EEC66ABCF1000F00F054
:10F04800A183032A80ED026A3CF4B7AB94ED0C6A05
:10F058009DED0D5A25EE866AA5EE076AB0EE675A51
:10F06800A6EE265ABDEEC56A16EE106AB14200F346
:10F078002E81BE42A8BF3E4606EE106AB8EEC66AAA
:10F08800BCF1000F00F07383042A80ED036A3CF49E
:10F0980094AB94ED106A9DED0E5A25EE866AA5EEA6
:10F0A800076AB0EE675AA6EE265ABDEEC56A16EE96
:10F0B800106AB14200F30981BE42A8BF3E4606EE7F
:10F0C800106AB8EEC66ABCF1000F00F04583052A45
:10F0D80080ED046A3CF471AB94ED146A9DED0F5A0F
:10F0E80025EE866AA5EE076AB0EE675AA6EE265A9E
:10F0F800BDEEC56A16EE106AB14200F3E480BE4266
:10F10800A8BF3E4606EE106AB8EEC66ABCF1000F0C
:10F1180000F01783062A80ED056A3CF44EAB94EDA7
:10F12800186A9DED105A25EE866AA5EE076AB0EEBC
:10F13800675AA6EE265ABDEEC56A16EE106AB142A7
:10F1480000F3BF80BE42A8BF3E4606EE106AB8EE86
:10F15800C66ABCF1000F00F07E83072A80ED066ABC
:10F168003CF42BAB94ED1C6A9DED115A65EE865A62
:10F17800E7EE055AE6EEA57AFDEEE77A17EE902A55
:10F18800914203DCBA42A8BF3A46114607EE901AEC
:10F19800F8EEE77ABCF1000F7FF422AE089B002B53
:10F1A8007FF41EAE039B079A9342B8BFF0EE647AD1
:10F1B80016E69FED530A534B25EE800A1C4625F0B0
:10F1C800C3FEE080D9F81441FCF74ABE4E484F49C7
:10F1D8008446FEF7C3B9D9F89C41049B1C1BFEF773
:10F1E80009B84B49096811F0805C7EF481AEFEF7DE
:10F1F80077BE237DFEF774BD93F8FF21AA2A7EF41B
:10F20800E2ADD3F8C61149B193F8C221A2F10B00BF
:10F2180001282DD902F0F702062A29D0D3F8D611F1
:10F2280049B193F8D221A2F10B00012820D902F0AC
:10F23800F702062A1CD0D3F8E61149B193F8E22167
:10F24800A2F10B00012813D902F0F702062A0FD009
:10F25800D3F8F61100293EF4B6AD93F8F231A3F1D4
:10F268000B02012A04D903F0F703062B7EF4ABAD99
:10F2780041F2FC120123A150A370FEF7ADBDF8F7CF
:10F2880053FB029A1F4B1778039A98F80010D9F885
:10F298001441801A9880FEF71FBBF8F745FB029AC5
:10F2A800184B1778039A801A5880FEF780B9F8F738
:10F2B8003BFB029A134B1778039A801A5880FEF783
:10F2C800B7B90E4641E70E461CE70E46F7E60E466E
:10F2D800D2E60E46ADE60E4688E6084662E60AA97C
:10F2E800BDEEE46A01EB820296460A48034C099592
:10F2F8001A4616EE106A634614E000BFC03C0020B0
:10F308000000C842D03D00203C3A00201C200020CC
:10F31800A4370020244300207145A4EC016A00F1C1
:10F32800100039D090ED006AB1EC014A25EE866AEA
:10F33800A7EE046AB0EE674AA6EE864AB0EE446AC3
:10F3480032B1B4EE445AF1EE10FAC8BFB0EE646AB6
:10F35800BDEEC66A16EE10CA664506EE106A04DCF3
:10F36800BC45A8BFBC4606EE10CAB8EEC66A002B5C
:10F37800D2D1089D002DCFD1039DAC46079DAC4549
:10F38800B8BFB0EE646AC7E7D84A1278032A00F01B
:10F398007D810022FEF7A3BF099DFCF70EBAD44E6B
:10F3A80006F18002FEF780BADFEDD27AC2E5F4EE0C
:10F3B800C77AF1EE10FA40F37D81DFEDCF5A9FED69
:10F3C800CF6A01E0F0EE476AF4EEC66AF1EE10FA91
:10F3D80036EEE57AF6DCDFEDCA6AB4EEE67AF1EEEF
:10F3E80010FA40F15A81DFEDC45A9FEDC66A01E078
:10F3F800B0EE667AB4EEC67AF1EE10FA77EE256AC8
:10F40800F6D49FEDC17AF4EEC76AF1EE10FA71DD19
:10F418009FEDBE7A77EE666A66EEA65A9FEDBC5AF5
:10F428009FEDBC6A9FEDBC7AA5EE856A26EEA55ACB
:10F43800A5EE867AE5EE076A29E59FEDAE8AFFF725
:10F4480071BB9FEDAC8AFFF745BB9FEDB47AF4EE34
:10F45800C77AF1EE10FA44BF9FEDA97A77EE677A82
:10F4680058E59FEDAA7AF4EEC76AF1EE10FA40F378
:10F478002781DFEDA15A9FEDA16A01E0F0EE476A0E
:10F48800F4EEC66AF1EE10FA36EEE57AF6DCDFED58
:10F498009C6AB4EEE67AF1EE10FA40F10E81DFEDE7
:10F4A800965A9FED986A01E0B0EE667AB4EEC67A95
:10F4B800F1EE10FA77EE256AF6D49FED937AF4EE22
:10F4C800C76AF1EE10FA05DD9FED907A77EE666A6D
:10F4D800FFF777B99FED917AF4EEC76AF1EE10FA6B
:10F4E80044BF9FED877A77EE666AFFF76AB9604690
:10F4F800FEF7DABF9FED897AF4EEC76AF1EE10FAEB
:10F5080044BF9FED7F7A77EE666A85E7FDEEE77A7E
:10F5180017EE902AB242FFF65FAC59E4BDEEC66A18
:10F5280016EE101AB142BFF633AC314633E4BDEEE5
:10F53800C66A16EE101AB142BFF606AC314606E4AA
:10F54800BDEEC66A16EE101AB142BFF6D9AB314607
:10F55800FFF7D9BBBDEEC66A16EE101AB142BFF668
:10F56800ABAB3146FFF7ABBBBDEEC66A16EE101A61
:10F57800B142BFF67DAB3146FFF77DBBBDEEC66A33
:10F5880016EE101AB142BFF64FAB3146FFF74FBB2C
:10F5980014EE901AFFF726BB039BAAF8A860D88040
:10F5A800DFF84C91FCF774BF137C022B7EF428AC77
:10F5B80092F8FE31552B7EF423AC92F8FF31AA2B3A
:10F5C8007EF41EACD689E759554B37441F6092F834
:10F5D8000DE041F210210EF1FF337F2B44F801E0DA
:10F5E8003EF60EACCEF100033EEA03037EF408AC0F
:10F5F8004FEA4E2341F21821013B6350D08A00B9EB
:10F60800506A484941F20423E050B2F811305B01D6
:10F6180003F2FF135B120B60B2F8131001B9116A01
:10F6280040001E440644891B41F2082C40F6F4763B
:10F63800B1FBFEF1B14244F80C1048D94FF6F4760C
:10F64800B14240D903212170D26A37493B4418445A
:10F6580041F20C2641F21C230978A051E25009B965
:10F6680025F0DCF9A3780133A370FCF71BBB022853
:10F678007CF418AB41F2B4120123A3546370FCF775
:10F6880011BB10F079FE2369FEF7F9BA22F0DAF916
:10F69800FCF7F7BEF0EE477A30E4F0EE476AB0E6E2
:10F6A80099F87831002B7BF4A5ACFBF790BCB0EE51
:10F6B800677A0DE4B0EE667A8DE6F0EE476AFCE60E
:10F6C800B0EE667AE3E6022222700022BDE701234B
:10F6D8002370FEF795BB089B002B7FF48FAC039B30
:10F6E800079EB342B8BFB0EE646A87E4547800203E
:10F6F8001C20002000000000DB0FC940E4CB1641AD
:10F70800DB0F49C0E4CB16C1DB0FC93FDB0F494013
:10F7180092E741B99730083C15A82ABEDB0FC9BF4C
:10F728001469002034690020F4680020089B002B2D
:10F738007FF440AC039B07988342B8BFB0EE646A7D
:10F7480038E4089B002B7FF4E5AC039B079EB3428B
:10F75800B8BFB0EE646ADDE4089B002B7FF4B7AC59
:10F76800039B079EB342B8BFB0EE646AAFE4089B40
:10F77800002B7FF489AC039B079EB342B8BFB0EE61
:10F78800646A81E4089B002B7FF45BAC039B079EB3
:10F79800B342B8BFB0EE646A53E4132B05D1B0EEA0
:10F7A800480A25F0D1FB039B1880B0EE480ADAF826
:10F7B800083245489847029B1B78132BB0EE408AC5
:10F7C8007CF472AC25F0C0FB039B5880FCF76CBC42
:10F7D8003E4A3F4B10681B6898473E4BD6ED006A7F
:10F7E80093ED007A3C4BD3ED007A3C4B83ED020A53
:10F7F8003B4B67EE277A234427EEAC7AD3ED007AA9
:10F80800384B67EE277AF0EE665AEDEEA75A93ED7D
:10F81800006AB1EE467AB4EEE57AF1EE10FA08DC49
:10F82800B4EEE56AF1EE10FA8CBFB0EE657AB0EE90
:10F83800467A2D4B1B78012B02D0192B7BF444AB55
:10F84800DFED2A7AF4EEE7DAF1EE10FACCBF012305
:10F858000023FBF744BB089B002B7FF47EAC039B83
:10F86800079EB342B8BFB0EE646A76E4DFED207A53
:10F87800B4EEE7EAF1EE10FA20DCDFED1E7AB4EE22
:10F88800E7EAF1EE10FA19D41B4BD3ED007AB1EE8A
:10F89800677AF4EEC7DAF1EE10FA12D4F4EEE7DA8A
:10F8A800F1EE10FA88BFF0EE67DA144B86ED00CA65
:10F8B8001B689342BBF612AAFBF73ABADFED10DADF
:10F8C800F3E7F0EE47DAF0E78C4F0020A875002048
:10F8D800BC750020FC74002004000020503C00206F
:10F8E800CC75002034760020607400200000964219
:10F8F80000C0F84400C0F8C4307600201476002018
:10F9080000000000436A8269D154436A0169826B2E
:10F9180001338B4228BF00234362002A2FD0EFF324
:10F928001181502383F31288836B1A68D2072CD471
:10F9380070B45E686EB9456A826A954217D0846968
:10F948001444DC600ED9AA1A5A608562002280F835
:10F9580054201A6842F00102C9B21A6081F3118872
:10F9680070BC70470469A21A5A608662EEE70123E8
:10F9780080F85430C9B281F3118870BC7047026DA9
:10F98800136843F0800313607047C9B281F311888C
:10F99800704700BF426B10B462B1436CC2684469DF
:10F9A800D11A013B615C5DF8044B08BF1346436400
:10F9B800C8B27047016A4369C4685B5C0131A142FF
:10F9C80028BF114601625DF8044BD8B2704700BFEA
:10F9D800836B13B190F854007047836A406A181A11
:10F9E800B0FA80F040097047416A836A99420AD3A5
:10F9F800CB1A816B026961B14968501E0B4483427E
:10FA08000AD2C01A704702691144CB1A816B0029C7
:10FA1800F2D1501EC01A704700207047436B43B1A3
:10FA2800426C5B6893422FBF981AC0689B1AC01833
:10FA38007047C269036A9A422FBFD01AC0688018FB
:10FA4800C01A70470A4B30B503F10C0493F9002033
:10FA58005D78072AC8BF143A811804338D7213F8E9
:10FA6800025C855413F8012C0A75A342EED130BD0F
:10FA78005861030803682DE9F041DF691FB13B466F
:10FA8800BDE8F0411847002A164611DD04460D4628
:10FA98000E4400E023689B68204698470028F9D068
:10FAA800236815F8011B1B6820469847AE42F1D120
:10FAB800BDE8F08100232822027043708370C37070
:10FAC8007047232303702423C370252383712D23B8
:10FAD80043702E2303712F23C371704730B504463A
:10FAE800006D61710368A26823F00103036087B0A9
:10FAF800A379009213F004023DD04FF4805213F022
:10FB08000203019244D102934FF4806300220393CD
:10FB180011F00103059237D1049308238D07694634
:10FB280048BF04931AF078FA6079236DA17900F040
:10FB38000202002A15BF4FF440324FF480324FF4CE
:10FB48000034002410F0010F586808BF2246CC0783
:10FB58004CBF024320EA02025A609A6809074CBF68
:10FB680042F0080222F008029A601A6842F0010284
:10FB78001A6007B030BD13F0020301920BD04FF4A6
:10FB8800005513460295C1E7042304930C23C5E7E7
:10FB98004FF40053B7E70293B8E700BF10B5044627
:10FBA800006DA160036823F001030360A37986B0A8
:10FBB80013F00402009141D04FF4805213F0020375
:10FBC800019244D102934FF4806362790393D10781
:10FBD8004FF000030493059345BF042304930823BF
:10FBE8000C236946920748BF04931AF015FA607906
:10FBF800236DA17900F00202002A15BF4FF44032AC
:10FC08004FF480324FF40034002410F0010F58688C
:10FC180008BF2246CC074CBF024320EA02025A60C2
:10FC28009A6809074CBF42F0080222F008029A605D
:10FC38001A6842F001021A6006B010BD13F0020300
:10FC4800019207D04FF4005113460291BDE74FF4DB
:10FC58000053B7E70293B8E7002326220360027037
:10FC6800272282700122436002718371704700BFAE
:10FC78001D4B70B51C68236D626BDD69C2B1A36B47
:10FC88002BB12B0702D5236D08221A6270BD2A06F4
:10FC9800F7D5A26A616A8A4220D0511CA069A16284
:10FCA800825C2069266D81423285EAD3A362E8E747
:10FCB800A906E4D5E26A22B1988C216B80B29047FC
:10FCC800DDE7E1699B8C6069DBB24E1CE661435459
:10FCD800E169E368994228BFE261D0E7226D1368C1
:10FCE80023F080031360CCE7F42A002070B4EFF30C
:10FCF8001186502383F31288836B1A68D20720D4A5
:10FD08005D686DB9446A826A944217D0816911446A
:10FD1800D9600ED9A21A5A608462002280F8542051
:10FD28001A6842F00102F1B21A6081F3118870BCBE
:10FD3800704701698A1A5A608562EEE7012380F8E4
:10FD48005430F1B281F3118870BC704703685B6A64
:10FD580003B11847704700BF03681B6A03B118470F
:10FD6800704700BF03682DE9F041DF691FB13B46CA
:10FD7800BDE8F0411847002A164611DD04460D4635
:10FD88000E4400E023689B68204698470028F9D075
:10FD9800236815F8011B1B6820469847AE42F1D12D
:10FDA800BDE8F08103689B69184700BF0368DB68FA
:10FDB800184700BF03689B68184700BF03685B6863
:10FDC800184700BF03681B68184700BF054B53F866
:10FDD800203033B11A689B88918A0B4218BF1B04E4
:10FDE800936170479076002003682DE9F04F03F186
:10FDF8003845644EAD0A0124755D05F01F066D098E
:10FE0800022D04FA06F400F0A280032D00F0A4806D
:10FE1800012D52D08088B0FA80F4C4F11F04A4B236
:10FE2800E50803EB850504F007042E6AA4000F27F4
:10FE3800A74026EA07062E622E6A01F0030702FA97
:10FE480004F47A1E3443012AC1F3810CC1F300186B
:10FE58002C62C1F3411135D9C60700F19780850797
:10FE680000F1A380440700F1B180020700F1BF80D0
:10FE7800C60600F1CD80850600F1DB80440600F15E
:10FE8800E980020600F1F780C60500F105818505C5
:10FE980000F11381440500F12181020500F12F8151
:10FEA800C60400F13D81850400F14B81440400F152
:10FEB8005981020455D4BDE8F08F334D6E6934433F
:10FEC8006C61A7E7002422464FF0010E4FF00309AA
:10FED80004E00132102A04F10204ECD00EFA02F612
:10FEE80036EA0005F5D1D3F808A009FA04F5ED4380
:10FEF8000AEA050AC3F808A0D3F808B00CFA04FA0D
:10FF08004AEA0B0AC3F808A0B3F804A01FFA8AFA51
:10FF18002AEA06069E80B3F804A008FA02F646EA22
:10FF28000A06B6B29E801E682E401E60D3F800A056
:10FF380007FA04F646EA0A061E60D3F80CA001FA8E
:10FF480004F605EA0A0A46EA0A05DD60C1E70E4D2D
:10FF5800AE693443AC615DE70B4DEE693443EC6147
:10FF680058E71A6822F040421A601A6842EA87770E
:10FF78001F60DA6822F0404242EA8171D960BDE828
:10FF8800F08F00BF3C880308001002401A6822F076
:10FF980003021A601A683A431A60DA6822F0030208
:10FFA8000A438507DA607FF55DAF1A6822F00C0214
:10FFB8001A601A6842EA87021A60DA6822F00C02AC
:10FFC80042EA81024407DA607FF54FAF1A6822F0EF
:10FFD80030021A601A6842EA07121A60DA6822F0D8
:10FFE800300242EA0112DA6002077FF541AF1A686F
:08FFF80022F0C0021A601A6831
:020000040801F1
:1000000042EA87121A60DA6822F0C00242EA8112DC
:10001000C606DA607FF533AF1A6822F440721A60C0
:100020001A6842EA07221A60DA6822F4407242EA49
:1000300001228506DA607FF525AF1A6822F4406256
:100040001A601A6842EA87221A60DA6822F440626B
:1000500042EA81224406DA607FF517AF1A6822F47B
:1000600040521A601A6842EA07321A60DA6822F4CB
:10007000405242EA0132DA6002067FF509AF1A689F
:1000800022F440421A601A6842EA87321A60DA683B
:1000900022F4404242EA8132C605DA607FF5FBAEC7
:1000A0001A6822F440321A601A6842EA07421A605B
:1000B000DA6822F4403242EA01428505DA607FF5CF
:1000C000EDAE1A6822F440221A601A6842EA8742AA
:1000D0001A60DA6822F4402242EA81424405DA607A
:1000E0007FF5DFAE1A6822F440121A601A6842EAFD
:1000F00007521A60DA6822F4401242EA0152DA60CA
:1001000002057FF5D1AE1A6822F440021A601A681F
:1001100042EA87521A60DA6822F4400242EA8152C7
:10012000C604DA607FF5C3AE1A6822F040721A6026
:100130001A6842EA07621A60DA6822F0407242EAFC
:1001400001628504DA607FF5B5AE1A6822F040627C
:100150001A601A6842EA87621A60DA6822F040621E
:1001600042EA81624404DA607FF5A7AE1A6822F0A1
:1001700040521A601A6842EA07721A60DA6822F07E
:10018000405242EA0172DA6097E600BF036803F169
:1001900038422DE9F04F920A584DAA5C02F01F0533
:1001A00052090124022A04FA05F400F08C80032A83
:1001B00000F08E80012A3CD001F003077A1E012A4C
:1001C000C1F3810CC1F300188088C1F3411135D906
:1001D000C60700F19780850700F1A380440700F16E
:1001E000B180020700F1BF80C60600F1CD80850610
:1001F00000F1DB80440600F1E980020600F1F7809F
:10020000C60500F10581850500F11381440500F163
:100210002181020500F12F81C60400F13D81850492
:1002200000F14B81440400F15981020455D4BDE82A
:10023000F08F334A55692C435461BDE700242246B0
:100240004FF0010E4FF0030904E00132102A04F1CF
:100250000204ECD00EFA02F636EA0005F5D1D3F826
:1002600008A009FA04F5ED430AEA050AC3F808A054
:10027000D3F808B00CFA04FA4AEA0B0AC3F808A04B
:10028000B3F804A01FFA8AFA2AEA06069E80B3F899
:1002900004A008FA02F646EA0A06B6B29E801E6874
:1002A0002E401E60D3F800A007FA04F646EA0A06BC
:1002B0001E60D3F80CA001FA04F605EA0A0A46EA21
:1002C0000A05DD60C1E70E4A95692C43946173E726
:1002D0000B4AD5692C43D4616EE71A6822F040427C
:1002E0001A601A6842EA87771F60DA6822F0404293
:1002F00042EA8171D960BDE8F08F00BF3C880308F5
:10030000001002401A6822F003021A601A683A4389
:100310001A60DA6822F003020A438507DA607FF583
:100320005DAF1A6822F00C021A601A6842EA87026E
:100330001A60DA6822F00C0242EA81024407DA60AD
:100340007FF54FAF1A6822F030021A601A6842EA4D
:1003500007121A60DA6822F0300242EA0112DA600B
:1003600002077FF541AF1A6822F0C0021A601A68CE
:1003700042EA87121A60DA6822F0C00242EA811269
:10038000C606DA607FF533AF1A6822F440721A604D
:100390001A6842EA07221A60DA6822F4407242EAD6
:1003A00001228506DA607FF525AF1A6822F44062E3
:1003B0001A601A6842EA87221A60DA6822F44062F8
:1003C00042EA81224406DA607FF517AF1A6822F408
:1003D00040521A601A6842EA07321A60DA6822F458
:1003E000405242EA0132DA6002067FF509AF1A682C
:1003F00022F440421A601A6842EA87321A60DA68C8
:1004000022F4404242EA8132C605DA607FF5FBAE53
:100410001A6822F440321A601A6842EA07421A60E7
:10042000DA6822F4403242EA01428505DA607FF55B
:10043000EDAE1A6822F440221A601A6842EA874236
:100440001A60DA6822F4402242EA81424405DA6006
:100450007FF5DFAE1A6822F440121A601A6842EA89
:1004600007521A60DA6822F4401242EA0152DA6056
:1004700002057FF5D1AE1A6822F440021A601A68AC
:1004800042EA87521A60DA6822F4400242EA815254
:10049000C604DA607FF5C3AE1A6822F040721A60B3
:1004A0001A6842EA07621A60DA6822F0407242EA89
:1004B00001628504DA607FF5B5AE1A6822F0406209
:1004C0001A601A6842EA87621A60DA6822F04062AB
:1004D00042EA81624404DA607FF5A7AE1A6822F02E
:1004E00040521A601A6842EA07721A60DA6822F00B
:1004F000405242EA0172DA6097E600BF10B5040983
:10050000013C052C17D80D4B33F8142000F00F00D8
:1005100042FA00F313F001030DD0012303FA00F0B7
:100520000138104024F0BEF8054A064B125D104415
:1005300003EBC00010BD002010BD00BF28880308D9
:1005400034880308FC7E00202DE9F04F4A484B4BCD
:100550004B4C4FF090414FF0010A4FF002094FF021
:1005600004084FF0080C4FF0100E2027402680257D
:1005700030F8022B12F0010F03D01960A3F804A089
:10058000083312F0020F03D01960A3F80490083367
:1005900012F0040F03D01960A3F80480083312F09E
:1005A000080F03D01960A3F804C0083312F0100F2D
:1005B00003D01960A3F804E0083312F0200F02D032
:1005C00019609F80083312F0400F02D019609E809E
:1005D000083312F0800F02D019609D80083312F4A6
:1005E000807F05D04FF4807B1960A3F804B00833F6
:1005F00012F4007F05D04FF4007B1960A3F804B01B
:10060000083312F4806F05D04FF4806B1960A3F8A3
:1006100004B0083312F4006F05D04FF4006B19607A
:10062000A3F804B0083312F4805F05D04FF4805B68
:100630001960A3F804B0083312F4005F05D04FF43A
:10064000005B1960A3F804B0083312F4804F05D0A2
:100650004FF4804B1960A3F804B00833D20B04D0D8
:100660004FF4004219609A80083301F58061A1427D
:100670007FF47EAFBDE8F08F28880308FC7E002061
:1006800000180048002867D003682DE9F04F03F1F7
:1006900038445C4EA40A0125345D04F01F06640949
:1006A000022C05FA06F558D0032C00F0A580012C89
:1006B00058D08088B0FA80F4C4F11F04A4B2E508D1
:1006C00003EB850504F007042E6AA4000F27A7405A
:1006D00026EA07062E622E6A01F00307A2407C1E5E
:1006E0003243012CC1F3810CC1F300182A62C1F31B
:1006F00041113CD9C60700F18980850700F195803A
:10070000440700F1A380020700F1B180C60600F1A2
:10071000BF80850600F1CD80440600F1DB80020633
:1007200000F1E980C60500F1F780850500F105813B
:10073000440500F11381020500F12181C60400F196
:100740002F81850400F13D81440400F14B810204B6
:1007500000F15981BDE8F08F70472B4CA6693543F5
:10076000A561A6E7284C666935436561A1E70024C9
:1007700022464FF0010E4FF0030904E00132102A27
:1007800004F10204E6D00EFA02F636EA0005F5D1CD
:10079000D3F808A009FA04F5ED430AEA050AC3F8FC
:1007A00008A0D3F808B00CFA04FA4AEA0B0AC3F816
:1007B00008A0B3F804A01FFA8AFA2AEA06069E8067
:1007C000B3F804A008FA02F646EA0A06B6B29E801A
:1007D0001E682E401E60D3F800A007FA04F646EA11
:1007E0000A061E60D3F80CA001FA04F605EA0A0A0C
:1007F00046EA0A05DD60C1E7034CE6693543E56179
:1008000057E700BF3C880308001002401A6822F036
:1008100003021A601A683A431A60DA6822F0030287
:100820000A438507DA607FF56BAF1A6822F00C0285
:100830001A601A6842EA87021A60DA6822F00C022B
:1008400042EA81024407DA607FF55DAF1A6822F060
:1008500030021A601A6842EA07121A60DA6822F057
:10086000300242EA0112DA6002077FF54FAF1A68E0
:1008700022F0C0021A601A6842EA87121A60DA6827
:1008800022F0C00242EA8112C606DA607FF541AF6B
:100890001A6822F440721A601A6842EA07221A6043
:1008A000DA6822F4407242EA01228506DA607FF5B6
:1008B00033AF1A6822F440621A601A6842EA87224B
:1008C0001A60DA6822F4406242EA81224406DA6061
:1008D0007FF525AF1A6822F440521A601A6842EA7E
:1008E00007321A60DA6822F4405242EA0132DA60D2
:1008F00002067FF517AF1A6822F440421A601A68A0
:1009000042EA87321A60DA6822F4404242EA8132CF
:10091000C605DA607FF509AF1A6822F440321A6022
:100920001A6842EA07421A60DA6822F4403242EA60
:1009300001428505DA607FF5FBAE1A6822F4402299
:100940001A601A6842EA87421A60DA6822F4402282
:1009500042EA81424405DA607FF5EDAE1A6822F47E
:1009600040121A601A6842EA07521A60DA6822F4E2
:10097000401242EA0152DA6002057FF5DFAE1A68E2
:1009800022F440021A601A6842EA87521A60DA6852
:1009900022F4400242EA8152C604DA607FF5D1AE09
:1009A0001A6822F040721A601A6842EA07621A60F6
:1009B000DA6822F0407242EA01628504DA607FF56B
:1009C000C3AE1A6822F040621A601A6842EA87626F
:1009D0001A60DA6822F0406242EA81624404DA6016
:1009E0007FF5B5AE1A6822F040521A601A6842EAE2
:1009F00007721A60DA6822F0405242EA0172DA6045
:100A000002047FF5A7AE1A6822F040421A601A6805
:100A100042EA87771F60DA6822F0404242EA817139
:100A2000D960BDE8F08F00BF002852D0036803F101
:100A300038422DE9F04F920A504DAA5C02F01F0592
:100A400052090124022A04FA05F443D0032A00F0D3
:100A50009080012A43D001F003077A1E012AC1F3D6
:100A6000810CC1F300188088C1F341113CD9C6073D
:100A700000F18880850700F19480440700F1A2808E
:100A8000020700F1B080C60600F1BE80850600F1C5
:100A9000CC80440600F1DA80020600F1E880C60549
:100AA00000F1F680850500F10481440500F1128112
:100AB000020500F12081C60400F12E81850400F1B9
:100AC0003C81440400F14A81020400F15881BDE8F0
:100AD000F08F70472A4A95692C439461BBE7284AF6
:100AE00055692C435461B6E7002422464FF0010EAD
:100AF0004FF0030904E00132102A04F10204E6D0A9
:100B00000EFA02F636EA0005F5D1D3F808A009FA84
:100B100004F5ED430AEA050AC3F808A0D3F808B0C3
:100B20000CFA04FA4AEA0B0AC3F808A0B3F804A0C6
:100B30001FFA8AFA2AEA06069E80B3F804A008FA89
:100B400002F646EA0A06B6B29E801E682E401E6075
:100B5000D3F800A007FA04F646EA0A061E60D3F8A6
:100B60000CA001FA04F605EA0A0A46EA0A05DD6065
:100B7000C1E7034AD5692C43D4616CE73C8803087C
:100B8000001002401A6822F003021A601A683A4301
:100B90001A60DA6822F003020A438507DA607FF5FB
:100BA0006CAF1A6822F00C021A601A6842EA8702D7
:100BB0001A60DA6822F00C0242EA81024407DA6025
:100BC0007FF55EAF1A6822F030021A601A6842EAB6
:100BD00007121A60DA6822F0300242EA0112DA6083
:100BE00002077FF550AF1A6822F0C0021A601A6837
:100BF00042EA87121A60DA6822F0C00242EA8112E1
:100C0000C606DA607FF542AF1A6822F440721A60B5
:100C10001A6842EA07221A60DA6822F4407242EA4D
:100C200001228506DA607FF534AF1A6822F440624B
:100C30001A601A6842EA87221A60DA6822F440626F
:100C400042EA81224406DA607FF526AF1A6822F470
:100C500040521A601A6842EA07321A60DA6822F4CF
:100C6000405242EA0132DA6002067FF518AF1A6894
:100C700022F440421A601A6842EA87321A60DA683F
:100C800022F4404242EA8132C605DA607FF50AAFBB
:100C90001A6822F440321A601A6842EA07421A605F
:100CA000DA6822F4403242EA01428505DA607FF5D3
:100CB000FCAE1A6822F440221A601A6842EA87429F
:100CC0001A60DA6822F4402242EA81424405DA607E
:100CD0007FF5EEAE1A6822F440121A601A6842EAF2
:100CE00007521A60DA6822F4401242EA0152DA60CE
:100CF00002057FF5E0AE1A6822F440021A601A6815
:100D000042EA87521A60DA6822F4400242EA8152CB
:100D1000C604DA607FF5D2AE1A6822F040721A601B
:100D20001A6842EA07621A60DA6822F0407242EA00
:100D300001628504DA607FF5C4AE1A6822F0406271
:100D40001A601A6842EA87621A60DA6822F0406222
:100D500042EA81624404DA607FF5B6AE1A6822F096
:100D600040521A601A6842EA07721A60DA6822F082
:100D7000405242EA0172DA6002047FF5A8AE1A68B6
:100D800022F040421A601A6842EA87771F60DA68E8
:100D900022F0404242EA8171D960BDE8F08F00BF85
:100DA00010B1036882881A85704700BF10B10368CC
:100DB00082889A61704700BF38B100298388026831
:100DC00014BF002110218B409361704710B40A4B6F
:100DD0000A4A1C7801238340234052F8200029B995
:100DE000B3FA83F149095DF8044BE5E7191C18BF14
:100DF00001215DF8044BDFE78C760020907600201F
:100E000030B1036882881B8A1A4214BF0120002077
:100E1000704700BF2DE9F0410B4E346873691C40E8
:100E20000FD0DFF828800127B4FA84F3C3F11F0341
:100E300007FA03F558F8230003689847AC43756137
:100E4000F2D1BDE8F08100BF00040140342200204F
:100E50002DE9F0410B4E346873691C400FD0DFF868
:100E600028800127B4FA84F3C3F11F0307FA03F5BE
:100E700058F8230003689847AC437561F2D1BDE888
:100E8000F08100BF00040140342200202DE9F04130
:100E90000B4E346873691C400FD0DFF8288001279F
:100EA000B4FA84F3C3F11F0307FA03F558F82300DB
:100EB00003689847AC437561F2D1BDE8F08100BF8B
:100EC00000040140342200202DE9F0410B4E34682B
:100ED00073691C400FD0DFF828800127B4FA84F32F
:100EE000C3F11F0307FA03F558F823000368984776
:100EF000AC437561F2D1BDE8F08100BF0004014050
:100F0000342200202DE9F0410B4E346873691C40F7
:100F10000FD0DFF828800127B4FA84F3C3F11F0350
:100F200007FA03F558F8230003689847AC43756146
:100F3000F2D1BDE8F08100BF00040140342200205E
:100F40002DE9F0410B4E346873691C400FD0DFF877
:100F500028800127B4FA84F3C3F11F0307FA03F5CD
:100F600058F8230003689847AC437561F2D1BDE897
:100F7000F08100BF00040140342200202DE9F0413F
:100F80000B4E346873691C400FD0DFF828800127AE
:100F9000B4FA84F3C3F11F0307FA03F558F82300EA
:100FA00003689847AC437561F2D1BDE8F08100BF9A
:100FB0000004014034220020084A936910B5084C0F
:100FC00043F00103936120464022002124F07DFF7D
:100FD0004FF0FF332364C4F8433010BD00100240CB
:100FE0003422002003681B6A184700BF70B44E1CEF
:100FF0000568C2728672AC69A44670BC604700BFC7
:101000002DE9F041044618460D461646984622F052
:101010002FFE2768E6722844A07229467D69434660
:1010200032462046AC46BDE8F0416047036810B543
:1010300004461B689847236820469B689847A37B13
:101040000133A37310BD00BF03681B69184700BFBD
:1010500010B5036804469B689847FF230122637319
:10106000227310BD08B5FFF749FA38B12D228271FD
:101070000022C2712021BDE80840D5E408BD00BFB0
:101080000B4B984206D0A3F5784398420DD04FF011
:10109000FF3070470022074B03EB02135A890132DD
:1010A00092B25A81588980B270470122F3E700BF9B
:1010B00000300140283D0020F8B5054680681646FE
:1010C0001F4610B1036882881A8541F08001686864
:1010D00040F2E93401E0002C44D00389013C13F0D4
:1010E000020FA4B2F7D0017340F2E93101E0002908
:1010F00038D00389013913F0010F89B2F7D0037B8F
:10110000686883894FF0000C4FF47A714FF6FF72D4
:101110004FF0FF0E674502D11DE0914219D00389BF
:1011200001399C0789B2F8D580F80CE04FF47A7148
:1011300002E0A1B291420CD00389DB0701F1FF3438
:10114000F7D5037BDBB20EB1337001360CF1010C25
:10115000E0E7FFF795FFAB6813B11A689B889361CE
:101160000120F8BDFFF78CFFCAE700BF38B58368E0
:101170000446154613B11A689B881385606840F2CF
:10118000E93300E07BB30289013B12F0020F9BB20E
:10119000F8D0017340F2E93300E023B30289013B48
:1011A00012F0010F9BB2F8D0037B606840F2E93384
:1011B00000E0DBB10189013B11F0020F9BB2F8D0D6
:1011C000057340F2E93300E083B10289013B12F07C
:1011D000010F9BB2F8D0037BA36813B11A689B88F8
:1011E0009361012038BDFFF74BFFDEE7FFF748FFB3
:1011F000F2E700BFF0B50E460178012985B004463C
:101200004BD002294FD11D46836846F0800113B1AF
:1012100018689B880385606840F2E93301E0002B81
:1012200055D00689013B16F0020F9BB2F7D001732F
:1012300040F2E93301E0002B49D00189013B11F074
:10124000010F9BB2F7D0037B60684FF0000C8389DD
:101250004FF6FF764FF47A734FF0FF0E654502D1DB
:1012600026E0B34222D00189013B8F079BB2F8D51B
:1012700080F80CE04FF47A7302E0BBB2B34215D0B1
:101280000189C90703F1FF37F7D5017BC9B20AB15C
:10129000117001320CF1010CE0E790F90400411CDF
:1012A00001D002280CDD002005B0F0BDFFF7E8FEFC
:1012B000A3688BB11A689B889361012005B0F0BDCB
:1012C000617900923246F1F7D1FF05B0F0BD03928B
:1012D000FFF7D6FE039AB7E70120E5E7F8B50378F4
:1012E000012B49D0022B4DD1836801F07F0113B14E
:1012F0001C689B88238504461546406840F2E93304
:1013000002E0002B00F0B1800289013B12F0020FD5
:101310009BB2F6D0017340F2E93302E0002B00F0FB
:10132000A4800289013B12F0010F9BB2F6D0037B2F
:10133000606840F2E93302E0002B00F093800189FD
:10134000013B11F0020F9BB2F6D0057340F2E93376
:1013500002E0002B00F086800289013B12F0010FB1
:101360009BB2F6D0037BA368002B00F088801A683C
:101370009B8893610120F8BD90F904305C1C01D07A
:10138000022B01DD0020F8BD464C03EB830304EB88
:1013900083035E68002EF5D04579434C4FF420431B
:1013A0006D00A364EDB249F6FF73B06907044CD435
:1013B00070683E4F45F0807343F4903338401843D3
:1013C0004FF420437060A36401E05F1C50D0B0690B
:1013D00010F0020003F1FF33F7D04FF42043A36471
:1013E000B16249F6FF7301E09F1C4AD0B06910F06A
:1013F000800003F1FF33F7D073682C4945F0007586
:101400000B4045F480351D434FF42043A3647560C1
:1014100049F6FF7301E0991C33D0B06910F0020067
:1014200003F1FF33F7D04FF42043B262A3641A46AE
:1014300002E012F1FF322DD3B36913F02003F8D08C
:101440002023A264F3610120F8BD013B981CACD1BC
:10145000174A138801339BB24FF0FF311380A16408
:101460000020F8BDFFF70CFE7DE7FFF709FE5FE700
:101470000F4AA364138801339BB21380F8BD012087
:10148000F8BD0B4A138801339BB24FF0FF31138034
:10149000A164F8BD0649A2640A88013292B21846D6
:1014A0000A80F8BD6476002034220020009800FCF9
:1014B000142D0020427A02B9704710B50446036823
:1014C000406804F10A0198470023637210BD00BF11
:1014D000437A5A1C0344D2B242729972037A9342FD
:1014E00000D802B9704710B504460368406804F19B
:1014F0000A0198470023637210BD00BF98B10B4BDF
:10150000012210B402FA01F103F1750402E0033381
:10151000A34209D01A788242F9D15A780A42F6D009
:1015200001205DF8044B70470020FAE7646103086E
:1015300030B40A4D002305F10C0401E0272B09D03B
:1015400003EB43020133A15C8142F7D12A4430BC52
:10155000907B7047002030BC704700BF5861030883
:101560002DE9F341056906460F467DBBD0F80080A2
:10157000C8F30A0323B30023D6F8008001931FF0B9
:10158000D5FC042819D1224C236943F001032361BF
:10159000BBB2A8F800301FF0C9FC04282ED108F116
:1015A00002030193019B3F0C1F801FF0BFFC2369C6
:1015B000042823F00103236125D06FF0010505E025
:1015C0001FF0B4FC042805D04FF0FF35284602B0C8
:1015D000BDE8F0810E4C236943F002032361C4F897
:1015E0001480236943F0400323611FF09FFC2369AB
:1015F000042823F002032361BDD0E5E7236923F02B
:1016000001032361D9E7336804333360DEE700BFA9
:1016100000200240F8B504460D468E180027B5425A
:1016200001D12069F8BDE368591CE160234415F835
:10163000012B1A720429F2D1A1682046FFF790FF0E
:10164000E7602061EBE770B5448806460D46C4F3B9
:101650000B0422460021284624F037FC33690A4A4D
:10166000934209D3094A934206D222462846194694
:10167000BDE8704023F098BA23B121462846BDE862
:101680007040184770BD00BF0CC60308F4C60308BD
:10169000064B07498B4202D30023184670471A882D
:1016A000C2F30B029042F8D01433F3E798C1030859
:1016B0000CC60308024A136823EA00001060704752
:1016C0006082002030B4034600F12405064C07CCAC
:1016D0000C3343F80C0C43F8081C43F8042CAB42C1
:1016E000F4D130BC704700BFDC610308034B33F812
:1016F0000C2F02809B788370704700BFDC61030869
:10170000084B196861B130B45D68074C642202FB74
:1017100005F2B2FBF1F2228030BC00201860586064
:10172000704700BF80220020182D00200B4A13684C
:1017300003605368436030B59368094C836014219B
:10174000002301FB03429579AD0602D51379C372DC
:1017500030BD01330C2BF4D130BD00BFEB61030869
:1017600018860308704700BFF0B53B4B5B79012B2F
:1017700083B03AD0022B0FD0384B00221A805A8007
:10178000374B1B78022B05D1344A364B51881288CF
:1017900019805A8003B0F0BD334B1B681B01EFD595
:1017A000FF200DF009FE03780A2B51D8B0F9022072
:1017B0002E49D31781FB0212C3EBA2039BB207EEA3
:1017C000903AB8EE670A2A4C04F10C006381EEF7F8
:1017D0006BFEFCEEC07A214A6389CDED017A53801D
:1017E000BDF8043023811380CAE7224A224B927845
:1017F0001F4D33F81240A4B207EE904A05F13400B1
:10180000B8EE670AEEF750FE1C4A14491078967835
:101810005378FCEEC07A00EB4010CDED017ABDF8B4
:10182000042044F6FB77C3EB033300FB027200FB9A
:101830000474B2FBF3F2B4FBF3F3B2FBF6F2B3FBC6
:10184000F6F392B29BB22A866B860A804B8097E7AA
:101850009FED0B0A0023B6E7A8400020D43E0020ED
:10186000CC3D0020D03D00201C50002067666666FD
:10187000802200203C7600205C760020F980002049
:1018800000000000F8B5314D31496879314C324BD8
:10189000324E042264270A7001284FF0000184F8B8
:1018A000582084F86170A4F85A10A4F85C1084F8E9
:1018B000601061663170198059802DD002280ED0D9
:1018C000A979274A00230229136084F868305360FD
:1018D000936034D004292DD001290ED0F8BD2822E0
:1018E00004F1080024F0F1FA4CF250319FED1D0A8A
:1018F00004F10C00F0F7A8FDE2E71B4AE366536031
:101900009360D3609FED190A02F110004CF2503140
:10191000BDE8F840F0F798BD282204F1300024F02B
:10192000D4FA4CF250319FED0F0A04F13400F0F775
:101930008BFDC5E70E4AC4F8AC305360F8BD0D4AC4
:10194000C4F8A03053609360F8BD00BFA8400020E9
:101950005478002080220020D43E0020EA3E00205F
:10196000B8400020CDCCCC3DEC220020CDCCCC3EEC
:101970002C23002020230020F8B5264C94F8B43006
:10198000002B46D094F8B530002B42D094F8B630F6
:1019900003F0FF07002B3CD1D4F8B830C31A002B5A
:1019A00037DB1D4B1D491B780625013B05FB031248
:1019B0000A26128CB2FBF6F2D4F8BC6006F1010ED6
:1019C0000E4405FB031196F82E60CB8BC4F8BCE0E7
:1019D000724318441044BEF10E0F88BFC4F8BC70A7
:1019E000C4F8B800F5F77BFA012384F8B6300C4B45
:1019F000D4F8C0201B8AD4F8C410536000234B6273
:101A00000B889BB243F001030B80136843F0010382
:101A10001360F8BD80220020347B0020DC610308C5
:101A2000407B0020044B587920B1044B18780030DB
:101A300018BF0120704700BFA8400020EA3E0020E8
:101A40001F4B1878002839D01E4A1389FBB11E4A53
:101A50009FED1E6AD2ED026A07EE903AF8EEE66A52
:101A6000F8EE677A07EE103A77EEE66AB8EEC77AD4
:101A700066EE866AC6EE877AFDEEE77A17EE900A82
:101A80006428A8BF642020EAE070C0B2704710B498
:101A90000F4B54781B88117804FB1032091B642308
:101AA00000FB01F003FB02F3B3FBF0F06428A8BFD6
:101AB00064205DF8044B20EAE070C0B2704700BFBC
:101AC000EA3E0020A8400020B84000200000C842A4
:101AD000D43E00202DE9F04F794D81B0F5F728FF75
:101AE000D5F8CC400022C5F8C820002C00F0A58015
:101AF000237D052B074617D9216A23690B44C31A96
:101B00009342B8BF05F1CC010ADBD5E0137D052B6C
:101B10000AD9136A12691344FB1A002B80F2CC8095
:101B200051F8042F002AF1D14FF0010B0023B946E0
:101B30001E46C5F8C83098469A46274623E07A6A7A
:101B400039693B7DA9EB0204B4FBF1F40134A4B282
:101B500013FB04F3013301369BB2B6B23C83FB8224
:101B6000984506D2BBF1000F01D1012C5FD99846F0
:101B7000BA46D5F8C830013305EB8302C5F8C83042
:101B8000D2F8CC7047B3BB68C3B1FC8A002CD6D165
:101B9000396A4846A9EB01019847D0B195F82C3134
:101BA000002B52D13B7DC7F82490013601334FF012
:101BB0000102B6B23A83FB820124D1E73B6A3A695B
:101BC000A9EB0304B4FBF2F4A4B23C8334BBFB8A5C
:101BD000C6E73C83FB8AC3E72B686A68394901334F
:101BE00016443C4685E848004F46C1F800A0BAF1CB
:101BF000000F27D0DAF8203095F82C21AAF81640EB
